:020000040800F2
:10000000F0FF022045B505088DB5050869E3010834
:100010008DB505088DB505088DB5050800000000F3
:100020000000000000000000000000008DB5050881
:100030008DB50508000000008DB50508A59F0108D5
:100040008DB505088DB505088DB505088DB5050874
:100050008DB505088DB50508CDB00008D5B00008F0
:10006000DDB00008E5B00008EDB000088DB505086A
:100070008DB505088DB505088DB505088DB5050844
:100080008DB505088DB505088DB505088DB5050834
:100090008DB505088DB505088DB50508F5B00008C6
:1000A0008DB505088DB505088DB5050889D70008FB
:1000B00099D70008A9D70008B9D7000819A40008E3
:1000C0000DA4000861A4000855A400088DB505081A
:1000D0008DB505086D9801083D9901080D9A010834
:1000E000FDB000088DB505088DB505088DB505086E
:1000F0008DB505088DB505088DB505088DB50508C4
:100100008DB505088DB50508C9D700088DB505085A
:10011000DD9A0108AD9B01088DB505088DB5050870
:1001200095AD0008A9AD0008BDAD0008D1AD00082F
:10013000E5AD00088DB505088DB505088DB5050838
:100140008DB505088DB505088DB505087DD200086B
:10015000F9AD00080DAE0008000000007D9C01080C
:10016000A9A400089DA400080000000000000000F1
:100170008DB505088DB505088DB505080000000092
:10018000000000008DB505084D9D01081D9E010869
:100190008DB5050800000000000000000000000010
:1001A0000000000000000000000000008DB5050800
:1001B0008DB50508000000008DB5050800000000A1
:1001C000000000000000000000000000000000002F
:1001D00000000000000000008DB505088DB5050881
:1001E0008DB5050891D100088DB505088DB50508B8
:1001F00021AE000835AE000849AE00085DAE00082B
:0C02000071AE000885AE000899AE000841
:10800000B4224FF4A57C4FF4EB7182804FF4E172FF
:108010000023A0F802C0C1804FF4877C42819621E2
:10802000442203700381A0F80CC0C1810282438204
:10803000704700BF30B5EAB18E464FEA014C0346A7
:1080400000F1C005002419689A6841EA0C0142EA6F
:108050000E029A60C3E900140C33AB42F3D1D0F89E
:10806000C030C0F8C44043EA0E03C0F8C030C0F8C6
:10807000C84030BD4FEA014E8C46E0E710B40C4CCE
:108080002368002B11DD002004F1040C0146DCF80C
:10809000743003F1C00259600C339342FBD1236862
:1080A000013083420CF1AC0CF1DC5DF8044B7047FD
:1080B0001017002070B5474C04EB401393F8D02202
:1080C00002B970BD4C2202FB004294F8145694F899
:1080D00015E692F8B66383F8B66275454FF0000373
:1080E0004FEA401C82F8B6330CD00EEB4E0304EB83
:1080F000C30393F81826561E012E4FEA4E035BD990
:10810000032A53D004EB0C00A0F8B412EFF3118251
:10811000902383F3128890F8B632B0F8B41243EA91
:1081200041030021D2B29BB280F8B61282F31188CB
:108130001A0994F8781682EA13225A40D1B1D0F87D
:10814000CC42D0F8B812646FD2431B019BB202F04C
:108150000F0201208840134304F1C0015A0013F4B8
:10816000004F93B202D16268024362600C348C42C9
:10817000F4D170BDD0F8CC12D0F8B8024C6F1B010E
:1081800000F110019BB202F00F020120884013435E
:1081900004F1C0015A0013F4004F93B202D1626897
:1081A000024362600C34A142F4D170BD0EF10102B1
:1081B00002F00302AA42A5D0734404EBC30318449F
:1081C00090F8251600299DD004EB0C03012283F8BA
:1081D000B62297E710170020704700BF704700BF16
:1081E000024B03EB401090F8D102704710170020AB
:1081F0004368826C10B49A61EFF31182502383F3C9
:1082000012884168C46B0B6823EA0403446C23435F
:10821000D2B20B6082F31188D0E90741826803690A
:1082200012681C605960D0E909419C60D960B0F8BF
:108230005C10D16200235DF8044B0376704700BFE9
:10824000026890F810C01168022303FA0CF3194277
:1082500000D1704710B4074C41684FF0000C84F80F
:1082600079C608686CF3000008605DF8044B536041
:10827000704700BF10170020704700BF0B4890F8F0
:10828000B01689B101EB4101002310B4490000F59B
:10829000D7601C4650F82320063302B114608B428D
:1082A000F8D15DF8044B7047704700BF10170020ED
:1082B0000B4890F8B01689B101EB4101002310B4CE
:1082C000490000F5D7601C4650F82320063302B160
:1082D00014609942F8D15DF8044B7047704700BFB5
:1082E0001017002001207047034B00EB400003EB08
:1082F000C00090F8C9067047101700201F4890F87A
:10830000B036CBB300222DE9F04100F5D7631C4F06
:1083100050262C25144607E053F8181B0C6090F8E3
:10832000B0160132914225DD197C0029F4D059683C
:108330004FEA912EAEF5801EBEF1530F4FF0FE0CAA
:1083400098BF17F80EC0EFF3118E86F31288D1F89C
:10835000248005FB0C0C08F10108CCF8A087D1F8AB
:10836000148048F001085FFA8EFCC1F814808CF389
:108370001188D1E7BDE8F081704700BF10170020D9
:1083800080CD050807EE900AB8EE670A704700BF77
:10839000BCEEC00A10EE103A98B2704708B51D2026
:1083A00010F050FF08B183794BB11E2010F04AFF46
:1083B00008B1837903B108BD5523C38008BD552397
:1083C000C380F2E7704700BF704700BF704700BF2F
:1083D000704700BF01207047094A0A4BD2F8BC29F8
:1083E000D3F89002526AD3F8941292F85330012BCA
:1083F00008BFB2F85030A0EB010008BFC0187047AA
:108400001017002008280020012380F85130704701
:1084100010B4EFF31181802383F312880C4AC9B2A0
:10842000D2F89832D2F89C42D2F89802D2F89C2224
:1084300081F31188904203F1FF33A3EB04038CBF57
:108440000020012003EBC0205DF8044B704700BF03
:10845000082800204A4B4B4A1B6893424CD015D940
:10846000494A934251D027D9484A934256D002F103
:10847000B77202F5585293427DD1454BD3F8A420F0
:108480000B2161F30F32C3F8A4207047414A934295
:108490004DD020D9404A934252D002F1B77202F532
:1084A000585293426AD13A4BD3F8A420052161F384
:1084B0000F32C3F8A4207047384A934249D0384A53
:1084C00093425AD1324BD3F8A420062161F30F32E4
:1084D000C3F8A4207047334A934243D002F1B772E5
:1084E00002F55852934247D1294BD3F8A4206FF399
:1084F0000F32C3F8A4207047254BD3F8A4200421E1
:1085000061F30F32C3F8A4207047214BD3F8A420A5
:10851000092161F30F32C3F8A42070471C4BD3F834
:10852000A420082161F30F32C3F8A4207047184B30
:10853000D3F8A420032161F30F32C3F8A4207047BD
:10854000134BD3F8A420022161F30F32C3F8A42007
:1085500070470F4BD3F8A420072161F30F32C3F803
:10856000A42070470A4BD3F8A420012161F30F32F5
:10857000C3F8A4207047704770477047704700BF2A
:1085800000000020007A030A001C4E0E0052BC0FAF
:108590000038024000D8B805000E270700B0710B64
:1085A00000E6DF0C006CDC02074BD0F894105B682F
:1085B000D0F8A0205B1A9A42B8BFC0F8A0300123BF
:1085C00080F8CC3000207047001000E003689A6902
:1085D000D10508D54FF4807213218177DA611A68CA
:1085E00022F080021A609A69920508D54FF4007251
:1085F00013218177DA611A6822F080021A609A6981
:10860000510508D54FF4806213218177DA611A6829
:1086100022F080021A609A69120508D54FF40062B0
:1086200013218177DA611A6822F080021A609A6950
:10863000D10408D54FF4805213218177DA611A688A
:1086400022F080021A609A69920408D54FF4005211
:1086500013218177DA611A6822F080021A6070476C
:10866000184BD3F8A012D3F8A4228A1A322A15D8AC
:10867000D3F8B8228A4200D37047D3F8A822E2B1D7
:108680001068928810B44469224218BF1204323133
:108690005DF8044B8261C3F8B8127047D3F8A82282
:1086A0003AB193F8B40291881268C00748BF090430
:1086B00091610022C3F8B82270473231C3F8B81272
:1086C000704700BF08280020064AD2F8A8323BB104
:1086D00092F8B4129A881B68C90748BF12049A61BD
:1086E00000207047082800204FF40070034B1060F2
:1086F000D3F8C8320B600020704700BF0828002064
:10870000002070470120704701207047002070470B
:108710000123437700207047D0E90B2108B5836916
:108720000B4483610AB108469047002008BD00BF92
:10873000436A1B681B6A5B685B78024613F00100A2
:1087400008BF5077704700BF70B5224A224C234BB8
:1087500094B00546CDE90042214A0992A4F10802ED
:108760000A922A7F0493201D0023CDE905039A4233
:10877000CDE90E330B931093139314BF05200420FF
:1087800011936B6A0C9002200122029018688DF8F8
:108790000C200E4607928DF820208DF834208DF89D
:1087A000482051F021FB2B7F93B1330E04F8073C96
:1087B000063C320C330A22706370A670686A694600
:1087C0000FF000FE6B6A186851F00EFB14B070BD1C
:1087D000073CEEE7002B00200C000020318700084A
:1087E0001187000810B5044694B050220649684627
:1087F00054F0FEF9606A69460FF0E4FD636A186898
:1088000051F0F2FA14B010BDD4CD0508C2628161F6
:10881000704700BF2DE9F0410446406A00681E46DB
:108820000F46904651F0E0FA237F002B37D0254DBC
:10883000A0690523EB64030E6B7505F116039870B0
:10884000020C000A58701A703B68AB650020D8F81B
:1088500000302B66012E2363286727D0022E1CD1FF
:10886000D8F80420A866796885F86400E96613449E
:1088700015496A670120236385F87800E967134B7F
:10888000617F606A03F11402002914BF1946114682
:108890000FF098FDE36A83B1206BBDE8F081094DCC
:1088A000A0690423EB6405F11503C8E7064B85F8BE
:1088B0006460C5E91A306867E1E7636A186851F0D7
:1088C00093FAE9E700000020198700081C00002047
:1088D000704700BF00B583B081610192049A009394
:1088E000C26201236A4601A9FFF794FF03B05DF855
:1088F00004FB00BF043070470D4B93F80023D3F8FE
:10890000FC120244D2B283F8002393F800230844F7
:108910001206C3F8FC0205D593F8002382F080020A
:1089200083F80023034B012283F89420704700BF93
:1089300008280020000000202DE9F047144FD7F848
:108940000453ED0A1ED00026B04607F54F79D7F83C
:1089500008331048D3F828A0C7F83483AC19641042
:1089600010234A46E102D0470F280BDD0A4B03F1E2
:10897000100C53F8041B013107D16345F9D125468A
:10898000B542E4DCE802BDE8F087661CF8E700BF0A
:1089900008280020102B0020442B0020012141F248
:1089A0000102002341F2011C017202804FF60B719B
:1089B000FF22A0F804C043818381C38101828274B5
:1089C000704700BF164BFF224FF0FF3CF0B5C2705E
:1089D000027102724272427382738274C27403F132
:1089E00012076646172516244FF0150E002202EBDB
:1089F00082028118BB4200F802E04C708D70CE708C
:108A000081F804C00BD093F9062093F807E01C7A94
:108A10005D7A93F90A6093F90BC00633E7E7F0BD7E
:108A200024CE05084FF0000C01210222032380F818
:108A300005C08171C2710372704700BF4FF4F071BD
:108A400040F22E4C01804FF47A71A0F81EC0418490
:108A50004FF4FA6C4FF4F5610122A0F820C0818434
:108A600040F2262C42F22011A0F81CC0418142F2B3
:108A7000267C0E218271427440F201220723A0F865
:108A800008C080F826104FF0000C40F203418282AB
:108A900040F205628370A0F812C0C182028383761F
:108AA000704700BF002306214FF47A72C0E901230A
:108AB00001700373704700BF10B50023411CFF22F3
:108AC00000F8132001F8132001330B2BF8D10C4BC5
:108AD0004FF0FF3103F1180400228C4605E013F932
:108AE00002CC13F9011C13F8032C00F812C000EBA0
:108AF000420E03339C428EF80110F0D110BD00BF2E
:108B00003FCE05084FF0260C2721022280F800C036
:108B1000C1704FF0200C0321427180F806C0C27171
:108B20004FF0210C0172827204212C22012380F863
:108B300009C0C1724FF0000C02731221FF22437072
:108B400083700371437380F80EC0C1730374427461
:108B5000704700BF03230370704700BF704700BF1A
:108B6000D0ED007AD0ED016A30EE677AE6EE877AD2
:108B7000B0EE670AC0ED007A704700BFD0ED017A11
:108B8000D0ED026A30EE677A90ED000AE6EE877A61
:108B900037EEC07AC0ED017AA6EE870A80ED000AB2
:108BA000704700BF90ED017AD0ED036AD0ED027AF4
:108BB00030EE470AA6EE807A90ED000A80ED017A49
:108BC00037EE676AE6EE867A37EEC07AC0ED027A53
:108BD000A6EE870A80ED000A704700BFDFED277A16
:108BE000B4EEE70AF1EE10FA0CDDDFED256A9FED39
:108BF000257AF0EE407AF4EEC77AF1EE10FA30EE14
:108C0000660AF6DCDFED207AB4EEE70AF1EE10FA40
:108C10000CD5DFED1B6A9FED1D7AF0EE407AF4EE85
:108C2000C77AF1EE10FA30EE260AF6D4DFED187AA4
:108C3000B4EEE70AF1EE10FA14DDDFED107A37EE4C
:108C4000C00A60EE006A9FED136A9FED137ADFEDB4
:108C5000137AA6EE867A20EE266AE6EE877AA6EEEC
:108C6000270A7047DFED0E7AB4EEE70AF1EE10FA4C
:108C700044BFDFED057A37EEC00AE2E7DB0F49407B
:108C8000DB0FC940E4CB1641DB0F49C0E4CB16C172
:108C9000DB0FC93F92E741B99730083C15A82ABEBF
:108CA000DB0FC9BFD0ED056AD0ED017A90ED007AF7
:108CB00090ED066AD0ED025A90ED035A80ED050A58
:108CC00066EEA77AC0ED066AE7EE007A90ED077AC5
:108CD000E5EE867A90ED086AD0ED045A80ED087AC8
:108CE000E5EE477AE5EEC67AB0EE670AC0ED077AA0
:108CF000704700BFD0ED057A90ED006A90ED067ADE
:108D0000D0ED035AE6EE007A90ED016AF0EE406A8B
:108D1000A6EE267AB0EE670AD0ED047A90ED026AEC
:108D200067EEC07AA5EEC07AE6EE267A80ED057A87
:108D3000C0ED067A704700BF2DE9F047089F3C461A
:108D40000E4614F8011B002B054614BF4FF03009E6
:108D50004FF0200941B3002A2CDD234600E0B2B1D8
:108D600013F8010B9046013A0028F8D1A8F1020847
:108D70006AB1C24649462846B0475346002B0AF11D
:108D8000FF3AF7DC397828EAE872013249B1D71B9B
:108D90002846B047E01914F8011B0029F8D1BDE8B6
:108DA000F0871046BDE8F087002A02F1FF38E0DCCA
:108DB0000846F4E70022EAE703685A1C02601970CB
:108DC000704700BF024BD3F84C0303681B68184779
:108DD0000828002030B4436919690A686FF300025B
:108DE0000A609A68B3F80CC01468E26822EA0C02C0
:108DF000E260046890F810C02068082202FA0CF2C1
:108E000002403AD1224890F87856022000FA0CF03D
:108E10006060002D2FD0187E01282FD0D3F8A0102D
:108E20000131C3F8A010EFF31180502181F31288B3
:108E30005C68DD6B216821EA05011D6C2943C0B225
:108E4000216080F3118898681969DC6A00680C60F9
:108E50001C6B4C605C6B8C609C6BCC604262B3F8AA
:108E60007C20C2620A68012422430A601C76C26820
:108E70009B891343C36030BC7047FEE7D3F8A4005E
:108E80000130C3F8A4000B6862F300030B60F2E743
:108E9000101700201A4A0368934210B504460AD0FE
:108EA000184A934213D0184A93421CD01A6842F0D1
:108EB00001021A6010BD154849F0CAFD1449236823
:108EC000D1F8202822F40012C1F82028EEE711483A
:108ED00049F0BEFD0E492368D1F8202822F4800213
:108EE000C1F82028E2E70C4849F0B2FD08492368A0
:108EF000D1F8202822F40002C1F82028D6E700BFCC
:108F00000054004000580040005C00401500200064
:108F10000030024016002000170020003D220223EE
:108F200002704370704700BF4FF4007141F201427C
:108F3000002340F21F4C0180428040F68C21012228
:108F4000A0F806C0038143818181C281704700BFC0
:108F500010B5084C084849F07BFD4022002104F57B
:108F6000547053F0A8FE4FF0FF33C4F89033C4F8A8
:108F7000933310BD082800200E004400114B00213F
:108F800030B50160818003F10C054FF448748E46C2
:108F90000A4602EB420200EB420C00F812E08CF8A9
:108FA0000110DA788CF80220AB42ACF8044007D00C
:108FB00093F9062093F807E0197A5C890633E8E70D
:108FC00030BD00BF54CE0508F8B5164D1648174FF2
:108FD00000214FF40F7253F06EFE05F644364FF049
:108FE000804105F628343A46002301E054F8332046
:108FF00091420BD001330F2BF8D100201C354FF0DC
:10900000DFFCB5420CD055F81C1CECE7084A02EB1B
:10901000C3031C3593F8300C4FF0D2FCB542F2D1AB
:10902000F8BD00BF84CE0508881E00200000014066
:1090300080CD050810B5044653F03EF881B22046B5
:10904000BDE81040FFF736B838B50B4D00EB4000D7
:1090500005F5D76303EBC00393ED027AD3ED037AF2
:10906000E7EE007AC4002C44B0EE670A53F024F80F
:10907000D4F8B836186038BD101700202DE9F84331
:1090800010F0DCFF204F214E05464FF000094FF055
:10909000AC083C68002C2ADD00231A4608FB03714B
:1090A000013391F8A1109C4242EA0102F6D142EA52
:1090B0000904E4B291467368C3F30803A3B9EFF35C
:1090C00011838BB914F01CFA431BB3F5FA6F02DC61
:1090D000B9F1000FDDD124B10D4B93F89723542A39
:1090E00009D02046BDE8F88310F07AFFECE74C4643
:1090F0004FF00009DFE7B3F89C230132A3F89C236B
:109100002046BDE8F88300BF1017002000ED00E006
:1091100008280020C94B93F878360BB90120704716
:109120002DE9F04FC64FC749D7F8A022C64BA1FB87
:1091300002125209A3FB023B4FEADB0B0BEB8B0B3A
:1091400085B0A2EB4B0B5FFA8BF3039307F5D1636A
:109150000193BA4B07F56A7A03F52D7900230AEBE0
:109160008B0B1D46D7F89837AB4240F31A81D9F8DC
:109170001830D9F80460D3E9258410F05FFF4FEA76
:10918000860E0EF1085E0EEB481E97F8978302904C
:1091900004F1806197F890073939B8F1540F0EEB5C
:1091A00081110EEB801301D1A7F89E03994240F282
:1091B0006B811A68002A00F05F811A6C002A00F0A7
:1091C0007181D3F88020002A00F06E81D3F8C0208E
:1091D00003F58073002AE9D1A3EB0E0E99424FEA02
:1091E000AE1E40F25181A4EB0E0145294FF0000460
:1091F00028BF452103EB81119C46204626460DE001
:109200001A6C002A40F0D480D3F88020002A40F065
:10921000FA80D3F8C02003F580732AB9994206D9A1
:109220001A68002AECD04033994200F2C580112E12
:10923000344640F22D81D6F1150200F1298183498F
:10924000029ED1F898309E45D7F8943738BFC1F8C0
:1092500098E0F11A002919DB03F5F42303F5907364
:109260009E4288BF029B794988BF0533C7F894376F
:10927000764BD3F89830052B86BF053BDBB2002335
:1092800087F890374FF0FF33C1F8983042B100FAB9
:1092900002F2C4F11404012000FA04F444EA0200CA
:1092A0006B4BC0F3C43203EB8202D2F8A44C00F043
:1092B0001F0203EB8202D2F8A41CC0F3441203EB9A
:1092C0008202C0F3842003EB8000D2F8A43C41EA80
:1092D000043141EA0311D0F8A43C41EA032181EAB8
:1092E000112383EA131303F00F030F2B40F0B48014
:1092F000B1F5803F80F0B080B8F1540F4FEA111102
:1093000004D1B7F898330133A7F89833D7F89036DB
:10931000B1F5606F03F10103C7F8903600F0D58016
:10932000019B99819AF858300398834214D0DBF856
:109330000820DAF800309B1ACAF80030DBF8302039
:10934000DAF804309B1ACAF804300023CBF808304E
:10935000CBF830308AF85800DAF800300133CAF818
:109360000030DBF808300133CBF808304FF6FF73DC
:10937000994209D1DAF804300133CAF80430DBF835
:1093800030300133CBF83030019B01351433082DD8
:109390000AF15C0A0BF15C0B019309F120097FF4DF
:1093A000E1AE0123012087F88C3705B0BDE8F08FCE
:1093B000803399427FF63BAFA3EB0C029211541C11
:1093C000244A82FB04C2A2EBE472012AB8BF012244
:1093D000904001241644013A04FA02F210431C465C
:1093E000226892B1226C002A60D0D4F88020002A32
:1093F0005ED0D4F8C02004F580743AB1A142EFD811
:109400009C4623460AE7C0330EE74034A142F7D911
:10941000E31A9B115A1C0F4B83FB02C3A3EBE273AD
:10942000012BB8BF012398401E440122013B02FAE0
:1094300003F3184323469C462346EFE6101700200B
:10944000082800201F85EB51CDCCCCCC000000209B
:1094500080CD050856555555B8F1540F2AD0D7F888
:1094600090360133C7F89036D7F88C360133C7F8F9
:109470008C364FF6FF7155E74033A3EB0E0E994241
:109480004FEAAE1E3FF6AFAE10B1013887F8900735
:10949000B8F1540F7FF478AFB7F89A330133A7F8D7
:1094A0009A3371E7803397E6C03395E68034ADE7B1
:1094B000C034ABE7B7F898330133A7F89833D7F83F
:1094C00090360133C7F89036CEE7084A92F8153641
:1094D00003EB430302EBC3032B4493F825360D2B18
:1094E0007FF41EAF019A802393771BE710170020AB
:1094F000F8B51F4E96F8142696F815369A4231D1D3
:109500003568002D12DD002496F878661948274644
:1095100006B3037E012B20D002691368013443F0A7
:109520000103AC4200F1AC001360F1D110F086FDF4
:10953000114BD3F89C47002C0BDD03F5F46303EBD0
:10954000C40419689A88C86808330243A342CA60F1
:10955000F7D1F8BDFEF74CFEDEE780F89C70FEF711
:1095600047FED9E74FF0B6F80028C9D1F8BD00BFD3
:1095700010170020141700200828002038B51A4BB7
:1095800093F8142693F815369A4228D1174D95F87A
:10959000C0371BB34FF0000C05F2C472614613686C
:1095A00059621868083261F3C710186032F8040C69
:1095B000D862186840F080001860186861F34100B4
:1095C0001860DC6832F8020C95F8C0E70CF1010C69
:1095D0002043E645D86022F8021CE0DC38BD4FF09D
:1095E00079F80028D2D138BD1017002008280020B3
:1095F0000C4AF8B5136855692B4003EA000555611C
:109600007DB1094F0126B5FA85F4C4F11F0407EBBB
:10961000840306FA04F4D3F8500303689847A5437B
:10962000F1D1F8BD003C0140082800200269C36860
:109630002DE9F04712EA03092AD005460E464FF0FD
:1096400000474FF00008B9FA89F327FA03F2D24332
:109650001B3B2A6109EA0209042B16D8DFE803F054
:10966000332A221A0300B36A002B35D003F1FF3AE4
:109670001FFA8AFAC6F82880746A34B12368204633
:10968000514698476468002CF8D1B9F1000FDAD13F
:10969000BDE8F0877068A98E03689847B9F1000F9C
:1096A000D1D1F5E7B068298F03689847B9F1000F69
:1096B000C9D1EDE7F068E96B036889B29847B9F161
:1096C000000FC0D1E4E73069296C036889B298477C
:1096D000B9F1000FB7D1DBE7E96A1FFA81FACBE7EE
:1096E00030B5124A124CD2F8303883B043F001033F
:1096F000C2F830384FF4C0554FF0817369462046A8
:10970000CDE9005349F03AFA636A23F470236362A7
:10971000636A43F420236362636A23F470436362E1
:10972000636A43F42043636203B030BD00300240FB
:10973000000002402DE9F04704460068237C0268DF
:10974000022101FA03F31A4201D1BDE8F087D4F8EF
:1097500014A0DFF878829C4ADFF874925268C9F846
:1097600004284C2707FB0A87D7F8BC23B7F8C01397
:109770001668D7F8F453F26822EA0102F2602A6808
:109780006FF300022A6098F8782612B94360BDE8AA
:10979000F087284649F06AF9D9F80C38012287F891
:1097A000E023002B00F00A8133686FF3C7133360A6
:1097B0004C2303FB0A834FF0FF3293F8F033F2623D
:1097C000062B29D8DFE813F0D2002800AA002800D1
:1097D000820028000700336A6FF30C3333624C2396
:1097E00003FB0A83326A93F8F11361F34D3232625C
:1097F000F26993F8F21361F30922F26193F8F3230B
:10980000F36962F30F33F361F3696FF38B23F36151
:10981000336A43F4805333622A684C2303FB0A8380
:109820004BF6EF7002400020A3F8D4032A602968A9
:10983000B3F8D4230A432A602A6893F8DD1361F34E
:109840000D322A602A6893F8DB1361F38B222A60B9
:109850002A6893F8DA1361F309222A602A6893F8D8
:10986000D91361F3C7122A6093F8D8132A6861F3F9
:1098700086122A6093F8DC132A6861F345122A6085
:10988000B3F8D6136A6861F30F026A60D3F8CC2389
:10989000AA60D3F8D023EA60D3F8F42316215160EC
:1098A000116841F001011160D3F8BC23B3F8C03353
:1098B00012682068D1680B43D360434A237C516807
:1098C000C9F80818022202FA03F35FE7336A6FF35C
:1098D000082333624C2303FB0A83316A93F8F12394
:1098E00062F349213162316AC2F3400262F3CB2153
:1098F0003162F26993F8F21361F30102F26193F8B5
:10990000F323F36962F30713F361F3696FF38303DE
:10991000F361336A43F4807333627DE7336A6FF334
:10992000041333624C2303FB0A83316A93F8F12357
:1099300062F345113162316AC2F3400262F3C7112A
:109940003162B26993F8F21361F30922B26193F8BC
:10995000F323B36962F30F33B361B3696FF38B23FE
:10996000B361336A43F01003336255E7336A6FF330
:10997000000333624C2303FB0A83316A93F8F1231B
:1099800062F341013162316AC2F3400262F3C30102
:109990003162B26993F8F21361F30102B26193F894
:1099A000F323B36962F30713B361B3696FF38303FE
:1099B000B361336A43F0010333622DE710F03EFBDD
:1099C000C9F80C08F0E600BF001000E010170020F6
:1099D0000828002038B51E4CD4F8903273B1D4F862
:1099E0009422D4F890329A4208D0D4F89432E218F3
:1099F000013392F81008C4F8943238BD154BD3F8EF
:109A0000BC390022596AC4F8942291F8533003F00B
:109A1000FF05ABB1B1F8505081F853205DB193B25E
:109A2000C8182344007983F81008B1F850000132B7
:109A300093B29842F3D80848402204314AF076F9AC
:109A4000C4F89052D4F890020028CED1D5E700BFD8
:109A50000828002010170020C820002090F850305F
:109A60005A1C0344D2B280F8502083F83C1090F87E
:109A700051300BB1132A01D950F040BE704700BFDE
:109A8000002280F8512050F039BE00BF38B54AF0AE
:109A9000D3F9214B93F89D412922012C23F88A2CDC
:109AA00023F8822C01D0012038BD1C4DC3F8A051F1
:109AB000FFF716FE1A4848F0CBFFFEF7CBFC4EF03E
:109AC0005BFF184A02F580534FF0A04083F87843BB
:109AD00083F88543C2F8B409816B41F400118163B6
:109AE00005F1200205F148010F4DC3F87C534FF4F6
:109AF0000165A3F87A534FF481750024A3F88053CD
:109B000083F883434FF030FA224621464FF0FF306E
:109B100049F07CF8204638BD003900209C00002028
:109B20000700340010170020400040012DE9F043E9
:109B30000446406A354D006895B00E4691469846F9
:109B400050F052F9324B0193324B049305F58A736E
:109B50000093217F0223029305F5867201230027DB
:109B60008DF80C3005920697002937D08DF83430E7
:109B70008DF84830CDE90977330ECDE90E77CDE980
:109B8000107785F80D310523CDF82C908DF82070D5
:109B9000CDF83080139705F587750793330C1E4F6A
:109BA0002B70330A6B70AE70D7F8A801656A0EF09F
:109BB000C7FF637FA8803BBB05A928460EF002FCC7
:109BC000636A186850F010F9D7F8AC010EF0B8FFCE
:109BD000636A9880404615B0BDE8F0838DF8343054
:109BE0008DF848300423CDE90911CDE90E11CDE9F6
:109BF0001011CDF82C908DF82010CDF830801391F5
:109C000005F20D150793C9E76946D6E70000002065
:109C1000A43A002031870008003900202DE9F047E0
:109C2000089F884615460021202204461E4653F010
:109C300042F84FB13B68E3811B0C23827B687A8931
:109C4000E3821B0C62822383404650F07BFDEB06CF
:109C500019D4431EB8B108EB000701E0013B12D351
:109C600017F801CDBCF12E0FF8D1C01A421E032AFD
:109C7000A8BF0322082B03F1010AA8BF08239146BD
:109C8000C2441A4606E008280246C246A8BF082277
:109C90004FF000094FF0203341462360636004F128
:109CA0000807204652F0A4FF174B23815146BB7092
:109CB0004A46384652F09CFF611EE31D11F801CF61
:109CC000ACF1610EBEF1190F9CBFACF1200C81F814
:109CD00000C08B42F2D1384604F10B0110F8013B71
:109CE000A3F16102192A9CBF203B00F8013C884285
:109CF000F4D118232373330CA382E572099B668386
:109D0000E361BDE8F08700BF202020002DE9F04F7F
:109D1000DFF88094D9F8A002C9F8A40287B0002B1C
:109D200000F0D88001F5FE781344DFF86CB403939B
:109D3000164601F12007C2461FE0002E62D0D9F876
:109D4000D432B34200F0CA80D9F8D032B34200F026
:109D5000FD80D9E9B631B3424BD8B14200F29781C8
:109D6000711A20464CF07EFE039B01369E4207F599
:109D700000770AF5007A00F0AD80D9F8E052B542DC
:109D8000A7F12004D9D8751BD9F8F08205F0070295
:109D9000EB080492D8F830200233934203D3D8F86A
:109DA000382093420BD94146184605934CF02AFEC1
:109DB000059B8046002800F08A81C9F8F00298F8D7
:109DC0000420002A40F03281D8F82850002D00F0FD
:109DD0007781D8F830209B1A049A02EBC303D8F895
:109DE0000C20204602EB43224FF400714346A84763
:109DF000BAE7B142B4D920464FF40072002152F0C4
:109E00005AFFB1E74FF400723146204652F053FF3B
:109E1000802387F89E310C2387F8A231D9F8D032FD
:109E2000D34AD9F8C812C4F8C6319342C4F8CA114B
:109E300000F33281CF4AD04C82FB03021A44D81778
:109E4000C0EB621284FB0254CC4D85FB03C5C0EB12
:109E50002530C2EB821587F8A1015B1B801020F032
:109E60003F0001330343144487F8A031D317C3EBF9
:109E7000E4142244BE4B87F89F214A1E9A4200F305
:109E80001781BC4BBC4883FB02311144D317C3EB91
:109E9000611180FB0140B94C84FB0254C3EB2433B5
:109EA000C1EB811487F8A531121B9B1023F03F03EF
:109EB00001321343084487F8A431CB17C3EBE010F9
:109EC000014487F8A311552387F8DE31AA2387F8C8
:109ED000DF3149E7002007B0BDE8F08F4FF0FF33D6
:109EE00084F8EC3184F8ED3184F8EE3184F8EF3108
:109EF000D9F8E832C4F8E831522323706370612343
:109F0000A37084F8E73141230025E37084F8E6313B
:109F1000722384F8E43184F8E5314FF4F072294675
:109F2000A7F11C0052F0C7FE5523C7F8D051C7F85F
:109F3000D451C7F8D85184F8FE316FF0550384F836
:109F4000FC5184F8FD5184F8FF310DE700214FF4F6
:109F50000072204652F0AFFE894A03CA47F81D0C32
:109F6000EB2007F8200C582007F81F0C902047F82A
:109F7000191C07F81E0C002302220821F820E372A6
:109F8000227307F8131CA273E37307F8102C07F869
:109F90000B0CD9F8D00284F82C20D9F8C8226376AB
:109FA000121A2262D9E9B602121A3F2020764FF027
:109FB000FF30A0763E2020770120E3766377A377F9
:109FC000E37784F82D3084F82E3084F82F306262E5
:109FD00084F8300084F8313087F82610802187F823
:109FE0002010292187F82210942187F823100E21B0
:109FF00087F824100D21634A87F82510552187F82A
:10A00000DE11AA2187F8DF1103CA5F4BC7F82700CA
:10A01000C7F82B1003CB1388A7F82F309378C7F815
:10A020003200C7F8361087F831309DE64FF40072E1
:10A030000021204652F03FFE049B002B4ED1D8F861
:10A040004030002B00F0AA80049AD8F830304F49F5
:10A05000CDE9002220461122FFF7E0FDD8F840307C
:10A060001A6C002A00F0AD80049A1B6BCDE9002227
:10A07000474911223846FFF7D1FDD8F8448007F14F
:10A0800020044FF4E075B8F1000F3FD16CE6F11AEF
:10A0900020464CF0E7FC67E6FF2387F89F3187F8FE
:10A0A000A13187F8A031324B4A1E9A427FF7E9AEC0
:10A0B000FF2387F8A33187F8A53187F8A43102E799
:10A0C000294620464FF4007252F0F5FD4CE6A7F108
:10A0D000240343F804BF9A45FBD145E6D8F8403045
:10A0E000049AD8F84480002B0CBF01230223C3EB51
:10A0F00002154346002B3FF437AE013D9B6CF9D16E
:10A1000098464FF40075002B3FF42EAE25442034C2
:10A11000234620354446049698460EE05CF81C1B06
:10A12000236BCDF800C000260196FFF777FDA46CE5
:10A1300008F12008CCB1A84517D02379A44604F132
:10A140001C0E1122A8F12000002BE7D162792669AC
:10A15000236B216842F02102CDE900E6FFF75EFDA6
:10A16000A46C08F12008002CE5D1049EFCE500BF9A
:10A17000FF03FB0083200882818080809755454142
:10A1800004450608104506081C450608FC44060858
:10A190000045060808280020DEADBEEF049BD9F874
:10A1A000CC12CDE9003320460822FFF737FDD8F85E
:10A1B0004480B8F1000F3FF4D7AD3C464FF4F07542
:10A1C000A4E7049BCDE9003352E700BF38B590F80F
:10A1D0002830012B044604D0407F40B10023637730
:10A1E00038BD406A03681A7B92B9637F0BB90120BE
:10A1F00038BD0A4D0A49022305F5D8720EF000FA5F
:10A2000095F8B13103F0010383F001006377E7E7CC
:10A210001B6A002BE9D0002038BD00BF00390020A8
:10A22000180100202DE9F0410446154E90F8280051
:10A23000637F144F06F5D878012805D00BB10023B1
:10A2400063770120BDE8F081606A05682A7B82B9E6
:10A25000002BF6D00223424639460EF0D1F996F88B
:10A26000B13103F001036377002BEAD094F82800A2
:10A27000E2E72A6A002AE8D1002BE2D0EAE700BF31
:10A280000039002018010020F0B511F0010583B05D
:10A290000AD190F82860012E044607D0C368B3F1B4
:10A2A000807F01D90123237703B0F0BD0A4B476AB1
:10A2B000D3F8A8010EF044FCE368B880B3F1807FC6
:10A2C000F2D9B7218DF80410267733462A4638464E
:10A2D00001A90EF095F9E7E700390020144B154964
:10A2E00010B5044618681B79206284F824301522C2
:10A2F00004F1250052F030FD0F4B93F8B2214FF0DE
:10A30000010E84F83AE012B984F83B2010BD03F541
:10A31000DA7CBCE80F0020606160A260E360BCE80A
:10A320000F0084F83BE020616161A261E36110BD30
:10A3300028450608304506080039002010B50021E0
:10A340003822044652F0B7FC0D490E4A0E482061EF
:10A35000C4E905120D480E4AE061012341F61E6171
:10A360004FF0090CE18484F808C0A37384F821300D
:10A37000A26221460748BDE8104035F0CDB800BFC5
:10A380001A046C07001975036400DC0543080E000D
:10A390001E7D010140450608174A1849D2F8883049
:10A3A00030B443F47003C2F888300B6843F0010303
:10A3B0000B600B689B07FCD58B68104A6FF3010399
:10A3C0008B60936813F00C0FC3F38101F9D1916096
:10A3D000136809480A4D23F0867323F48033136011
:10A3E0004FF41F044FF000635560C2F8A010D46012
:10A3F00030BC8360704700BF00ED00E000380240D1
:10A4000002300300704700BF002070470148FEF78C
:10A41000DDB800BFEC3A00200C4BD3F80432023B0D
:10A42000072B11D8DFE803F00D0D0A0A0707040413
:10A4300007484FF013BF06484FF06CBF04484FF079
:10A44000E7BF034850F08CB8704700BF00390020C8
:10A45000EC3A00200148FEF7B9B800BF403B0020AD
:10A460000C4BD3F85832023B072B11D8DFE803F02E
:10A470000D0D0A0A0707040407484FF0EFBE06480F
:10A480004FF048BF04484FF0C3BF034850F068B8CE
:10A49000704700BF00390020403B00200148FEF714
:10A4A00095B800BF943B00200C4BD3F8AC32023B74
:10A4B000072B11D8DFE803F00D0D0A0A0707040483
:10A4C00007484FF0CBBE06484FF024BF04484FF07A
:10A4D0009FBF034850F044B8704700BF00390020C8
:10A4E000943B0020F0B40668D6E9041574684A6805
:10A4F000A36813F08003FBD1002D00F09080686109
:10A500000F7CD1F800C06968022000FA07F747F015
:10A510000C07CCF804702F7C2D68B84040F00C007C
:10A520006860106863F300001060086863F300005F
:10A5300008600B68B06943F002030B6013684BF6C8
:10A54000EF752B401360176803893B431360136852
:10A55000477C67F30D3313601368C77B67F38B2366
:10A560001360877B136867F309231360477B1368C5
:10A5700067F3C7131360077B136867F386131360D1
:10A580001368077C67F3451313605368478967F3C3
:10A590000F035360F369066840689660D0600868EE
:10A5A000284008600D6818892843086008685D7CA9
:10A5B00065F30D300860DD7B086865F38B2008606B
:10A5C0009D7B086865F3092008605D7B086865F37A
:10A5D000C71008601D7B086865F38610086008686E
:10A5E0001D7C65F34510086048685D8965F30F00C0
:10A5F0004860D3E900038860CB600B6843F0010337
:10A600000B60136843F001031360636843F00103B8
:10A610006360636843F002036360F0BC70474861A5
:10A62000087C09680223834043F00C034B601368E5
:10A6300065F3000313601168B3694BF6EF700140D6
:10A64000116010681989014311601168587C60F32A
:10A650000D3111601168D87B60F38B211160116896
:10A66000987B60F3092111601168587B60F3C71172
:10A6700011601168187B60F386111160187C1168F5
:10A6800060F3451111605889516860F30F01516002
:10A69000D3E900139160D360136843F001031360A2
:10A6A000136843F002031360636843F002036360BE
:10A6B000F0BC7047F8B505462C6895F838706368AB
:10A6C000012284F824201A686FF386121A60A88881
:10A6D0002289824219D0B0F5807F0246A8BF4FF48C
:10A6E0008072022AB8BF02221968002A92FAA2F2E6
:10A6F000B2FA82F208BF4FF0FF32013A21F038017E
:10A7000041EAC20292B21A6020812A7BA17A914268
:10A710000AD01968002A72D06FF3410119601968D4
:10A720006FF300011960A2721A6842F040021A60C9
:10A73000216A8A68002A79D000200646143116441E
:10A740008A680130002AF9D1227B62B15FB1012809
:10A7500072D8072E70D800EB80029200216A0A445A
:10A76000127B002A68D0226A92680026002A4FD005
:10A770000EB1327B22B1AA6812B1116892888A6246
:10A78000226A1768226A5168226A926802F1FF3CC5
:10A7900092B117B33A4612F8010B17469A6892071E
:10A7A000FCD5D8609A68D207FCD5DA6809B101F8FF
:10A7B000012BBCF1010CECD2236A1B7BC3B9236AC9
:10A7C0001B6963B1236A686C1B69984701280AD02A
:10A7D000022804D100232362F8BDFF20DEE7266AA9
:10A7E000236A14332362236A9B688BB16368BFE7D3
:10A7F000AB68002BE3D01A689B889361DFE741F0D8
:10A8000002011960196841F001011960A2728BE719
:10A81000236A1B68002B35D0236A1D68236A596898
:10A82000236A21620022C3E9002245E7217B002937
:10A8300099D0002F92D196E7206AA36982680168B7
:10A84000B9B159600121597392B25A812B685B6981
:10A8500033B14168E369B9B10120596058735A8135
:10A86000AB6813B11A689B8893622846BDE8F8402C
:10A8700038E659730649FF2681F81A6101F58D7192
:10A880005960E1E72362F8BD024858605973E6E772
:10A8900000000020243C002038B5D0F890102B4B4D
:10A8A00004465A68D0F8880071B1131A99420BDC3B
:10A8B00094F88030C4F88820012B10D0D4F884306C
:10A8C0000133C4F8843038BDD4F89430C4F88820FB
:10A8D0000344C4F88C3094F88030012BEED16168C9
:10A8E000201D04F19805EFF3118C102383F31288D7
:10A8F00063681B6A0BB3D4F8A0302A461BB1D36936
:10A900001432002BFBD10B6A6BB1996839B99342B1
:10A9100009D0196829B15B6899680029F7D0143308
:10A92000F3E7C3E900055FFA8CFC8CF31188D4F8D7
:10A9300084300133C4F8843038BD0D625FFA8CFC7A
:10A940008CF31188FFF7B6FEB8E700BF001000E0F7
:10A950002DE9F041826992F88C30012B8AB00546CE
:10A9600049D0023B012B50D892F8FC30D26C2D4CD0
:10A9700063F07F0313708669336DD6F8108003F19E
:10A98000010E0FCCEC46ACE80F00F36CCDE9003EB5
:10A990000FCCACE80F0094E8030006F110078CE838
:10A9A0000300EFF31180102383F3128833691B6ACD
:10A9B000002B2ED0029B6A461BB1D3691432002BA8
:10A9C000FBD1D8F8203073B1996839B993420AD0D5
:10A9D000196829B15B6899680029F7D01433F3E747
:10A9E0001F60C3F804D0C0B280F31188AA6911694E
:10A9F0000B6A002BFCD1136D5A8852BAEA819A88EF
:10AA000052BA2A82DB885BBA6B8201200AB0BDE8A9
:10AA1000F081C8F820D0C0B280F311883846FFF723
:10AA200049FEE3E7A4DA05082DE9F04190F88C30FF
:10AA3000056D012B8AB004466ED015D8C36C4FF05B
:10AA4000FF321A605A609A60DA60D0F890300522BE
:10AA5000B3F57A7FC0F8A02079D8032380F88C3032
:10AA600001200AB0BDE8F081023B012BF8D890F834
:10AA7000FD30C26C4F4E63F07F031370036DD0F84E
:10AA8000108003F1010E00F110070FCEEC46ACE888
:10AA90000F00E36CCDE9003E0FCEACE80F0096E866
:10AAA00003008CE80300EFF31180102383F3128876
:10AAB00023691B6A002B6FD0029B6A461BB1D369C6
:10AAC0001432002BFBD1D8F8203073B1996839B912
:10AAD00093420AD0196829B15B6899680029F7D0B8
:10AAE0001433F3E71F60C3F804D0C0B280F31188B9
:10AAF0002269136A002BFCD16B885BBAA4F8803002
:10AB0000AB885BBAA4F88230EB8801205BBAA4F86A
:10AB100084300AB0BDE8F08190F8FC2090F8FD3058
:10AB20009B1A5B100133DBB205EB430235F813309F
:10AB30005BBAA0F8803053885BBAA0F88230938863
:10AB40005BBAA0F8843001200AB0BDE8F081036947
:10AB50001A7B52B35B6943B390F848302BB390F83B
:10AB6000FC30C26C606563F07F03137090F8FC10DA
:10AB700090F8FD30026D1048C4F8B4005B1A07333A
:10AB80000121C4F8AC30E36C84F8B0100A44C4E985
:10AB9000293284F88C1063E7C8F820D0C0B280F363
:10ABA00011883846FFF786FDA2E7022384F88C302F
:10ABB00056E700BFA4DA0508A985000810B10368AC
:10ABC00082889A61704700BF10B1036882889A62D8
:10ABD000704700BFF8B5644CDFED647AB4F82A33EF
:10ABE000DFED636A04EB400007EE103AB0F8323351
:10ABF000B4F82E036422B8EEC77A02FB03F327EE03
:10AC0000277A07EE903AF8EEE77A02FB003327EE58
:10AC1000277A07EE903AF8EEE77A94F8283387EE31
:10AC2000270A00250E46C4F83C5320EE260A43B3FB
:10AC3000012B00D0F8BDD4F8507307EE907AF8EEEF
:10AC4000677A27EE800A51F037FA78BB94F85433CC
:10AC5000002B77D0D4F8443313B11A689B889361E2
:10AC6000B4F82C03304412F04BFE94F85433002B0C
:10AC700070D0D4F84433002BDCD01A689B889362E0
:10AC8000F8BDD4EDD47AF8EE677A27EE800A51F059
:10AC900013FAD4F84823374B1060D3F8A032B4F835
:10ACA0002C1319443144C4F85813F8BD324A334BBD
:10ACB0005062D7625D62DF62EFF31181502080F352
:10ACC0001288106840F001001060186840F0010020
:10ACD000C9B2186081F31188D16841F00101D160D7
:10ACE000D968244A41F00101D960D2F8A032B4F801
:10ACF0002C1319443144D2F8A0329942FBD8EFF317
:10AD00001181502383F312881B4A1C4B10686FF388
:10AD10000000106018686FF30000C9B2186081F37A
:10AD20001188D168D4F8440321F00101D160DA68B8
:10AD300022F00102DA6000283FF47CAF03688288C9
:10AD40009A61F8BDD4F84433002B89D01A689B88E7
:10AD5000936285E7D4F84433002B3FF46BAF1A6855
:10AD60009B889361F8BD00BF003900200AD7233CBF
:10AD7000CA269B3E08280020001000400014004016
:10AD8000034B93F8402312B1042800D822E7704700
:10AD9000003900200348D0F8283113B100F58E7037
:10ADA00018477047000000200348D0F84C3113B119
:10ADB00000F5A07018477047000000200348D0F845
:10ADC000703113B100F5B2701847704700000020D1
:10ADD0000348D0F8943113B100F5C4701847704798
:10ADE000000000200348D0F8B83113B100F5D67048
:10ADF00018477047000000200348D0F8DC3113B139
:10AE000000F5E87018477047000000200348D0F8AC
:10AE1000003213B100F5FA701847704700000020A7
:10AE20000348D0F8243213B100F506701847704774
:10AE3000000000200348D0F8483213B100F50F702D
:10AE400018477047000000200348D0F86C3213B157
:10AE500000F5187018477047000000200348D0F82C
:10AE6000903213B100F521701847704700000020A0
:10AE70000348D0F8B43213B100F52A701847704770
:10AE8000000000200348D0F8D83213B100F5337029
:10AE900018477047000000200348D0F8FC3213B177
:10AEA00000F53C70184770470000002010B50138CD
:10AEB0000B4C0C4B00EBC00004EB8004D4F81C01DD
:10AEC00098420CBF362038204DF07AFDD4F81C2172
:10AED000D2F8003143F00103C2F8003110BD00BFC9
:10AEE0000000002000640240F8B50138124C00EB6D
:10AEF000C00004EB80041E461048D4F81C31834285
:10AF00000CBF3620382015460F464DF059FDD4F8B9
:10AF10001C01D0F8003143F00103C0F8003194F96E
:10AF20002D01C4F82871C5F30112A909C4F83061D4
:10AF3000BDE8F84047F06ABE00000020006402400F
:10AF4000D3B20D2B2AD84FF0000C10B46346144C2A
:10AF500004E00133202B1DD014F803CF6045F8D155
:10AF600094F801C08C45F4D10E4902EB420401EB88
:10AF7000840201F545700C4903EB43030B4400EBDD
:10AF8000840093F84E3D5DF8044BC2F81C3382F800
:10AF90001433704700205DF8044B70470020704761
:10AFA000CCDA05080000002080CD050810B40C4C58
:10AFB000002304F5577C01E0152B0CD003EB430272
:10AFC00001331CF802108142F6D122445DF8044B93
:10AFD00092F95E0370474FF0FF305DF8044B704705
:10AFE0000039002030B40023114C124D04E001332D
:10AFF0001C2B1AD054F8085FA842F8D125798D424D
:10B00000F5D10D480D4902EB420400EBC30001EB02
:10B01000840390F8B12DC3F81C2301F5457101EBB1
:10B02000840083F8142330BC7047002030BC704784
:10B030002CDB05080000014080CD05080000002041
:10B04000F0B110B504460F4894F804E0002300F571
:10B05000577C01E0152B11D003EB430201331CF8A0
:10B0600002107145F6D10244617992F95E2320689D
:10B07000D3B20D2B02D8BDE81040B3E7002010BDBD
:10B080000020704700390020800AA0F58010532866
:10B0900006D8044B1B5C0C2B02D8034AD0567047D1
:10B0A0000020704780CD0508DC45060858B183882C
:10B0B0004FF00042B3FA83F332FA03F303D00249AC
:10B0C0000A6813430B607047003C01400120FEF703
:10B0D0008FBA00BF0220FEF78BBA00BF0420FEF734
:10B0E00087BA00BF0820FEF783BA00BF1020FEF722
:10B0F0007FBA00BF4FF47870FEF77ABA4FF47C4005
:10B10000FEF776BA30B1036882881B691A4214BF11
:10B1100001200020704700BF30B50C4683B00546C3
:10B1200018B3036803F13F4303F57E039B0A104AFB
:10B13000134493F88C0E4DF043FCA9880091C4F39E
:10B140000013C4F341128DF8043028688DF80520EF
:10B1500004F003036946C4F381048DF806308DF8CA
:10B16000074047F00BFD03B030BD4FF0FF33DEE783
:10B1700080CD050800B1CFE7704700BF0E4B70B51A
:10B18000D3F89867002E14DD0C4C002503E0B5427F
:10B1900004F120040DD0237F0135002BF7D0E068A7
:10B1A0000028F4D0217DFFF7B7FFB54204F1200459
:10B1B000F1D1012070BD00BF08280020C419002073
:10B1C000F8B502680446007C1368022181400B42F6
:10B1D00006D1116808238340194218BF5360F8BD97
:10B1E00004238340656951605360EFF3118350225B
:10B1F00082F312882A6C1168C9070BD5DBB283F37E
:10B20000118895F86C3013B195F88560EEB122681D
:10B21000207CDEE7516889B279B9D5E909708742A7
:10B220002AD0AE690644D66021D82E69301A80B281
:10B230005060A962002185F86C10116841F001018D
:10B24000DBB2116083F31188DBE795F87A000DF02B
:10B25000F9FFAB6EDA68012166F3C302DA6085F8A4
:10B2600085100028D3D02821FFF756FFCFE7381AE2
:10B2700080B25060AF62DDE7012285F86C20BDE747
:10B2800070B50C4682B016460546002847D00368C4
:10B2900003F13F4303F57E039B0A224A134493F8CC
:10B2A0008C0E4DF08DFBAB880093C4F34113C4F3B7
:10B2B00000128DF80530694604F0030328688DF804
:10B2C0000420C4F381048DF806308DF8074047F060
:10B2D00055FCAB882A68B3FA83F3C3F11F0303F06C
:10B2E0000701890013F0F80F06FA01F60BD1136A73
:10B2F0000F2000FA01F123EA01011162136A1E43D3
:10B30000166202B070BD536A0F2000FA01F123EA01
:10B3100001015162536A1E43566202B070BD4FF084
:10B32000FF33BAE780CD050800B1A9E770472DE9E2
:10B33000FF47A04C542303FB00430746D3F8D461D6
:10B34000002E00F02B81D3F8DC81B8F1000F04D07F
:10B3500098F80630002B40F02181542303FB07436B
:10B36000D3F8E0511DB1AB79002B40F017817B1C65
:10B37000DBB2B8F1000F04D0152288F8062088F857
:10B38000073015B11622AA71EB71307E4DF018FB13
:10B39000294640464EF02CFD542047433C4440464D
:10B3A00094F8E63194F8E421002B14BF36211621DD
:10B3B000FFF7BAFF94F8E63194F8E521002B14BFAB
:10B3C000362116212846FFF7AFFF7B4807443C2271
:10B3D0000021384651F06FFCD4F8D4315D68C4F8D0
:10B3E000EC51684647F0C6FADDED037AB4F8E8811F
:10B3F0009FED727ADFED725AF8EE677AF0EE083A56
:10B40000C7EE274A4FF0000E40F2145407EE908A20
:10B410009FED6C7AF8EEE77A64EEA33A87EE274A5E
:10B42000DFED697AB0EE007AE4EE877AE4EE875ACF
:10B4300074EE672A37EEA56AB7EE005AB8F5C87FF2
:10B440000EF1010C07EE90CAD5BF642332234FF4EE
:10B45000967078200344B8EEE77A07EE903A27EE2C
:10B46000247AF8EEE76AD8BF4FF4167986EE873A69
:10B47000CABF4FF4827921464FF4FA7101EB0903F8
:10B4800073EE456AFCEEE67A17EE902A07EE909A84
:10B49000B8EEE73A07EE903A23EE043AF8EEE77A90
:10B4A000C3EE276A36EEE53A72EEE66AC3EE077A35
:10B4B00077EEC57AFCEEE77A17EE901AC6EE877A39
:10B4C00077EEC57AFCEEE77A17EE903A03F10209BF
:10B4D00009EB010A07EE90AAF8EE677AF0EE466AE9
:10B4E000E7EE276AB4EEE64AF1EE10FA5BDC5FFAAB
:10B4F00082F9B9F10F0F58D8323807EE900AF8EEFA
:10B50000E77A77EEE37AC7EE876AFCEEE67A17EE23
:10B51000900A5FFA80F9B9F10F0F46D81FFA81F946
:10B52000B9F1FF0F41D81FFA83F9B9F1FF0F3CD8E9
:10B530001205264B49EA0E7402F07F6200041443A0
:10B5400000F47F00044303EA01210C433846FDF771
:10B55000A1FC2B686FF300032B602C612B6843F474
:10B5600070632B60AB686FF38A23AB60AB686FF3DB
:10B570000903AB60AB6843F40043AB6000221146A3
:10B5800096F91A0047F042FB002296F9190011467D
:10B5900047F03CFB2B6843F001032B6004B0BDE88F
:10B5A000F087E6464AE7013192E7BCF10F0FF8D188
:10B5B0000024CBE700390020EC3A0020286B6E4EC7
:10B5C00000001643002474490000704200FFFF0091
:10B5D0002DE9F843B04D05EB0017D7F89C33002B4D
:10B5E00000F0C5800446060197F8A6034DF0E8F97F
:10B5F00097F8A63303F01F025B090121013B01FA12
:10B6000002F2042B0BD8DFE813F0DC000500E200A7
:10B61000E800EE00A14B596921EA02025A61AB1918
:10B62000013493F8A0030DF00DFEE4B2804610B192
:10B6300012238371C471AB1993F8A1030DF002FEBC
:10B64000814610B11323C4718371AB1993F8A2031F
:10B650000DF0F8FD074610B11423C4718371AC19C5
:10B66000404694F8A3232621FFF75EFE94F8A42316
:10B6700048462621FFF758FE94F8A52338460621B0
:10B68000FFF752FED4F89C33854A934200F0C980FC
:10B69000844A934200F0AD80834A934200F0E680F2
:10B6A000824A934200F0ED80AB19814AD3F89C3373
:10B6B000596841F002015960596841F0010159602F
:10B6C000D9696FF3CB21D96192F8BC1300295FD1FE
:10B6D000186861F3CF301860186861F38E30186015
:10B6E000186861F38A201860196892F8C34364F3FC
:10B6F0004921196092F8BD03196801285BD06FF3E6
:10B7000008211960196860F38201196092F8BE136C
:10B7100007292ED858686FF34920586058686FF38E
:10B7200008205860186861F3C5001860196892F81D
:10B73000BF4364F3C7111960196892F8C04364F3FA
:10B74000CB211960196892F8C14364F34101196073
:10B75000196892F8C22362F3000119601A69072080
:10B7600060F30F021A611A6842F040021A60BDE8E5
:10B77000F8830A296DD058686FF3492058605868DB
:10B7800040F480705860186861F3C5001860CDE718
:10B79000012951D0022937D00329A5D1196841F4D4
:10B7A00000411960196841F48041196019686FF30C
:10B7B0008A21196098E7012CA1D141F480711960A8
:10B7C000A0E7364B196921EA02021A6127E7334BD9
:10B7D000996921EA02029A6121E7304B596A21EA0C
:10B7E00002025A621BE72D4B196A21EA02021A6211
:10B7F00015E7304847F02CF92F4AD2F8203823F4C7
:10B800008043C2F820384FE7196841F400411960BD
:10B8100019686FF38E31196019686FF38A21196006
:10B8200062E7264847F014F9234AD2F8243823F473
:10B830008053C2F8243837E719686FF3CF311960A5
:10B8400019686FF38E311960196841F480611960CD
:10B850004AE7596841F40071596059686FF308214B
:10B86000596019686FF3C50119605FE7144847F024
:10B87000EFF8114AD2F8203823F40043C2F82038F8
:10B8800012E7104847F0E4F80B4AD2F8243823F4C2
:10B890000053C2F8243807E700390020003802407E
:10B8A0000030014000380040003C004000340140BE
:10B8B000000000200E002000003002400C00240098
:10B8C0000F0020000D0024002DE9F04F8DB0A94B92
:10B8D0000793A94BDFF8C0820024A3F69465A74F15
:10B8E000DFF894A2BB0AA3F58013532B4FF0000698
:10B8F0004BD8EB5C0C2B48D818F90390A04B93F86D
:10B90000EE33012B40F00781B9F1010F33D14FF035
:10B91000010B1FFA8BF1484612F0DAFB12F066FCBD
:10B92000037813B1542B40F01F810BF1010BBBF1D5
:10B93000050FEED1ACB34FF0000C8E4A00210BE0A6
:10B94000EB5C0C2B0FD818F903304B450ED00131AE
:10B95000A14202F1AC0221DA906803689B0AA3F5C8
:10B960008013532BECD900234B45F0D143799AF83F
:10B9700005009842EBD10136082E45D05AF81C7FBD
:10B98000BB0AA3F58013532BB3D97D4B93F8EE3349
:10B99000013B012BEFD94FF00009B8E7BCF1000FD4
:10B9A000E9D1DAF80800774B002205E001320E2ACF
:10B9B00003F10C0300F0CA8359688842F6D152B2F1
:10B9C0009AF805103846FFF70DFB6F4A40680023D0
:10B9D0005168884203F1010300F09A800E2B02F1B6
:10B9E0002402F5D14FF0FF33684A03EBC30302EBA7
:10B9F000830393F83431002BBDD15F4BC6EBC606F1
:10BA000003EB8606079B9E60079B0134AC33042C36
:10BA100007937FF464AFDFF8849109F204434FF099
:10BA2000010B98465A4BD3F898270BF1FF339A42F3
:10BA30006BDDD9F80C50002D00F084832968AE88A6
:10BA400001F13F41B6FA86F601F57E01C6F11F0607
:10BA5000890A504B1F68002F40F3A4800433002450
:10BA600005E00134BC4203F1AC0300F099801A6890
:10BA70008A42F6D13F4AC9F80460AC2303FB042490
:10BA8000C9F818405FFA8BF315B1EB710323AB7162
:10BA9000404B616C93F87806E36B72000327974084
:10BAA0003B43E363012303FA02F20A436264002882
:10BAB00039D0A26C03FA06F63243A2646DB1304B62
:10BAC000AA8893F844142B68490141F0050101F05C
:10BAD000E5019A612846FFF71FFB606FB1B20122B2
:10BAE000FCF7A8FA20460BF1010BFCF781FB0123C0
:10BAF000BBF1090F89F81C3089F81D3088F8113026
:10BB000009F1200908F118088CD10DB0BDE8F08FBB
:10BB1000DBB2013B68E7022B7FF4F9AEB9F1080F05
:10BB20003FF4F5AE27E7A26C06F1100103FA01F12C
:10BB30000A43A264002D00F08B8003FA06F6104B36
:10BB4000AA8893F844142B68490141F005011204B6
:10BB500001F0E5019A612846FFF7DEFA606FB1B2A5
:10BB60000022FCF767FABDE74FF0010C002C7FF4D0
:10BB7000E4AE00E71417002014DC050800040140BF
:10BB800000390020140300201C01002000000020C8
:10BB90000828002010170020DC450608C4190020E2
:10BBA000032C58DC8B4AAC2303FB0723D8680028FE
:10BBB00000F0C1825422596083F8AC200131854ADB
:10BBC00083F8AD107B1C1360834B99F8102093F819
:10BBD000053408928168814C00229C4605E00132C0
:10BBE0000E2A04F10C0400F0B18263689942F6D188
:10BBF00041790068CDF81CC052B2FFF7F3F9754BDC
:10BC0000DFF800A2D0E90141AC2202FB0732079B1A
:10BC1000C2E90541514600224868844202F101020E
:10BC20001ED00E2A01F12401F6D16D4B93F810219C
:10BC3000002A00F0288268486A496B4A6B4BC0F8BA
:10BC40002C14C0F82424C0F834340DB0BDE8F08FB3
:10BC500003FA06F682E7604A032382F80434EAE72F
:10BC6000D2B25F49013A02EBC20201EB8202AC247C
:10BC7000584992F83401099007FB04F401EB040CD5
:10BC80000146BCF8AC000029D5D1A2F834016210FD
:10BC900002EBA402C2EBC21202EB8232920102EB6F
:10BCA000A4025349520002EBA40202EB420E0C44E0
:10BCB00050498C200EEB0E1E00FB02F201EB8E0EA3
:10BCC00001F54C7101EB42020A922A68CCF8082077
:10BCD0000A9ACCF898203322DCF80C10CCF87C209F
:10BCE0003F4ACCF89C00062B086812680791CCF8F4
:10BCF00078E000F0F581072BDFF80CC13E4B3F499F
:10BD000008BF19463E4B08BF6346B2FBF1F101F193
:10BD1000FF3C3049B2FBF3F3AC2202FB0712013BBC
:10BD20009BB2A2F86030A2F880C0C3620023836295
:10BD3000426942F001024261026863F30922026033
:10BD4000026863F306120260036843F08003036035
:10BD5000036843F080030360079B59790139490068
:10BD6000C9B207290BD8DFE811F0B8010A00B50104
:10BD70000A00B2010A00AF0108000A234367036802
:10BD80006FF30003036000220123039301930492E5
:10BD90000292009206224DF0D3FC01231A46079B23
:10BDA000597918680139914001F0FE0147F08EF988
:10BDB000079A53791268013B5B00DBB2072B29D845
:10BDC000DFE813F07D0128007801280073012800C6
:10BDD0006E012400101700200039002014030020F9
:10BDE00000000020CD6F0108C96F0108D56F010860
:10BDF00014170020483D00201055220044950800EB
:10BE0000D0DD06001C01002040771B00136F43F0BB
:10BE100008031367079B1879002840F0778113689F
:10BE200043F001031360B04AAC2303FB07235969B5
:10BE30000023DAF80420914203F1010300F01E818F
:10BE40000E2B0AF1240AF4D14FF0FF3AA74A0AEB6D
:10BE5000CA0302EB8303A64AD3F81C01079390425E
:10BE60000CBF362038204CF0ABFD079B9E4AD3F820
:10BE70001C11A048AC2303FB0723D1F8002142F09A
:10BE80000102C1F80021DA684FEACA030793537927
:10BE9000D2F800C0944A013BDBB2032B9BBF96490A
:10BEA00001EB43030021B3F8741FAC2303FB07230A
:10BEB0004FF0000E1982734606E0944500F0408171
:10BEC0000133042B00F0458150F83320002AF4D1CF
:10BED0008A4A9E461346D2F89C270132C3F89C2713
:10BEE00003EBCE024FEACE03C2F8A0C70344099881
:10BEF0009A8811439980902281492346FEF7F4FFE6
:10BF0000079B7A4A7849534402EB8303AC2202FB35
:10BF10000717D3F83C31B9691A6861F306021A6051
:10BF20007B691A6842F002021A604FF4407C4FF4B9
:10BF3000807A1022A4F870C0A4F86CA0A4F868203D
:10BF4000B7F87CE0A4F86AE0B968022201F11800B1
:10BF500084F86E20206609901031B86F84F86F2045
:10BF600007911968606621F4804121F010010904ED
:10BF7000090C1960196841F010011960196841F441
:10BF800040511960196862F38B211960196862F3D6
:10BF9000092119601A6842F080021A601A686FF36A
:10BFA00086121A601A686FF345121A605A686EF3A7
:10BFB0000F025A60099A9A60D8601A68E2615A685A
:10BFC00022629A6862620021DA68A262A4F88CA0F8
:10BFD000A4F890C0A4F88810079AB7F89C00C4F899
:10BFE0008020012284F88E20A4F88A00D7F898C017
:10BFF00084F88F201F68C4F884C027F4804727F096
:10C0000010073F043F0C1F601F681F601F6847F444
:10C0100040571F601F6862F38B271F601F6862F321
:10C0200009271F601A6842F080021A601A6861F3DB
:10C0300086121A601A6861F345121A605A6860F332
:10C040000F025A60079A9A60C3F80CC01A68E2623D
:10C050005A6822639A686263DA68A2631A6842F0D7
:10C0600002021A60089B89F81030C9F80460C9F808
:10C070000C50C9F818405FFA8BF306E5DBB2099360
:10C0800003F1FF3AE2E61849AC2202FB071292F8EC
:10C09000AD1092F8AC2083F8102183F81111CAE595
:10C0A000D36943F40063D361B4E6D36943F0080372
:10C0B000D361AFE6936943F400639361AAE69369A1
:10C0C00043F008039361A5E60A23036457E60A23B5
:10C0D000C36354E60A23836351E60A2343634EE6AF
:10C0E0000849094B11E600BF10170020000000208E
:10C0F00000640240A82F002080CD050808280020F9
:10C10000D58D0008882A1100A0BB0D000B920DF000
:10C1100099F80B9A0A9048B1079B0A21DA79FFF740
:10C12000AFF80A9B5422DA80079B1A68536C43F4D9
:10C130000043536473E6084A022382F804347AE524
:10C14000DB00D3E64FF0FF36314682E400235B6824
:10C15000FFDE00239B88FFDE00390020F8B590F851
:10C160007A301C09013C072C0FD81A4E06EB44020A
:10C170000546B2F87C0F03F00F0340FA03F2D20732
:10C1800003D595F88570012F01D00120F8BD07FA7D
:10C1900003F3013B184034444FF000F894F88C2F1F
:10C1A0000D49104451F8302001EBC00110698B8813
:10C1B0001840EBD0002395F87B2085F885300846A1
:10C1C0000A21FFF75DF8AA6ED36843F00803D36035
:10C1D0003846F8BD80CD050818380020094AD2F845
:10C1E000D83BD2F8DC2B002140F62A00586051627F
:10C1F000116841F0010111601A6842F001021A60F1
:10C20000704700BF00390020002800F0AB812DE905
:10C21000F04F002287B02F21064612F03DF8054668
:10C22000E0B1654FD0F80090C7F8DC9BFEF708FF3F
:10C23000804698B14068C7F8D80B78B15F4C0023AE
:10C2400022465168884202F1240203F101030FD013
:10C250000E2BF6D15A4B93F8100118B1002007B0FD
:10C26000BDE8F08F2F2283F8102183F81101F6E743
:10C27000DBB2DFF84CA1013B03EBC3030AEB830302
:10C2800093F834B1BBF1000FE8D130462F26A3F864
:10C2900034610CF0D7FF0346C7F8E40B20B1DE8011
:10C2A000EA790A21FEF7ECFF464A4749002301E0FC
:10C2B00051F83320914500F05F8101330F2BF7D106
:10C2C00000204CF07DFBD7F8DC0B404A03686FF38D
:10C2D00000030360DAF800309342C0F0458103F1B7
:10C2E000B7723B4902F55852A1FB0221890D013971
:10C2F00089B24A1C0139B3FBF2F3364A364E1B0AA7
:10C30000A2FB03231A09A6FB026252081B09A7F825
:10C31000E22B013B5200C362A7F8E02B8162436924
:10C3200043F00103436103686FF30923036003686B
:10C330006FF306130360AA7912F0020600F017816A
:10C3400002F00106002213464FF0010C6979013911
:10C350004900C9B207290DD8DFE811F041010C00EE
:10C360003C010C0037010C00320108004FF0000EB8
:10C37000C0F874E0CDE90126002203930092CDF8C5
:10C3800010C006224DF0DCF9D7F8DC0B036843F04F
:10C39000800303606B79013BDBB25A00D1B20729FD
:10C3A00020D8DFE811F008011F0003011F00FE0084
:10C3B0001F00F9001B0000BF003900201C010020F5
:10C3C0000000002000000140ACD90508006CDC0230
:10C3D000819F5E16598B4F01ABAAAAAA066F46F041
:10C3E00008060667032B9CBF844BD218C36894BF12
:10C3F000B2F8742F00221343C360AB799B0748BF88
:10C4000001314FF0010248BFC9B246F05FFED7F8D4
:10C41000D80B224600235168884202F1240200F022
:10C42000B78001330E2BF6D14FF0FF3606EBC60670
:10C430000AEB8606724BD6F81C0198420CBF3620D8
:10C4400038204CF0BDFAD6F81C11D1F8003143F079
:10C450000103C1F80031D7F8D86B22460023516898
:10C460008E4202F1240203F1010300F08E800E2BB4
:10C47000F5D16449584600236022FEF735FD336844
:10C480006FF300033360304646F0F0FA6B79D7F86B
:10C49000DC5B012B00F0A880022B00F0A880032BAE
:10C4A00000F0A880042B16BF05EB830305F14001C3
:10C4B00003F13001D7F8D83B1A684BF6EF70024011
:10C4C0001A601A6842F010021A601A68012060F3BC
:10C4D0000D321A601A68022060F38B221A601A6803
:10C4E00060F309221A601A6842F080021A601A6822
:10C4F0006FF386121A601A686FF345121A605A6851
:10C5000040F62A0060F30F025A603F4A9960DA60F1
:10C51000002261688B4204F1240402F1010231D04F
:10C520000E2AF6D14FF0FF3202EBC2020AEB820A6A
:10C53000D8F80800DAF83C21116860F306011160B0
:10C540001A6842F002021A601A68012002431A6057
:10C550006B6C43F400436B642B6803432B6007B0A0
:10C56000BDE8F08F002070474FF0FF31C5E602F0C4
:10C570000102B4460123E9E6204A02EBC30393F823
:10C58000300C9EE6D2B2013ACEE75FFA83FB70E749
:10C590005E1CF6B2013E49E7C66946F40066C66114
:10C5A00020E7C66946F00806C6611BE7866946F4BF
:10C5B0000066866116E7866946F00806866111E71F
:10C5C0004FF0000EC0F840E0D4E64FF0000EC0F887
:10C5D0003CE0CFE64FF0000EC0F838E0CAE64FF07E
:10C5E000000EC0F834E0C5E605F1340162E705F15C
:10C5F00038015FE705F13C015CE700BF80CD05082D
:10C60000006402404182000860CB002030B40B4A35
:10C610000B4B82B0CA25532402EB800000225D62DE
:10C620005C62019201905D625C620198FF22016090
:10C630005A625A6202B030BC704700BF50280040B6
:10C6400000280040F0B5013B0E469DB2644B3468B3
:10C650001B68B3FBF2F2013AE562A262636987B03C
:10C6600043F00103BDF830109DF834206361236866
:10C670006FF30923236023686FF306132360757932
:10C68000B37907460AB183F0010313F0020010D01A
:10C69000002203F001004FF0010C1346013D6D0034
:10C6A000EDB2072D0AD8DFE805F01D094A09800917
:10C6B0005C6E03F0010284460123EFE7CDE901201F
:10C6C000002200922946CDF810C00393062220468E
:10C6D000023D4DF035F8052D14D8DFE805F03D1387
:10C6E00073134F6161630021CDE902030192CDF81C
:10C6F00010C00091062220464DF022F8A36943F0B5
:10C700000803A3613268536C43F400435364136815
:10C7100043F0010313607379012B58D0022B59D0D9
:10C72000032B5AD0042B16BF02EB830302F1400304
:10C7300030330021C7E90032196007B0F0BDA163B2
:10C7400001920022CDE902030092CDF810C006222A
:10C75000022120464CF0F4FFA36943F40063A36177
:10C76000D0E721640192002200920622CDE9020363
:10C77000CDF810C0114620464CF0E2FFE36943F4C7
:10C780000063E361BEE7616701920022CDE9020325
:10C790000092CDF810C00622072120464CF0D0FFB1
:10C7A000236F43F008032367ACE7E16301920022A3
:10C7B000CDE902030092CDF810C0062204212046E4
:10C7C0004CF0BEFFE36943F00803E3619AE702F12E
:10C7D0003403AEE702F13803ABE702F13C03A8E70C
:10C7E000000000202DE9F04FD0F80890046C99F873
:10C7F00005A099F80680D9F80060054687B0204664
:10C800000AF1FF3B46F032F95FFA8BF35F0000223A
:10C81000FFB208F0020885F82C20072F0DD8DFE8BA
:10C8200017F0D2000C00DB000C00E4000C00ED005F
:10C830000800326F6FF3C3023267B8F1000F15D1F1
:10C84000AAF10203022B05D84FEA4A08A8F1020810
:10C850005FFA88F800224146304646F037FCBBF1CB
:10C86000030F11D8DFE80BF096918C0C022B00F22D
:10C8700084804FEA4A0808F1FF385FFA88F8E9E750
:10C88000F3696FF30923F36195F83B30049395F84E
:10C890003A30039395F83930029395F83830019384
:10C8A00095F83730009395F8363095F835203946AD
:10C8B00030464CF045FF99F805309A1E022A50D9AF
:10C8C0000023736341460122304646F0FFFB072FE9
:10C8D00009D8DFE807F073086E0869086404336F4D
:10C8E00043F00803336723684BF6EF7110220B40C7
:10C8F0002A842360236813432360236895F8292042
:10C9000062F30D332360236895F8272062F38B23AD
:10C910002360236895F8262062F3092323602368A7
:10C9200095F8252062F3C7132360236895F8242027
:10C9300062F386132360236895F8282062F3451379
:10C94000236063686A8C62F30F036360D5E9062392
:10C95000A260E360236843F00203236007B0BDE8F0
:10C96000F08F5B00023BDBB2042B53D0062B4ED082
:10C97000022BA7D10023B363A4E74FF0000869E7B7
:10C98000F3696FF30103F3617EE7B3696FF3092382
:10C99000B36179E7B3696FF30103B36174E7F369D6
:10C9A00043F40063F3619EE7F36943F00803F36126
:10C9B00099E7B36943F40063B36194E7B36943F063
:10C9C0000803B3618FE7B2696FF3C302B261B8F1D4
:10C9D000000F3FF435AF49E7B2696FF3CB22B26184
:10C9E000B8F1000F3FF42CAF40E7F2696FF3C302D8
:10C9F000F261B8F1000F3FF423AF37E7F2696FF34C
:10CA0000CB22F261B8F1000F3FF41AAF2EE70023FA
:10CA1000336457E70023F36354E700BF2DE9F04F79
:10CA2000B44B93F8784685B024B90124204605B06C
:10CA3000BDE8F08FB04ED6F8A0520DF0FFFAAF4B24
:10CA400093F81C3C002B00F04D81AD4BAD4FA3FB88
:10CA500005235B09A7FB0327FF0807EB8707A3EB69
:10CA60004707D6F80C38C31A0093A24B03F56D7B29
:10CA7000FBB206F56A78019306F5D16308EB8707E8
:10CA80005D4600269946CDF80CB011E02846FFF728
:10CA9000A9FE9A4B93F81C4C0136A64208F15C089B
:10CAA00007F15C0709F1140905F14C0580F2C1801A
:10CAB000009A002A03DB2B6B934200F3FD808D4B21
:10CAC0004C2202FB063393F8E033002BDED0AB6838
:10CAD000A9891A682B6C5B681FFA83FED368CEF1B4
:10CAE000160E23EA0103BEF1070FD360CED9824AA6
:10CAF000D2F890360133C2F89036AB6C02939C4664
:10CB0000002201215CF8044B92468B461BE0DCF8C6
:10CB10000000BAF1140FA0EB04031DDC13F10804AC
:10CB200048BF03F1170423110AEB241A0446581EC8
:10CB3000013102FA03F38E450BFA00F242EA0302D6
:10CB40000CF1040C08D37145E1D3CAF11503DCF8EC
:10CB500000404FF0150AEAE7BAF1150F5ED16A48B6
:10CB6000C2F38423C2F3441100EB830300EB810181
:10CB7000D3F8943FD1F8941F1B0243EA011302F04B
:10CB80001F0100EB8101C2F3C43200EB8202D1F835
:10CB9000941FD2F8942F0B4343EA023383EA132203
:10CBA00082EA121202F00F020F2A37D1C3F30F13D9
:10CBB0004FF6FF72934231D0B3F5606F00F0818081
:10CBC000A9F80C3098F858200198824210D0B96822
:10CBD000D8F80020521AC8F80020396BD8F8042081
:10CBE000521AC8F804200022BA603A6388F8580044
:10CBF000D8F800200132C8F80020BA680132BA60C3
:10CC00004FF6FF7293427FF441AFD8F804300133FE
:10CC1000C8F804303B6B01333B6337E7364AD2F840
:10CC20008C360133C2F88C36002E3CD04FF6FF73A1
:10CC3000C8E73149DDF80CB00122002381F88C27C8
:10CC4000C1F80C38002C3FF4F0AE04EBC40304EB45
:10CC500043040BEB840403250CE0022E03F1FF33A5
:10CC60001FD9002101220BF14C0B46F02FFA5C4535
:10CC70003FF4DBAEDBF808301868426865F3061253
:10CC800042609BF810105B7911F0020103F1FF364E
:10CC9000A3F102024FEA4303DFD1022AA3F1020308
:10CCA000E0D8D9B2DEE702F23470029958224FF090
:10CCB0009FFF4FF6FF7385E70024204605B0BDE8CF
:10CCC000F08F0C4991F8152602EB420201EBC202EB
:10CCD000324492F825260D2A7FF472AF802289F81B
:10CCE0001E206FE70449012281F88C27C1F80C3817
:10CCF0009CE600BF10170020082800200039002003
:10CD00001F85EB51CDCCCCCC80CD0508F0B50446C9
:10CD100085B0A56EEB686FF34D33EB6068466679BE
:10CD2000A76845F027FE934B9D4206F0020605D00A
:10CD300003F580639D4201D0039B00E0029B03EB5F
:10CD400083035A008C4BB2FBF7F2A3FB0213DB0800
:10CD500003EB8301A2EB4102042A88BF0133AA68D6
:10CD60009BB263F30F02AA60EB686FF31C73EB6076
:10CD7000EB686FF30C33EB602B6966F30D332B61BB
:10CD80006679A26E7107C6F3800300F18880D168CE
:10CD900063F34921D160D16863F38A21D16053697B
:10CDA0006FF30823536153696FF34923536121796A
:10CDB00011F0010740F0C48011F0020540F0BB8083
:10CDC0006E4B03F1200053F8041F8C4254D098425C
:10CDD000F9D116F008035DD0536943F0080353619D
:10CDE000D36843F40053D360002F3DD0E06B00289C
:10CDF00000F0AB806569666EA78945F037FEE36B8E
:10CE00001A684BF6EF710A401A601A681A601A68BD
:10CE1000012161F30D321A601A686FF38B221A60D8
:10CE20001A686FF309221A601A6842F080021A60C9
:10CE30001A686FF386121A601A6842F020021A60AC
:10CE40005A6867F30F025A609E60DD601A680A43F1
:10CE50001A60A16E4A6942F040024A615B6821791A
:10CE60009BB2E36501F0020515BBA26ED36843F4E3
:10CE70000053D36005B0F0BD002CAAD094F88430E4
:10CE8000002BA6D0A16E0B6943F400430B6116F092
:10CE90000803A1D1516963F3C3015161A0E7D368CD
:10CEA0006FF34923D360D36843F48063D36076E79C
:10CEB000206C002855D0266EA569278A45F0D6FD3E
:10CEC000236C1A684BF6EF710A401A601A6842F038
:10CED00010021A601A68012161F30D321A601A6893
:10CEE0006FF38B221A601A686FF309221A601A68AE
:10CEF00042F080021A601A686FF386121A601A688C
:10CF00006FF345121A605A6867F30F025A609E6009
:10CF1000DD601968A26E41F00201002019605860BE
:10CF2000536943F0800302F10C0153610B6843F035
:10CF300040030B609AE7D36843F00803D3603FE7F0
:10CF4000D36843F00403D36036E76FF02003136027
:10CF5000D36843F02003D360D36843F01003D36059
:10CF600082E7A26ED36843F0800302F10C01D36024
:10CF7000DCE700BF00100140CDCCCCCC2045002028
:10CF80002DE9F843434C04EB8004D4F8244C002CE6
:10CF90003DD0656FA1601F463F4B23606B68A36661
:10CFA000AB6B63616B6BA361EB8FE360AB8F236152
:10CFB0003A4B23670646204690460CF0A1FA95F8B6
:10CFC0002C0000285DD194F87A000CF03BF9022285
:10CFD000390794F8789084F885201BD588B317F02A
:10CFE000510F0CBF0122002217F0410F14BF402146
:10CFF000202141EA021101360B22C671827194F898
:10D000007B2041F00601FEF73BF9E36B6BB3204652
:10D01000BDE8F88318F0020F13D090B10B22827193
:10D0200017F0410706F10102C2712DD1A36EDA6833
:10D03000012167F3C302DA6084F885102821FEF726
:10D040006BF818F0010FE0D048460CF0FBF8002810
:10D05000DBD00C220136C671827194F879200A2146
:10D06000FEF70EF9E36B002BD1D195F8301095F94E
:10D070002E00C1F30112890945F0C8FD2046BDE824
:10D08000F8834BF09DFC9EE794F87B200A21FEF785
:10D09000F7F8D6E70039002094DD05085DC10008E7
:10D0A0002DE9F047884600294AD04618DFF89890C5
:10D0B000DFF898A0451E013E8024EFF3118184F330
:10D0C0001288D9F89832D9F89C02D9F89822D9F860
:10D0D0009CC2C9B281F31188624512E0012010F0B0
:10D0E0000FFCEFF3118184F31288D9F89832D9F844
:10D0F0009C02D9F89822D9F89C72C9B281F31188A0
:10D10000BA428CBF002201221B1A03EBC223012B5F
:10D11000E4D0EFF3118284F31288D9F89C3215F829
:10D12000011F5344D2B283F8441CD9F89C32013316
:10D13000C3F30A03C9F89C3282F31188B542BCD10B
:10D140004046BDE8F08700BF0828002000390020D5
:10D15000F8B50D4B93F89C3C032B00D0F8BD0B4E5B
:10D160000D46D6F8A072144609E0FFF799FFD6F8ED
:10D17000A032DB1B322BA4EB00040544EED8002CBC
:10D1800021462846F1DCF8BD1017002008280020B1
:10D19000344BD3F8BC39596A91F85230012B56D12F
:10D1A00070B5314C314AD4F84C0360BBD2F89802C8
:10D1B000D2F89C32984221D0D2F89802D2F89C3210
:10D1C000984249D8D2F89C32D2F898021B1AD2F869
:10D1D000982291F8520088B1B3F5007F28BF4FF430
:10D1E00000731D46002381F85230214921480A442A
:10D1F000ABB2812145F096FFC4F84C531E4B6FF043
:10D2000001021A6170BDD2F8985200F03F03284421
:10D21000C2F89802D2F89802B0F5006F04BF00205F
:10D22000C2F898020020C4F84C03002BBED1D2F8FB
:10D23000982291F852000028E4D00D4881F852302D
:10D240000244BDE870400B48812145F06BBF0A4B9A
:10D250006FF001021A617047D2F89832C3F500638B
:10D26000B5E700BF10170020F8490020082800206B
:10D2700044450020C8200020004C01404AF0CABAB2
:10D28000344B292270B523F88A2C23F8822CFCF722
:10D2900027FA314A314ED2F83438314C43F080030A
:10D2A000C2F83438FBF7D6F84BF066FB46F0C4FD05
:10D2B0004FF0A0402B49826B01F5805342F40012DD
:10D2C0008263C3F87C634FF401660122A3F87A639A
:10D2D0004FF481760025C1F8B40983F8782383F8E8
:10D2E000852304F57B7104F57172A3F8806383F8DC
:10D2F00083534BF039FE23681B4A1C4C1C4EA2FB87
:10D3000003239B09013B0422E262A3626369194A79
:10D3100043F001036361236865F3092323602368F5
:10D32000C6F8502365F306132360236843F0800397
:10D330002360E36843F00103E36069202A46022189
:10D3400045F064FC236843F00103236006F5547044
:10D3500070BD00BF00390020003002404000400195
:10D360000000002010170020D34D6210004C014037
:10D37000F8490020C4DD0508BFF34F8F0549064B6F
:10D38000CA6802F4E0621343CB60BFF34F8F00BF63
:10D39000FDE700BF00ED00E00400FA0508B500213C
:10D3A0000320FFF733F972B6FFF7E6FF08B5184C14
:10D3B000D4F8A42394F8AA034AB1116893880969A0
:10D3C0000B40F8B9003B18BF0123002BF4D1142007
:10D3D00010F096FA00BFD4F8A43363B11A689B88A2
:10D3E000116994F8AA230B4042B9003B18BF0123EE
:10D3F0000BB1FFF7D3FFFBF733F9EBE7B3FA83F396
:10D400005B09F5E7B3FA83F35B09002BD4D1DEE7C0
:10D41000F849002008B572B6FFF7AEFFF0B5A34B90
:10D42000B3F5C07F85B000F0918100F21781B3F5AC
:10D43000807F00F03881B3F5A07F40F00A8103249B
:10D440009B4B1B8A03F00703A34240F0818199485C
:10D4500045F0FEFA9849994B0A68994842F480725F
:10D460000A60FF24CA2153225C6259625A62D0F8D2
:10D470007438DB0000F1FD80924A904B924FCA2530
:10D4800053240020FF215D625C62029002925D6283
:10D490005C62029E0432BA42306059625962F2D133
:10D4A0008A490020FFF7B2F8894B002103910393CA
:10D4B000039B1B680093009B012B00F0EA807D48D2
:10D4C00045F0C6FA7C4A834B1069012161F30200E2
:10D4D00010611A6E61F301021A6645F021FA7E4965
:10D4E000774A0B6843F480330B60D2F800389F030F
:10D4F00007D44FF44053D2F800188E0301D4013BF7
:10D50000F9D1D2F800389D03EFD573496C4A0B6806
:10D5100043F001030B60D2F800389C07FBD56E4B3B
:10D5200067495A6842F480025A605A68482464F392
:10D530008E125A605A68012060F303025A605A68DA
:10D5400060F312425A601A6842F080721A60D1F891
:10D5500000389801FBD5604B9A686FF307129A6008
:10D560009A68042161F34F329A609A6861F38C22C1
:10D570009A60D3F8A42042F03002C3F8A4209A683D
:10D58000022060F301029A609A68C2F38102022AC3
:10D59000FAD1D3F8A4206FF30512C3F8A420D3F86E
:10D5A000A4200B2161F30F32C3F8A420D3F8A020EC
:10D5B0006FF34D32C3F8A0209A6812F00C0FC2F33B
:10D5C000810100F0B580022900F09C80434C444B5F
:10D5D0002360414A434990682368434DC0F30310D8
:10D5E0000144424811F8841CCB402360EB684FF69D
:10D5F000FF010B4043F0052343F47A03EB603C4BFF
:10D60000516FC3F8AC132E493A4BAB60D1F83438A4
:10D6100023F00043C1F83438536F43F080735367ED
:10D6200045F016FA0CF092FC2368334AA2FB032360
:10D630009B09013BB3F1807F09D24FF0E022F0203B
:10D6400053610021072385F823009161136105B020
:10D65000F0BD802B14BF05240624F1E6B3F5E07F6E
:10D6600005D0B3F5007F14BF05240024E8E60124AB
:10D67000E6E6224B002201920193019A03F119730D
:10D68000126803F59E3303F2E1139A427FF4F4AE7D
:10D690000AE70320FEF7BAFF194B1A6882F30888DD
:10D6A0005B689847FEE70424CAE600BFC00000009C
:10D6B00000C0FF1F1C004000007000400028004018
:10D6C00000300240542800406C280040316665421A
:10D6D0005C280040003C024000380240000000206E
:10D6E00000127A0078DE050800ED00E01F0030002F
:10D6F000F849002000000008D34D62105028004077
:10D700000000FF1F5A685A6859685868174C184D2E
:10D71000C2F38813C0F30240164A125C01F00F01F5
:10D7200005FB03F312FB01F2B3FBF2F3236050E7B6
:10D73000D3F8A0200D4C52047FF549AFD3F8A030A8
:10D74000DB047FF544AF0C4B236042E7022477E60D
:10D750000A4B0B490B4A59605A6059645A644CF0A1
:10D7600083F820464CF05EF8FFF754FE00000020DE
:10D7700000127A00D4450608006CDC02003C02402E
:10D7800023016745AB89EFCD01490248FBF74EBF46
:10D79000881E00200000014002494FF08040FBF746
:10D7A00045BF00BFB41E002001490248FBF73EBF41
:10D7B000E01E00200004004001490248FBF736BF8C
:10D7C0000C1F00200008004001490248FBF72EBF53
:10D7D000381F0020000C0040F8B5CB7813B90025A5
:10D7E0002846F8BD00F110070C46064689783846F1
:10D7F0000BF0D6F905460028F1D0E0780BF022FDB9
:10D80000B06123780133DBB210B1C371222383717D
:10D810000521FDF7AFFCB069FDF7D0F90D4AD2F84C
:10D82000A032632BFBD90C480BF08AF9B082384642
:10D8300044F0C6FC074630B9E0780BF003FD0BF06E
:10D8400061FD3D46CCE7306986F888704CF028FBD6
:10D85000C6E700BF0828002040420F00264A92F881
:10D86000C0377BB3D2F8C417884235D0012B29D0FA
:10D87000D2F8CC17814233D0022B23D0D2F8D41760
:10D8800088422FD0032B1DD0D2F8DC1788422BD032
:10D89000042B17D0D2F8E417884227D0052B11D0DB
:10D8A000D2F8EC17884223D0062B0BD0D2F8F4170D
:10D8B00088421FD0072B05D0D2F8FC17814208BF41
:10D8C00007230AD002EBC30103F1010CC1F8C4071E
:10D8D00082F8C0C7184670470023DBB2184670476D
:10D8E0000123FAE70223F8E70323F6E70423F4E72A
:10D8F0000523F2E70623F0E70828002038B5384B67
:10D900004C2202FB003292F8C32302B938BD93F8CF
:10D9100014C693F8152694450ED002EB420403EB8F
:10D92000C40494F818E60EF1FF35012D4FEA4204C5
:10D9300046D9BEF1030F3ED04FF04C0C0CFB003C1F
:10D94000ACF8B413EFF31181902282F31288BCF883
:10D95000B4439CF8B62342EA44020024C9B292B20E
:10D960008CF8B64381F31188110A93F8784681EA5E
:10D970001211514004B1C9434C2404FB003412017C
:10D98000184BD4F8FC03D3F8B03301F00F0192B276
:10D990000A4301219847D4F8F813B4F8C0C3CA88E1
:10D9A000D4F8F43342EA0C02CA8058601A6842F094
:10D9B00001021A6038BD551C05F003056545BBD052
:10D9C000224403EBC202024492F825160029B3D088
:10D9D0004C2202FB0032012482F8B643ACE700BFC0
:10D9E00010170020F849002030B4037F083300EB03
:10D9F00043035B88047F9BB214B98469022C51D025
:10DA0000FF2B3AD80382037F012B16D08369032BA7
:10DA100026D08369022B23D0038A0468244D6068D2
:10DA2000DBB242EA034242EA010300EA0502134381
:10DA300043F00073636030BC70478369022BE5D10B
:10DA4000038A04681A4D6068DBB242EA034242EA84
:10DA5000010300EA05010B4343F080736360EAE7CA
:10DA600004680A43018A636811480340C9B213433A
:10DA700043EA0143636030BC7047FF230382B0F880
:10DA800010C005685FFA8CF06C6842EA00420848F2
:10DA900042EA010304EA00010B4343F080736B6028
:10DAA00030BC7047448A838A23449BB2A8E700BFF6
:10DAB000009800FC2DE9F04FBC4D0746542000FBB8
:10DAC000075083B0D0F8EC41002C00F0A4800C9EED
:10DAD000C0F8F8619BB20126C0F8046280F80862C1
:10DAE000A0F80032002380F80A3280F80A3240F6AB
:10DAF0007103A669360415D4542303FB075393F826
:10DB00000A32DBB2DBB1542303FB0753012283F853
:10DB10000A2293F80A32DBB2002B37D1012003B07E
:10DB2000BDE8F08F013BE4D1542303FB07531220DF
:10DB300083F80A0293F80A32DBB2002BE3D1606863
:10DB40009B4E304040EA41004FEA4108542101FB1E
:10DB5000075140F49030606081F80A3240F671035A
:10DB6000A169880731D5542303FB075393F80A3280
:10DB7000DBB2002B36D0542303FB0753022283F879
:10DB80000A2293F80A32DBB2002BC7D0542303FBDE
:10DB900007530022D3F8EC1183F80A2240F67103F0
:10DBA0008A6992062CD5542000FB075595F80A3255
:10DBB000804A2023CB61B2F8B433013300209BB2FA
:10DBC000A2F8B43303B0BDE8F08F013BC8D15423B1
:10DBD00003FB0753122183F80A1293F80A32DBB2CF
:10DBE000002BC8D1A262542202FB075292F80A12FB
:10DBF000A9B1032382F80A3292F80A32DBB28BE72A
:10DC0000013BCDD1542303FB0755122385F80A327B
:10DC100095F80A32CCE7204603B0BDE8F08F82F8D1
:10DC20000A3240F67103A269510613D5542303FB4F
:10DC3000075393F80A925FFA89F9B9F1000F18D0E7
:10DC4000542303FB0753042283F80A2293F80A3271
:10DC5000DBB261E7013BE6D1542303FB07531222F9
:10DC600083F80A2293F80A925FFA89F9B9F1000F52
:10DC7000E6D15148542607FB06F630442E444FF4B3
:10DC80001052414601904FF02A0AFFF7ADFE96F878
:10DC900008320AFB07FA5344143305EB4303B3F885
:10DCA000D6319BB2002B4ED007EB470B0198CBEB44
:10DCB000CB0B06F20A24D6F8EC1184F8009040F65B
:10DCC00071038A6952075DD52378DBB20BB1052356
:10DCD000237096F808324A6A5B44083305EB8303E5
:10DCE000D3F8D41101F1010CC3F8D4C10A7096F82D
:10DCF00008325344143305EB4303B3F8D621013AF9
:10DD000092B2A3F8D621B6F8FC31013B9BB2A6F83B
:10DD1000FC31B6F8FC319BB253B996F80822524454
:10DD2000143205EB4202B2F8D62192B2002A45D154
:10DD300096F808325344143305EB4303B3F8D63155
:10DD40009BB2002BB7D1542303FB07530022D3F817
:10DD5000EC1183F80A2240F671038A69900618D5FF
:10DD6000542303FB075393F80A32DBB2002B3DD058
:10DD7000542303FB0753072283F80A2293F80A323D
:10DD8000DBB2C9E6013B9CD1122323702378DBB2BE
:10DD90009CE7013BE1D1542303FB0753122283F894
:10DDA0000A2293F80A32DBB2E0E700BF0039002014
:10DDB000009800FCF8490020EC3A0020D6F8EC115D
:10DDC000237040F671038A69120608D52278D2B210
:10DDD0004ABB41460190FFF707FE0198A8E7013BC7
:10DDE000F1D1122323702278D2B2F1E72022CA6146
:10DDF0004A6863F309024A604A6863F30C324A6076
:10DE00004A6863F317424A604A6863F318624A60DB
:10DE10004A6863F38A22542303FB07534A6093F84A
:10DE20000A32DBB278E6542303FB0753062283F859
:10DE30000A2293F80A32DBB26EE600BF032108B56E
:10DE400005460846FEF7E2FB72B6104BD3E9EE2317
:10DE500052EA03010AD1002421460420FEF7D6FB32
:10DE600021460520FEF7D2FBFFF786FA0848D0F8D6
:10DE7000A04229B24EF6602000FB01F1A41843F144
:10DE800000030C1943EBE171E7E700BFF8490020FC
:10DE9000082800200548D0F8083323B1DB6A13B105
:10DEA00000F5427018470248704700BF082800205C
:10DEB00004DE050838B5184CD4F8C0331B8843B9C4
:10DEC000164D002384F8CC3385F80033C5F8FC32B6
:10DED00038BDD4F8C423002AF2DD012A09D0D4F8D1
:10DEE000C83359880D4DA4F8CE13012384F8D033DC
:10DEF000E7E7D4F8C8138A8849880132521A9A424F
:10DF0000F0D1064DD5F8083300221B69C5F834233B
:10DF100005F542709847D4E7F8490020082800200A
:10DF20000748D0F804331BB1064B93F8D0330BB13C
:10DF300000207047D0F8083300F542705B6818473E
:10DF400008280020F849002030B4154A154D92F8F1
:10DF5000003305F575742344036095F8CC334460B1
:10DF600092F80003834292F8000312D8834204D34C
:10DF7000002030BCC1E90000704792F80023002B5C
:10DF8000C2F180020CBF0120022030BCC1E9002395
:10DF900070471B1A0022012030BCC1E900327047D3
:10DFA00008280020F84900200E4B0F4A93F8001370
:10DFB00092F8CC0393F80023904293F800230CD8F6
:10DFC000904238BF93F80023D3F8FC323ABFC2F135
:10DFD00080028018002018447047D3F8FC32801A61
:10DFE0001844704708280020F849002030B51C4C20
:10DFF0001C4D94F8003394F8001385B005F5757244
:10E000001344029395F8CC3303928B421DD894F8B5
:10E010000023934211D294F800130193C1F18001BF
:10E020000091D3B9012208B93F2906D900236946D6
:10E0300002A84CF0C1F895F8CC3394F80003C01A4C
:10E04000B0FA80F0400905B030BD94F8001300220A
:10E05000591A019200910122E5E719440222E2E7F0
:10E0600008280020F84900202DE9F043164685B025
:10E07000002936D0441E254D254F04EB01084FF0F2
:10E08000000901E0A0452CD095F8CC0314F8013F1D
:10E09000411C2844C9B280F8D4330B0648BF002085
:10E0A00097F8003385F8CC134ABF0146084685F837
:10E0B000CC938B4297F800338ABFC3F18003C01A18
:10E0C000C0183F28DED997F800338B42DAD0114BC5
:10E0D00093F89430002BD5D00020FFF787FFA045A0
:10E0E000D2D1694602A8FFF72FFF20B1DDE9003247
:10E0F00013443F2B02D805B0BDE8F08302463346F7
:10E1000002A84CF059F805B0BDE8F083F8490020AA
:10E11000082800200000002030B585B0694602A81C
:10E12000FFF712FF58B9094C04F54275D4F80833CB
:10E1300028465B6898470028F8D005B030BD0246F5
:10E14000012302A84CF038F8EDE700BF08280020B2
:10E1500070B5124E1546D6F804330A464119994255
:10E160000F4988BF1D1A91F8CC1396F800339942D5
:10E1700082B0044603D00192FFF7CEFF019AD6F891
:10E18000081308480023C6F834332B468D6A21460D
:10E19000AC4602B0BDE87040604700BF08280020D0
:10E1A000F8490020102B00208C4613460146624699
:10E1B0001846CDE738B52448244C0023C4F804336E
:10E1C00002461178022902F106022CD00133062BF7
:10E1D000F7D11F4DD4F808330022C5F8C823F3B196
:10E1E000DA6AE2B11B489047D5F8C833C5F8C003D6
:10E1F000A3B19A885B88D21A436802FB0333C4F840
:10E200000433FAF799FB95F8CC2394F800339A423B
:10E21000054601D0FFF780FFC4F8FC5238BD0E4B15
:10E22000C5F8C03338BD0A4DD4F8082303EB4303C7
:10E2300000EB4303C5F8C83312B1D26A002AD1D12A
:10E240000548C5F8C003D4E74C4E0020082800203C
:10E25000F8490020102B002004DE050810B50A4CF8
:10E26000D4F808335B6A13B104F542709847074A43
:10E27000D4F8FC32D2F8C0235288013B13445242F6
:10E280001340C4F8FC3210BD08280020F8490020D3
:10E29000084B09498B4202460AD2184602E01C305C
:10E2A000884205D20388C3F30B039A42F7D1704723
:10E2B000002070474CD00608A0D7060870B58588A6
:10E2C0000B460446C5F30B052A46002118464EF0BE
:10E2D000F2FC6169084A9142034602D3074A91421F
:10E2E00005D319B1BDE870401846084770BD2A46ED
:10E2F000BDE870404EF07CBCA0D70608A8D906083F
:10E3000038B5064C064DAC4206D2A16820461C34F6
:10E31000FFF7D4FFAC42F8D338BD00BF4CD006089D
:10E32000A0D706088388C3F30B039342A8BF134604
:10E3300070B51A461D460C46064680684EF058FCDD
:10E3400062199442B569074B08D0074814F8011BBD
:10E3500000FB03F3A24283EA0103F7D12B60012003
:10E3600070BD00BFC59D1C81930100010A4491420C
:10E3700019D000B501F1FF3C02F1FF3E41F221014D
:10E380001CF8012F082380EA022010F4004F81EAD4
:10E3900040020ABF400090B280B2013BF5D1E64591
:10E3A000EED15DF804FB70474840082310F0800F61
:10E3B00082EA40010ABF4000C8B2C0B2013BF5D1B9
:10E3C000704700BF30B505688D4219D901F1FF3E95
:10E3D0006C1E00231EF801CF082183EA0C0313F002
:10E3E000800F82EA430C0ABF5B005FFA8CF3DBB25A
:10E3F0000139F4D17445EDD16A1C02602B7030BD37
:10E4000000236A1C02602B7030BD00BF07EE901A1B
:10E41000B8EE677ADFED7C7A27EE000A60EE277AA5
:10E42000BDEEE77A17EE103A2033402B00F2DB8086
:10E430009FED767AB4EEC70AF1EE10FAB0EE677A85
:10E440000CDDDFED735A9FED736AF0EE476AF4EE70
:10E45000C66AF1EE10FA37EE657AF6DCDFED6E6A29
:10E46000B4EEE67AF1EE10FA0CD5DFED695A9FEDC5
:10E470006B6AF0EE476AF4EEC66AF1EE10FA37EE18
:10E48000257AF6D4DFED666AB4EEE67AF1EE10FA9C
:10E4900000F39D80DFED636AB4EEE67AF1EE10FAE8
:10E4A00044BFDFED5D6A36EEC77A27EE075ADFED2F
:10E4B0005E5A9FED5E6ADFED5E6ADFED5E4AA5EEB5
:10E4C000256A27EE054AE5EE066AF7EE005AA4EE45
:10E4D000267AF0EE656AE7EE646AE7EE245A86EE85
:10E4E000A54A9FED4F7A77EE877ABDEEE77A17EE71
:10E4F000103A2033402B6FD89FED4F7AB4EEC70A05
:10E50000F1EE10FA0CDD9FED426ADFED426AB0EEEB
:10E51000677AB4EEE67AF1EE10FA77EEC67AF6DCB8
:10E520009FED3D7AF4EEC77AF1EE10FA0CD59FED2F
:10E53000386ADFED3A6AB0EE677AB4EEE67AF1EE69
:10E5400010FA77EE867AF6D49FED357AF4EEC77A34
:10E55000F1EE10FA4CDD9FED397A77EE677A67EECF
:10E56000A74A9FED317A9FED315ADFED316AA4EE73
:10E57000875A67EEA43AE4EE856AB7EE006AE3EEE6
:10E58000A67AB6EE007A36EE676AB8EE005A67EE03
:10E59000857A26EE077AB7EE005AC5EE256A002383
:10E5A000836143610362C36180ED044A26EE877A8A
:10E5B00026EE866A66EEA77A80ED095A80ED007A2B
:10E5C00080ED016A80ED027AC0ED037A7047DFEDDD
:10E5D0001B6A36EEC77A68E7DFED197AB6EE007A85
:10E5E000B7EE006AD7E7B7EE004AF0EE445A78E794
:10E5F0009FED0C7AF4EEC77AF1EE10FA44BF9FED6E
:10E60000067A77EE677AAAE727D4D2360024F44850
:10E61000DB0FC940E4CB1641DB0F49C0E4CB16C188
:10E62000DB0FC93FDB0FC9BF92E741B99730083C08
:10E6300015A82ABEF304353F00247448DB0F494077
:10E64000000000009FED2E7A70EE077AFDEEE76A7B
:10E6500016EE903A2033402B4FD8B4EEC70AF1EEB5
:10E6600010FA0CDD9FED276ADFED276AB0EE677ABE
:10E67000B4EEE67AF1EE10FA77EEC67AF6DC9FEDAC
:10E68000237AF4EEC77AF1EE10FA0CD59FED1D6AED
:10E69000DFED1F6AB0EE677AB4EEE67AF1EE10FABB
:10E6A00077EE867AF6D49FED167AF4EEC77AF1EE1D
:10E6B00010FA1DDC9FED177AF4EEC77AF1EE10FA2E
:10E6C00044BF9FED127A77EE677A27EEA76ADFEDF7
:10E6D000125ADFED126A9FED127AE6EE256A67EEB6
:10E6E000865AA6EE267AE5EE877AB0EE670A70477C
:10E6F0009FED0C7A77EE677AE7E79FED0B0A70479C
:10E70000DB0FC93FDB0FC940E4CB1641DB0F49C02B
:10E71000E4CB16C1DB0FC9BF92E741B99730083C83
:10E7200015A82ABEDB0F494000000000F0EEC07AB9
:10E73000B0EEE07AB4EEE77AF1EE10FAB4BFB0EEE4
:10E74000676AB0EE476AB5EE406AF1EE10FA46D05D
:10E75000B4EEE77AF1EE10FA8CBFF0EE675AF0EE05
:10E76000475AC5EE866ADFED1F2ADFED1F3ADFED5F
:10E770001F4A9FED1F5A9FED1F3A9FED1F4ADFED85
:10E780001F5AE6EEE23AA6EE834AE6EEA34AB7EE59
:10E79000006AA6EEA45AA6EE846AE6EE855AC5EE95
:10E7A000866AB4EEE77AF1EE10FA48BFDFED147A2C
:10E7B000F5EEC00A48BF77EEE66AF1EE10FA48BF00
:10E7C000DFED107AB5EEC00A48BF77EEE66AF1EEEB
:10E7D00010FA48BFF1EE666AB0EE660A7047DFEDE8
:10E7E000076ADEE739094E3DE3B59E3E88FA163EDC
:10E7F00045FE7F3F99FB243F69A2163EA7DFA83460
:10E80000DB0FC93FDB0F494090ED005A9FED4C0AEA
:10E8100035EE000A08B5FDEEC07A17EE903A2033C7
:10E82000402B7BD8FAF7DAF9F0EE403AFDEEC57AE4
:10E8300017EE903A2033402B7FD8B0EE450AFAF716
:10E84000CDF9B0EE405AD0ED014A9FED3D0A34EECD
:10E85000800AFDEEC07A17EE903A2033402B69D83B
:10E86000FAF7BCF9F0EE405AFDEEE47A17EE903A72
:10E870002033402B5BD8B0EE640AFAF7AFF9F0EE24
:10E88000404A90ED023A9FED2E0A33EE000AFDEE6B
:10E89000C07A17EE903A2033402B45D8FAF79EF90C
:10E8A000B0EE404AFDEEC37A17EE903A2033402B8B
:10E8B00037D8B0EE430AFAF791F9F0EE407A24EE39
:10E8C000233A27EEA36A24EE057A67EE856AB0EE56
:10E8D000462AF0EE432AA7EE242AE6EEE42AA6EE24
:10E8E000247AE3EE646A24EE254A65EEE77A25EEA3
:10E8F000655A65EEA35A81ED004AC1ED017AC1ED7A
:10E90000024A81ED032AC1ED042A81ED055AC1EDC9
:10E91000066A81ED077AC1ED085A08BDDFED093AB4
:10E9200084E7DFED087ACAE79FED064ABAE7DFED34
:10E93000054AA6E7DFED035A96E79FED025A82E704
:10E94000DB0FC93F000000002DE9F04389B0541CE3
:10E9500003941478002C00F00781002507468846B0
:10E960001E46A94609E021463846C047039A0135AC
:10E97000531C03931478002C3DD0252CF3D1931C09
:10E98000CDE903395078302800F09480A0F13003AD
:10E99000DBB2092B4FF0000440F297806C2838D08E
:10E9A000782822D857282AD9A0F15803202B1CD820
:10E9B000DFE803F0B41B1B1B1B1B1B1B1B1B1B9546
:10E9C0009D1B1B1B1B1B1B1B1B1BAF1B1B1B1B118B
:10E9D0001BA71B1BB40056F8043B049A00930023AA
:10E9E00041463846FAF7A8F90544039A531C0393A5
:10E9F0001478002CC1D1284609B0BDE8F083002866
:10EA0000F9D02528F1D125213846C0470135039A90
:10EA1000AEE7039B5A1C039219787829A8D8572986
:10EA200058D9A1F15803202BA2D801A050F823F007
:10EA300035EB000871E9000871E9000871E9000888
:10EA400071E9000871E9000871E9000871E900083E
:10EA500071E9000871E9000871E90008DFEA0008BF
:10EA60004DEB000871E9000871E9000871E9000840
:10EA700071E9000871E9000871E9000871E900080E
:10EA800071E9000871E9000815EB000871E9000858
:10EA900071E9000871E9000871E90008D7E9000888
:10EAA00071E9000859EB000871E9000871E90008F4
:10EAB00035EB0008D31C03939078A0F13003DBB250
:10EAC000092B4FF001043FF669AF04AA03A947F0F0
:10EAD00073FF63E700298ED0252994D048E756F8C4
:10EAE000041B3846C9B2C0470135039A40E756F8BF
:10EAF000040B05A901F0E6FA05AB0093049A23463E
:10EB00006EE756F8040B05AB00220A2101F092FAD9
:10EB1000F2E7039A56F8043B1D6029E7A0F158027A
:10EB2000B2FA82F256F8040B520905AB102101F03B
:10EB300081FAE1E7A1F15802B2FA82F256F8040B29
:10EB4000520905AB102101F075FAD5E756F8040B10
:10EB500005A901F0B7FACFE756F8040B05AB002280
:10EB60000A2101F067FAC7E7254644E70EB400B56D
:10EB700084B005AB019053F8042B0649039301A818
:10EB8000FFF7E2FE019B00221A7004B05DF804EB6F
:10EB900003B07047B98D00082DE9F04F41F694623B
:10EBA0008DB00021BF484EF086F8BF4A002309937C
:10EBB00009920999043209680A930A920A9A10681C
:10EBC00051EA000240F05C81B84B03934C220021D3
:10EBD000B4484EF070F84C220021B2484EF06BF869
:10EBE000039BB049D3F84434B14A0A600124C1E917
:10EBF00007334B620C714AF061FCFFF7DBFA00212E
:10EC000008460AF0ADFBF9F797FEB0F1000B40F3B0
:10EC10000881A84BA84D0193A24BA84E0024029452
:10EC200003F14C092746A24605F58F6804E00AF572
:10EC3000006AD34540F3AE80019AD2F8A032C2F800
:10EC4000A432F9F70DFD202241465046FFF780FA25
:10EC50009B49122240464EF06BF80028E7D1BA4596
:10EC600022D00299974BCDF8149001EB410203EBAF
:10EC700082004A1C944902920490FFF777FFDDE975
:10EC80000403D9F81C2043F84C0BC9E908228F4A29
:10EC9000C9F80C70C9F82820AAEB07070122C9E9B6
:10ECA0000477C9F808209946039BD3F84434C9F87F
:10ECB0001C3057461222A918335D91F878149942F6
:10ECC00002F101020BD00024202AF4D12037BB45E9
:10ECD0004146384654DBFFF73BFA0022EBE70134AC
:10ECE000152CF1D1D0197A492022FFF731FA0023EF
:10ECF0000A220BA97648CDF82C8000F0D9FF0490A9
:10ED00000B98002301300A220BA90B9000F0D0FFD2
:10ED100007900B98002301300A220BA90B9000F0FA
:10ED2000C7FF06900B98002301300A220BA90B9015
:10ED300000F0BEFF05900B980BA9013000230A22BA
:10ED40000B9000F0B5FF07460B98002301301946E1
:10ED50000A220B9000F0ACFF049989B1DDE906327C
:10ED600043EA4212059B7F0147EAC323A1F2BC712B
:10ED700043EA600342EA412243EA0243C9F81C30F5
:10ED8000029B642B00F0EE8057460AF5006AD345DB
:10ED90003FF752AF029A642A00F0E480BA4500F0CF
:10EDA000E580484C4849494E0C2303FB0244531C60
:10EDB0001A462046AAEB07050293FFF7D7FED9F8BB
:10EDC0001C30C9F80040C9E90375C9E908330123BB
:10EDD000C9F81450C9F82860C9F80830029B5D1CB6
:10EDE0004C22304F02FB05F57B19002118464DF0EF
:10EDF00062FF4C2200214DF05EFF039A3549D2F8A4
:10EE000044247951029C4262C0E904BBC0E9072254
:10EE100001220234866282604FEA4B03B3F1805FC5
:10EE20001EDA4C221F4D02FB04F42B191846002158
:10EE30004DF041FF4C2200214DF03DFF0399CBF1F5
:10EE40000062D1F844140346520023482851C3E914
:10EE50000422C3E9071102225A71012259629A6001
:10EE6000104A95682DB913791BB11368002B40F037
:10EE70008B80002108460DB0BDE8F04F0AF070BA53
:10EE80004FF47A72181800234CF020F9134B40F21B
:10EE90006D11A3FB00231B0C022440F2B2720D463D
:10EEA00027E000BFCCAC002060280040000000201C
:10EEB00050CD060808280020F849002070450608B3
:10EEC0004C450608904E002060450608A9E1000860
:10EED000704E0020884506089845060807452EC252
:10EEE000013212F00304A3EB01030CBF4FF4B7711E
:10EEF00029469942F4DD7949002C3FD003910399CA
:10EF0000D1F814148B4272DB754D01245B1A55F84D
:10EF1000041F994204F10104F8DD013343EA44136C
:10EF2000A2F2BC7243EA42236E4A039DB0FBF2F1A7
:10EF300002FB11024FF461603C24B2FBF0F100FBD4
:10EF400011221C20C5F81804B2FBF4F004FB1022B7
:10EF5000521042EA401242EAC12242EA0343C5F893
:10EF6000443433E66423604E029337E7029B012466
:10EF70005D1C002B3FF450AF5B4E31E70C46039114
:10EF80001D21C4F81814BAE7C2E911551564D563F8
:10EF900029462E46D46C02F14C0354B39C681E647F
:10EFA000481E8442C3E91166DE6312D0481C8442C5
:10EFB00016D08C427FF45DAF084600283FF459AF6D
:10EFC000116CCC6B0134CC631964936401461A460E
:10EFD000E0E700293FF44DAF884253F80C2CECD108
:10EFE000117900293FF445AF53641A64EEE7012418
:10EFF00093E73E490222264613E0CB6B0A635B018E
:10F000001DBF03F6FF7702F1FF3303EB17331346FF
:10F01000C1E90466C1E90D3351F84C0F5A1C0135A2
:10F02000C8B10B79002BE8D10F690A63002F47D1D3
:10F030004F691046531E4863002F4AD007F6FF77EA
:10F0400003EB1733201A8B63C41851F84C0F5A1C6A
:10F0500001350028E5D126492648C1F8F4523E2260
:10F060000D46013BC1F8D022019140223F21C5E964
:10F07000B512C5E9B934990F9A00C5F8CC0253B35B
:10F0800040F2FF10121841F10001520A42EAC15247
:10F0900002F1400101980A4402EBC303C0F8E022E8
:10F0A000DA0DC0F8C422114AC0F8EC22C0F8F022F0
:10F0B0005A02C0F8DC12C0F8C832C0F8C022D8E644
:10F0C00007F6FF77531E03EB17304F694863002F95
:10F0D000B4D11346B6E70122DAE700BF00000020F2
:10F0E0001404002080510100A9E10008CCAC0020EC
:10F0F00008280020A44506082DE9F043DFF8E89031
:10F10000374F93B0FEF7D6FEFFF754F899F8003367
:10F1100097F8CC239A4201D0FEF7FEFFD9F804837A
:10F120000025C9F8FC52B8F1000F11D02D4E6C46E5
:10F130002A4631462046FFF719FD20464BF002FBD8
:10F140002035014601222046FEF78EFFA845EFD864
:10F1500099F8003397F8CC239A4201D0FEF7DCFFF0
:10F16000D7F8C0339B7B012B33D099F8003397F845
:10F17000CC239A4201D0FEF7CFFF0027C9F8FC72DA
:10F18000B8F1000F28D0DFF85C903D466C462A4667
:10F19000494609A8FFF7EAFC2122002120464DF04C
:10F1A0008AFD202221462846FEF7D2FF202206466D
:10F1B00009A9204615444DF0BBFD08B9202E00D00A
:10F1C0000137A845E3D8B7FA87F0400913B0BDE886
:10F1D000F083FFF743F8C8E7012013B0BDE8F083E0
:10F1E000F8490020AC450608082800202DE9F04326
:10F1F000002483B00646048021463046013437F0AF
:10F20000DBFE082CF8D10023DFF8688086F8EA30AE
:10F21000C6F8EC30C6F8F030C6F8F430C6F8F8306E
:10F220001F46FC3699463A46414601A8FFF79EFC28
:10F230003546032401AA12F8013B6BB1013C05F8E5
:10F24000013BF8D10137082F85F8009006F104063C
:10F25000E9D103B0BDE8F0832846224620212544A9
:10F2600001374DF028FD082F85F8009006F10406BF
:10F27000D9D1EEE7CC4506080378202B024600F1F1
:10F280000100F9D0092BF7D02D2B28D02B2B03BF51
:10F290005378B7EE000A0246B7EE000AA3F1300138
:10F2A000C8B209289FED567A10D8F2EE046A07EE2C
:10F2B000901AF8EEE77A12F8013FE7EE267AA3F10A
:10F2C0003001C8B20928B0EE677AF0D92E2B5ED093
:10F2D00003F0DF03452B07D020EE070A7047537871
:10F2E000BFEE000A0246D9E710B451782D2978D034
:10F2F0002B296AD0A1F13003092B02F101026BD84E
:10F300000024002303EB830301EB430312F8011FE6
:10F31000A1F130000928A3F13003F3D9B3F59A7FA6
:10F320001A4628BF4FF49A72072B66D9DFED356A6B
:10F330001346F7EE007A083B072B67EEA67AFAD859
:10F3400002F00702DAB1F2EE046A012A67EEA67A49
:10F3500015D0022A67EEA67A11D0032A67EEA67AA4
:10F360000DD0042A67EEA67A09D0053A67EEA67A90
:10F3700005D067EEA67A012A18BF67EEA67A6CB3AD
:10F3800087EE277A5DF8044B20EE070A7047537822
:10F39000A3F13001C8B2092802F1010298D8F2EEB7
:10F3A000046AF0EE665A07EE901AF8EEE77A12F861
:10F3B000013F87EEA66AA3F13001C8B2092866EEC4
:10F3C000A56A37EE067AEED982E79178A1F130038B
:10F3D000092B02F1020293D9F7EE007A27EE277A81
:10F3E000D0E79178A1F13003092B02F1020288BF26
:10F3F000F7EE007AC4D8012483E7F7EE007AA1E79C
:10F400000000000020BCBE4CF0B5067906F0E00319
:10F41000402B03D145794FF0FF3406E0602B4FF0CD
:10F420000105F8D1447905FA04F40023012006F01F
:10F430000706AB4200D1F0BD052E0FD8DFE806F07D
:10F440000308101D242448B1C85CD75C78400FE045
:10F4500020B1C856D756C71B784278410133E8E738
:10F460000028FBD031F8130032F81370784080B2D6
:10F4700020420CBF01200020F0E70028EED031F937
:10F48000130032F91370E6E70028E7D051F82300A3
:10F4900052F82370DAE7F8B50C4E337805468BB98D
:10F4A000F8BD25B12388C3F30B039D4204D0D4E9F2
:10F4B0000201A2884DF09CFB1C34BC42F1D3002316
:10F4C0003370EDE7024C034FF7E700BF08EC002074
:10F4D0004CD00608A0D70608037903F01803102BB8
:10F4E0001CD004D82BB1082B06D000207047182B55
:10F4F000FBD1B0F80B007047104BB0F80B0093F93C
:10F500000030591C06BF0E4B1B78DBB203EB8302A5
:10F5100003EBC20300EB830080B27047074BB0F8E7
:10F520000B0093F901305A1C06BF054B5B78DBB228
:10F53000C3EB031300EB4300EEE700BF64040020BD
:10F540008057002020B10078B0FA80F04009704761
:10F550000120704738B5074C074DAC4203D3074B29
:10F5600001221A7038BDD4E90210A2884DF040FB88
:10F570001C34F2E74CD00608A0D7060808EC00209F
:10F58000092900D001B9704701394B0003F0080286
:10F59000930001F00301A3EB9203C1EB0111C3EB54
:10F5A0000313C1EB011100229B00890002608180DE
:10F5B00043807047B5EEC00ADFED337AF1EE10FA02
:10F5C000CCBF30EE270A30EE670ADFED307A20EE4E
:10F5D000270A70B5FDEEC07A86B017EE904A054650
:10F5E00084EAE470002303A9A0EBE470CDE90033C2
:10F5F000029344F081FF002CACBF20232D2303A8ED
:10F600008DF800304BF09EF801286E4626D0022877
:10F6100030D0032803BF302303A9304603A914BF09
:10F6200030468DF801304DF04EFB30464BF08AF8F5
:10F630000338C4B22246314628464DF0D9FA002399
:10F640002B5528464BF07EF82E232B5401303119D0
:10F6500028444DF054FB284606B070BD43F23002FA
:10F66000302303A93046ADF801208DF803304DF06A
:10F670002AFBDAE743F2300303A93046ADF8013044
:10F680004DF021FBD1E700BF6F12033A00007A442E
:10F6900008F0B8BD13B568B14C1E14F8011F21B9AC
:10F6A00002B0BDE8104008F0C1BD019008F0AAFD0D
:10F6B0000198F2E702B010BD73B5104C01920646F6
:10F6C00060680D46A0B10E49FFF7E4FF606831465F
:10F6D000FFF7E0FF0B496068FFF7DCFF0A49019B79
:10F6E00060682A46FFF730F908496068FFF7D2FFE3
:10F6F000237A0BB10123637202B070BD08EC0020C5
:10F70000EF450608104C060891F60008FC4506086F
:10F7100070B50546B0F80900FEF7BAFD054B1E7836
:10F7200004462846FFF7D8FE16B1E368184470BDBA
:10F73000A368FBE708EC002038B505460C46FFF748
:10F74000E7FF2B7903F0E002602A03F007032AD1D8
:10F75000052B0CD8DFE803F0030B0F0B1B1B6A799A
:10F7600001239340DBB2027814B11343037038BD18
:10F7700022EA0303FAE76A79012393409BB20288E5
:10F7800014B113430380F2E722EA0303FAE76A792C
:10F79000012303FA02F2036814B113430360E6E79E
:10F7A00023EA0203FAE7052BE1D8DFE803F00303BD
:10F7B000050507070470DAE70480D8E70460D6E798
:10F7C00008B520214DF08EFA034620B11A78202A80
:10F7D00000F10100F8D0184608BD08B5CB0701D4E8
:10F7E000FDF718FE08BDF7B5114E07463046002359
:10F7F00000F80A3F0C460F4B0F49002F08BF19466F
:10F8000015464DF060FA0D4F04EB45050A36AC4243
:10F8100002D10B4803B0F0BD394634F8022B6846DC
:10F82000FFF7A4F9694630464DF04DFAEFE700BF07
:10F8300008EC00200946060800460608124606089D
:10F8400012EC0020F7B50C4E0C4F002306F83B3F9E
:10F85000044600EB4105AC4202D1094803B0F0BDBB
:10F86000394634F8022B6846FFF780F9694630467E
:10F870004DF029FAEFE700BF08EC0020F548060834
:10F8800043EC0020F8B5084F4E1E054601F11F0459
:10F8900016F8012F28463946FFF768F9A64205F108
:10F8A0000205F5D1F8BD00BF174606080246531CF5
:10F8B000084605D1044B1A681B790A600B71704722
:10F8C0000249FFF753B900BF58460608F648060834
:10F8D0002DE9F341124D134F002305F8643F044610
:10F8E00000EB8106B44203D10F4802B0BDE8F081BD
:10F8F000394628464DF0E7F9214668464DF0FFF9B4
:10F900004FF00008202168464DF0ECF928B969460F
:10F9100028464DF0D8F90434E4E780F80080F1E798
:10F9200008EC0020054706086CEC0020024BD3F8D9
:10F9300088003AF065B900BF08EC00202DE9FF47C8
:10F940001E46C368BDF83070DDF834800446894631
:10F95000924643B3CBB20C2B9ABF1A4AD556002518
:10F96000BAF1FF3F21D02368174A3146CDE9005A4A
:10F970003846C047524620795FFA89F1FBF7E0FA32
:10F98000024600B10288D3B20393C2F30323120BE1
:10F99000CDE9005202930D4A236831463846C047EC
:10F9A00004B0BDE8F0874D1CDAE77B06F8D4236885
:10F9B000074A0C9531463846C44604B0BDE8F047C6
:10F9C000604700BFDC4506081C46060829460608B5
:10F9D0004E4606082DE9F041154686B06A1C884659
:10F9E000BDF830600D9F194626D0030900F00F04C2
:10F9F0004033CDE90045174A05933046B847C0B1BA
:10FA0000EAB20D2AD8F8000098F8051011D82A4655
:10FA1000FBF7E8FA68B1028801780391C2F3032189
:10FA2000120BCDE900420291059B0B4A00213046A2
:10FA3000B84706B0BDE8F0817306FAD40309074A57
:10FA400000F00F000C9040333046BC4606B0BDE8D5
:10FA5000F04160475D4606086F460608994606086D
:10FA600010B5013114460EF0D1FA28B9064B1A68C8
:10FA70001B792260237110BDC27904492046BDE87C
:10FA80001040FFF773B800BF58460608BA4606088C
:10FA90002DE9F04188B01F460309DDF8388015468E
:10FAA000403300F00F0429B307930EF0AFFAC27988
:10FAB000079BCDE900420646134A29463846C0470F
:10FAC000A8B13068114DFBF7DFFAB2797179079B65
:10FAD00012F0020F0E4A08BF2A46F5790094CDE9CC
:10FAE0000101CDE9032500210A4A3846C04708B084
:10FAF000BDE8F081084A0E9429463846C44608B04D
:10FB0000BDE8F041604700BFAD460608CF5106088A
:10FB100048490608BF460608E146060803685A1C1D
:10FB2000026019700368090A5A1C02601970704754
:10FB300002681146531C036011F802CB0160D31C0C
:10FB40005178036093781B0443EA0123111D01607F
:10FB5000D07843EA0C0343EA00607047A0F1300319
:10FB6000092B07D920F02000413819288CBF00202C
:10FB70000120704701207047303809288CBF0020D1
:10FB800001207047413819288CBF002001207047A0
:10FB9000613819288CBF002001207047202805D02B
:10FBA000093804288CBF00200120704701207047CD
:10FBB000A0F14103192B98BF20307047A0F16103D9
:10FBC000192B98BF2038704710B500F10044024649
:10FBD000013C04E0B3EB0E0015D1A24214D012F8A0
:10FBE000013BA3F14100192811F8010BA0F1410CD0
:10FBF00098BF2033BCF1190F00F1200EEAD91B1A6F
:10FC000004D10028E9D110BD002010BD184610BD58
:10FC100002B310B58446841804E0B3EB0E0014D18F
:10FC2000A44513D01CF8013B11F8010BA3F14102CC
:10FC3000192AA0F1410298BF2033192A00F1200EA1
:10FC4000EBD91B1A04D10028EAD110BD002010BD49
:10FC5000184610BD1046704770B5044608460D465C
:10FC60004AF070FD064602E014F8013F43B1204619
:10FC700032462946FFF7CCFF0028F5D1204670BD5B
:10FC80001C46204670BD38B507490546FFF7E4FF1E
:10FC90000649041E284618BF0124FFF7DDFF08B1FE
:10FCA00044F00204204638BDF3460608A45E060868
:10FCB0002DE9F041044686469EF800C0BCF1200FB5
:10FCC0007046ACF109050EF1010EF5D0042DF3D903
:10FCD000BCF12B0F5BD0BCF12D0F3BD1102A4FF0A4
:10FCE000010600F1010E58D19EF800C0BCF1300FA2
:10FCF0005FD04FF010086FF070450F2742460EF1AD
:10FD0000010E00200DE0ACF1300C5FFA8CFC944544
:10FD10000FDA854274462DD32AD008FB00C01EF8A6
:10FD200001CBBCF1390FEED94CF0200CBCF1600FC7
:10FD30000BD801B10C600EB323B1B0F1004F28BF56
:10FD40004FF000404042BDE8F081ACF1570C5FFA43
:10FD50008CFCDCE7102A864649D04FF0FF35B5FB16
:10FD6000F2F502FB05F7FF43FFB290460026C6E717
:10FD70006745D2D21E404FF0FF30D0E7002BE2D0D3
:10FD80006FF00043984228BF1846BDE8F081102A62
:10FD90004FF0000600F1010EA6D04FF0FF35B5FB85
:10FDA000F2F502FB05F7FF4390F801C0FFB2904661
:10FDB000A5E79EF801C0ACF1410019280EF101043D
:10FDC000624601D80CF12002782A4FF0100805D0C5
:10FDD000A6466FF070450F27424690E79EF802C096
:10FDE0006FF070450EF1020E0F27424687E700269E
:10FDF0007AE773B50E4611490546FFF7E5FE18B9D7
:10FE00003070012002B070BD2C78602C8CBF613C3A
:10FE1000413C072C10D8013501230A2201A92846AC
:10FE2000FFF746FF019B9D4206D00F2804D80134FE
:10FE300040EA04143470E4E70020E3E7584606087B
:10FE400001230A22002133E770B50D461446FFF75F
:10FE5000B7FC0646A0B1FFF7F3FF40F63403984223
:10FE6000A8BF1846B0F5617FB8BF4FF46170A0F528
:10FE700061731920B3FBF0F32B70237801332370E7
:10FE80003046FFF79DFC0646A0B1FFF7D9FF40F6CC
:10FE900034039842A8BF1846B0F5617FB8BF4FF44D
:10FEA0006170A0F561731920B3FBF0F36B702378D8
:10FEB00001332370304670BD2DE9F84317461E46C6
:10FEC00005464FF47A720023384631464BF0FEF86F
:10FED0004449454A014482FB0143C8170B44C0EB27
:10FEE000631382FB03021A44D817404CC0EB621222
:10FEF00084FB02044FEAE27C3D48CCEBA40C80FB7F
:10FF00000C404FEAEC74C4EBE010C3EB0314A1EB1C
:10FF10008401A971C2EB0211A3EB81036B710CEB9D
:10FF20004C03A2EBC30240F2B55303FB10CCBCF56B
:10FF3000896F2A714FEA800041DA40F2DA239C454A
:10FF400046DCBCF5B77FB4BF00220122DFF8A490E5
:10FF500002EB420309EBC30391B2DB8A4FEA42088A
:10FF600008EB020409EBC40416344FF00B0E01E059
:10FF700034F8023D63451DDDBEF1010EF8D1424467
:10FF80004FF0010E39F8323085F802E000F5FA60E2
:10FF90000CF1010C0844ACEB030C288085F803C07D
:10FFA0004FF47A720023384631464BF08FF82A819D
:10FFB000BDE8F8830EF1010E5FFA8EFEE4E703213F
:10FFC000DFF8309040F296530A464FF00608C7E734
:10FFD0000221DFF8209040F229430A464FF004083E
:10FFE000BEE700BF80BC92C789888888ABAAAA2ACE
:10FFF00073B06D1678E8050808B50C4BD3E90023FB
:020000040801F1
:1000000052EA030C09D1002340F20112428083809E
:10001000837103800381184608BD054909688A1861
:1000200043F10003FFF748FF012008BDB04D002059
:10003000A82A0020884210B54FF001043ED301FBEE
:1000400004F4B0FBF4FC8C45F9D2CCB122BB08E03F
:10005000A14203F801EBB4FBF1F211D8B0FBF2FCC2
:100060001446BCF1090F0CF1570E0CF1300204FBE1
:100070001C00EDDCA14203F8012BB4FBF1F2EDD939
:1000800000221A7010BDA14203F801EBB4FBF1F29B
:10009000F6D8B0FBF2FC1446BCF1090F0CF1370E98
:1000A0000CF1300204FB1C00EDDCA14203F8012B33
:1000B000B4FBF1F2EDD900221A7010BD8446002A7B
:1000C000EAD1CEE70028BEBF2D23404201F8013B14
:1000D000092870B54FF00103864607DD03EB830363
:1000E0005B00B0FBF3F2092AF8D8EBB1104CBEFB71
:1000F000F3FCA4FB0320C008BCF1090F0CF130068F
:100100000CF15705024607D8092B01F8016B03FBD8
:100110001CEE09D90346EAE7092B01F8015B03FB52
:100120001CEE01D91346E2E700230B7070BD00BF3F
:10013000CDCCCCCC2DE9F041904282B0CDE900127B
:10014000044615460B460BD2B0FBF5F6134A05FBE9
:1001500016441846135D00F8013B02B0BDE8F0817B
:10016000B0FBF2F69642B6FBF2F706D20B4A05FB5D
:100170001767D15D03F8011BE9E7BA42B7FBF2F854
:1001800007D9064A05FB187812F8081003F8011B76
:10019000EDE74046FFF7CEFF0346F2E7245F06088F
:1001A0005F4B9A88B3F808C05889D989B2F57A7F2D
:1001B00088BF4FF47A7210B588BF9A80DA88B2F59A
:1001C0007A7F84BF4FF47A72DA80BCF57A7F88BF79
:1001D0004FF47A7C9A8988BFA3F808C0B0F57A7F7B
:1001E00084BF00205881B2F57A7F84BF4FF47A72C1
:1001F0009A81B1F57A7F84BF0021D98184459CBF63
:1002000000201881914228BF0022598B28BF9A8173
:100210009A8B914284BF00225A83424B1B8882B042
:10022000002B40D0404CA278062A97BF3F499FED53
:10023000400A01EB820191ED180A2179002958D179
:100240003C49087807EE903A07EE100AF8EEE77A94
:10025000F8EEC76AA37986EEA77A0BB130EE000AF2
:10026000B4EEC70AF1EE10FA1DDD67EE807ABCEE3F
:10027000E77A8DED017A9DF8042007EE102AB8EE9A
:10028000C77AF4EEC77AF1EE10FAC4BF0132D2B2E7
:10029000002A42D0102AA8BF1022D2B282421346AE
:1002A00038BF03460B7024494B780A78032B95BF5F
:1002B00022482248C3EB0313002394BF00EB430002
:1002C0004B70032A1E4B98BF02EB8201C3F89403C4
:1002D0009BBF02EBC10203F58273002203EB820392
:1002E00088BF0A70174A88BF03F58273136002B093
:1002F00010BD042A02D8002AD5D002E0053A032A0C
:10030000D1D9F7EE007A87EE800A4BF0D5FE23882C
:10031000984228BF18462080C5E70122BDE700BFEC
:1003200050600020F45A0020DC3C002078E80508EA
:100330006F120338EC5A00208057002094EC002004
:1003400008EC0020E45F00202DE9F04F9E4B83B0C5
:100350001B78A3F11702022A00AF05D99B4A12F8B5
:100360003310002940F0A382994E9A4BDFF8909207
:1003700093F808A0984D34464FF000082DE008F19E
:1003800001085FFA88F84308810801F0333103F06F
:1003900077330B44C10801F01131C31A5B1A03EB28
:1003A000131303F00F33A9FB03C1C909C1EB0121EA
:1003B000591A830301D5012917D0012908D9082921
:1003C00013D80AB1284203D1514649F0BFFA60B1AF
:1003D000824B0C349C4200F06382206810F00102D2
:1003E000CDD194F90430142BCDD1794811F096FD7C
:1003F000DFF81082002488F80844022011F0D2FDB2
:1004000098F80C34022B00F0DD82002800F04983BC
:10041000734BDFF8F4B17B60724B98F8659403F589
:10042000247A4FF47A7E4FF0000C5A88B2F57A7F26
:10043000B3F8462088BFA3F802E0B2F57A7F9A8825
:1004400088BFA3F846E0B2F57A7FDA8888BFA3F8C0
:1004500004E09988B2F57A7F84BF0022A3F806C031
:100460009142B3F85A10B3F85C2098BFA3F804C0C7
:10047000914293F86B2088BFA3F85AC0013A632ACF
:1004800084BF642283F86B2093F86C200132D2B2CF
:10049000092A88BF83F86CC003F166001946002260
:1004A0008D7A10F8014B0132A54238BF00F801CC1B
:1004B000032A01F10601F3D1B9F1010F18BF83F846
:1004C00085C0A4339A45B0D1474B9B78042B00F0EC
:1004D000C7823BB9444A1388B3F5F07F84BF4FF419
:1004E000F0731380414CFFF75BFE98F87814404896
:1004F000FFF746F8E17904F10800FFF741F8617D64
:1005000004F11600FFF73CF8B8F89624B8F89434D4
:100510001343B8F8982413431BB213B10123A8F86E
:100520009A347B68334A1B681A40002A00F0D18253
:10053000DA0700F139825D0440F1C3812E497A68FF
:100540000B401360DBF800200A40CBF8002013F4C6
:10055000004200F00D821F490022CA73CA77D904F5
:1005600040F10F8298F8A734DFF89090022B04BF77
:10057000012388F8A73409F178044B4602E00633DA
:100580009C420CD01A78072AF9D19978DA789142EE
:1005900002D35A79002AF2D0072021F0CFFC0023A1
:1005A00088F808344FF4806011F0FCFC002800F05B
:1005B0006C82124DAA469AF8051091B39AF8000081
:1005C00068B34B4625E000BF6158002024E00508D1
:1005D000A0EF002098570020BC0202000CF0002081
:1005E000A46400200CED0020DC3C002060670020AB
:1005F00090F0002009600002F6DFFFFDB4F000205B
:100600008180808008EC00209457002006339C42B3
:1006100007D01A788A42F9D15A79002AF6D021F007
:100620008DFC0AF1060A5445C5D1B14B93F80290EE
:10063000B9F1080F00F0E98198F8661498F865049C
:10064000AC4ADFF8F0C2DBF80030A1F10101B1FAE9
:1006500081F14909A0F101001171B0FA80F09CF814
:100660000110400910700329C3F3C030907084BF9B
:1006700000228CF80120A04AA049907B7A68126879
:100680000B400A407968CBF800300A60002800F07F
:10069000C781DFF8A4B2BBF80430002B40F0CD8155
:1006A000974A136813F07F4F1CBF002313609368B1
:1006B00023F4007323F0020313B140F2022393608A
:1006C0001379013B042B84BF01231371A9F10509A0
:1006D0008C4BB9F1030F93F800A040F23F81BAF1BF
:1006E000000F1ED000237B60814A6FF00703A3EB4D
:1006F000020902F1080B04E009EB0B039A4540F2F2
:10070000E4801BF8010B0028F6D00DF0A9FC0028AE
:10071000F2D083799B07EFD57A680123002A40F055
:10072000D980734B9B7913B1714A00239371764B37
:10073000DA8812F00C0F03D1C2F30312022A02D995
:100740004FF42062DA801A8912F00C0F03D1C2F341
:100750000312022A02D940F601221A816B4B98F843
:1007600025155A78914298F8242505D9002188F852
:1007700025154AB1A8F82815197891423EBF0022E4
:1007800088F82425A8F8282593F8EA3098F8262533
:100790005F48DFF8A8B19A4284BF002388F8263565
:1007A00000F1780A10F8013C03EB43035B4400219D
:1007B00093F87C9093F87DE093F87EC003461A7816
:1007C0004A45A8BF4A4603F8012B5A797245A8BF8B
:1007D00072465A719A7801316245A8BF6246032970
:1007E0009A70ECD11E305045DCD14A4B1A6B002A6E
:1007F00000F02D81002001212B78282B07D16B7868
:10080000043301FA03F313421CBF9A430120063557
:10081000A542F1D108B13F4B1A633F4C04F10805E2
:10082000234613F8012B072A00F28A809D42F8D153
:10083000E94688B0EA462022FF2150464CF03BFAB8
:10084000354A12F8013B5AF8231001317FD1954205
:100850004AF82330F5D1B8F85E24B8F85C349A42EF
:10086000CD4602D32D4BC8F85C34FF232C4988F8C1
:100870002E3596F90430142B04D0326831EA020286
:1008800000F0EB80274B0C369E42F2D1264B5A7972
:10089000022A01D100225A710C37BD46BDE8F08F03
:1008A00008F1FF38B8F1020F7FF6A2AD9DE502EB2B
:1008B000C3035B68002B7FF457AD1C4A17231370EA
:1008C00052E51C0779D51A4939E67A680023002ACF
:1008D0003FF427AF06494A7C002A7FF428AF4A79C3
:1008E000012A3FF41EAF002B7FF41BAF1FE700BFB0
:1008F000DC3C0020ACAC0020805700209EDDCDFD0C
:10090000E85F00206858002088630020CC65002044
:1009100097EC002098570020EF3C0020AE014A01E0
:10092000010002000CF00020983A002061580020DD
:10093000FE9FFFFD50600020C0AC002078E8050855
:10094000E94688B02022FF2168464CF0B4F9002324
:1009500004F8013B0133082BFAD17CE7624A0023FB
:100960001371BAF1000F00F0AB8001237B60BBE68E
:100970005E48C17B00293FF4F2ADD904C2773FF550
:10098000F1AD1A067FF5EEAD594B1978182906D846
:10099000584B01228A401340002B7FF4E3ADDFF86F
:1009A0006C9109F17804FAE553497A680B401360B9
:1009B000DBF800200A40CBF8002098047FF5C7AD93
:1009C0004E49BCE500283FF423ADDFF844E14C4B31
:1009D0009EF8001090F904504FF0FF0C03F16C00EA
:1009E00093F90820AA4204BF01F1FF3183F808C03F
:1009F00003F10C0304BFC9B201248342F0D1002CDF
:100A00003FF406AD8EF8001002E51A469B79002BE4
:100A10003FF412AE537C012B04BF022353740BE648
:100A200038480343CBF80030DFF8E8B0BBF80430B7
:100A300002430A60002B3FF433AE9BF800000DF038
:100A40000FFB00287FF42CAEABF8040028E628202A
:100A500021F074FA254B1A6BCCE688F82E3515E791
:100A60007A68136823F480531360DBF800301E4A61
:100A700023F48053CBF80030538CB3F57A7FBFF466
:100A800031AD4FF47A7353842CE57A68136823F000
:100A900000631360DBF8003023F00063CBF8003014
:100AA00087E5194ADFF870B013687A6023F0800395
:100AB0001360DBF8003023F08003CBF80030ABE4A8
:100AC000537C002B7FF433AE5379012B7FF42FAE90
:100AD00027E67A6843F008031360DBF8002042F051
:100AE0000802CBF8002023E5DC3C002098570020CA
:100AF0006158002000410001F79FFFFDF6BFFFFD98
:100B0000F457002000040500A4640020B4F0002085
:100B1000F1570020C0AC0020945700202DE9F04F81
:100B2000DFF870828F4BD8F80C2002F2DC52C8F844
:100B30000C208D4A934285B080F0108103F11C0592
:100B40009B468A4B8A4E4FF0010A9F1C874B5A885E
:100B5000002A00F0EB80BB18B34280F0E7803C46EF
:100B600008E01A881C461344002A00F0DF80B342D4
:100B700080F0DC80052A40F2D98035F81C2C618891
:100B8000C2F30B029142ECD162799207E9D123883A
:100B900055F8141C94F8049001935846FDF78EFB09
:100BA00035F81C2CB9EB123F00F0C8804FF0000A5A
:100BB00035F8181C55F8140CC1F30B0145F008FB6F
:100BC00055F8043C1860684B0BF11C0B9B4505F174
:100BD0001C05BBD3674A684BDFF8BC9112681A60EA
:100BE000FFF7B2FB99F80030644F654C99F801208B
:100BF00003EB830103EBC10307F5827101EB830370
:100C00002360C2EB021207F18C0303EB4202C7F828
:100C1000942320F0FDFA5B4A20684FF0FF33002454
:100C200007F2AC46536035462DF05CFC0294ADF8FB
:100C30000C40C7F83045C7F834450CE0D7F83435D8
:100C4000FA180133C7F8343582F838B50134142C5A
:100C500005F1060519D06B792846062202A95FFA2C
:100C600084FB002BEAD14BF0FCFF0028EED0D7F834
:100C700030350134FA18142C03F10103C7F830356C
:100C800082F84CB505F10605E5D106F1780202E0DF
:100C9000063696425CD03378002BF9D1B078F178E3
:100CA000884202D371790029F2D0364A137297F83C
:100CB000A434B7F8A82403EB830303EB83039B005E
:100CC000632BD8BF6423C8F80430642303FB02F20B
:100CD000632ADCBF1A46C8F808304FF00003C8BFCB
:100CE000C8F80820C8E90732274AA8F82430C8E91C
:100CF0000333C8E9053388F82630244B93622EF07D
:100D0000B9FCB7F8600597F8621521F083FF39F058
:100D100017F816F0DFFD1E4A1268C8F80C200123F0
:100D2000504688F8253005B0BDE8F08F55F8141C02
:100D30005846FDF7C3FA4FF0000A39E7019BA11DA1
:100D40009A1F5846FDF7EEFA00287FF431AF2DE7E1
:100D500099F80F30003B18BF0123A6E74FF0010AB6
:100D600038E700BF4CD00608A0D7060800400008AE
:100D700000800008A46400209457002008EC0020A4
:100D8000E45F002064040020206000209CF000202C
:100D9000A82A0020F45F00208057002070B51C4D69
:100DA00001230328064685F864351ED9711CC9B293
:100DB00049004029174A28BF4021002302244FF050
:100DC000140ED454023302EB030C99420CF801ECDC
:100DD000F7D8FF2E08BF02212944FF2381F8683588
:100DE000BDE870400E2011F0C5BA00EB800005F59B
:100DF000827306EBC00003EB8000074A074B1670B6
:100E000018602DF06FFB22F0BBFA22F08FFBCDE7CC
:100E100008EC002070F1002080570020E45F0020E3
:100E2000054BD3F8AC25012142F4001283F8A91533
:100E3000C3F8AC25704700BF08EC0020F8B5164D8C
:100E40006B78BE2B26D1022229464FF6FF70FDF7A4
:100E50008DFA124FAC1C22884AB1A618BE4219D294
:100E6000052A17D92146FDF781FA3446F3E72146D2
:100E70000222FDF77BFA0222A118FDF777FA063469
:100E8000074B641BA3F8B04541F60F53C31A5842F1
:100E90005841F8BD0020FCE7004000080080000831
:100EA00008EC0020F8B5066904460F46002E5DD117
:100EB0000368C3F30A02CAB12368396803F17842B0
:100EC000B2F5002F48D2324D2A6942F001022A6160
:100ED0004FF48010196041F0F5FD2B696FF30003AA
:100EE0002B6103283FD06FF001063FE003F1784209
:100EF000B2F5002F16D2264D2A6942F002022A616D
:100F00006B612B6943F040032B614FF0004041F0CF
:100F1000D9FD2B6966F341032B610328CCD04FF038
:100F2000FF3623E003F1774202F57802B2F5002F95
:100F3000C2D2174D2A6D42F002022A656B652B6DF5
:100F400043F040032B654FF0004041F0E7FD2B6D6F
:100F500066F341032B65E0E703F1774202F578027F
:100F6000B2F5002F04D32368043323603046F8BD64
:100F7000074D2A6D42F001022A654FF48010196076
:100F800041F0CCFD2B6D6FF300032B65A9E700BF8B
:100F9000003C02402DE9F041584F3B78B12B8AB01C
:100FA00070D1FFF74BFF80F00104E4B2544B554D74
:100FB000B3F88B30544EADF8003004F00104B54264
:100FC00062D3002C00F097801022002106A84BF07D
:100FD00072FE4E4B4E494F4A0497DB1B05934E4B16
:100FE000484F59605A6059645A6401228DF8242090
:100FF0003422DA606946022204A80025089548F0E8
:1010000063FF022269464FF6FF70FDF7AFF9044611
:10101000B74246D3022201A904A80025ADF8045026
:1010200048F052FF022201A92046FDF79FF940BA7D
:10103000C043ADF80800022204A802A948F044FF0A
:10104000079860B106ABC0F10402294618444BF082
:1010500032FE06A904A8FFF725FFCDE907509DF849
:101060002430089843B12C4B1A6942F080021A616F
:101070001A6D42F080021A65B0FA80F040090AB099
:10108000BDE8F081012491E7A988A868C1F30B01AC
:1010900045F09EF8AB691B681C35834218BF0124DC
:1010A0008DE7B7F804808DF80D50C8F30B0808F1F0
:1010B0000603ADF808303B88C3F30B02ADF80A20F5
:1010C0001B0B062202A904A88DF80C3048F0FCFE88
:1010D000062202A92046FDF749F9B96804464246AE
:1010E00004A848F0F1FEB96820464246FDF73EF9F3
:1010F0001C3704468CE70120C1E700BF0040000810
:1011000078E805084CD00608A0D70608008000083B
:1011100023016745AB89EFCD003C0240F8B5144D83
:10112000144E154FFFF710F9EB68012403F2DC535E
:10113000EB6086F8B245FFF72DFF28B13B78B12B65
:1011400002D1FFF77BFE18B9032C0DD00134F2E772
:101150000A4A0023116886F8B2350122E96085F851
:10116000252086F8B335F8BD46F000F846F0A4FA1D
:10117000F45F002008EC002000400008A82A0020AE
:1011800010B50B4A0B4C012384F864359373FFF7B9
:10119000C5FFFFF7C3FC41F20242FF23A4F8682514
:1011A00084F86A350E20BDE8104011F0E3B800BFA6
:1011B0008057002008EC002090F88730DFED6A5A55
:1011C00003EE903A90F88B3006EE103A90F88930A2
:1011D00004EE103A90F88A30F8EEE33A04EE903AD2
:1011E00090F88D3063EEA57AB8EEC66A03EE903AB9
:1011F00026EE256AB8EEC44AF8EEE44AF8EEE33A81
:1012000026EE276A24EE254A64EEA54A63EEA53A47
:10121000F0B5564D24EE064A64EEA74A63EEA73AAF
:1012200000210626F7EE002AA5F10C0C00F1660E4F
:1012300006FB01F2B7EE005AAC1890F88670024433
:10124000F0EE456A15E0012904F1060402F10602F8
:10125000EED190F8883007EE903A90F8903006EE94
:10126000903AF8EEE77AF8EEE66A27EEA55A66EECF
:10127000A56A237807EE103A66EE867AB8EEC77A4A
:1012800027EE277AFDEEC77A17EE903AFA2BA8BF21
:10129000FA2323EAE3731372637807EE103A66EEDB
:1012A000847AB8EEC77A27EE277AFDEEC77A17EE72
:1012B000903AFA2BA8BFFA2323EAE37353725CF83F
:1012C000213007EE903A002BF8EEE77A49DDA3785B
:1012D00007EE103AB8EE477A90F88C3037EE677A1E
:1012E00003EE103A87EE272AB8EEC33AB0EE627AE0
:1012F00023EE253AA2EE037A64EEA77A66EEA36A9D
:1013000067EE857A27EE877AFDEEE77ABDEEC77A3B
:1013100017EE103AFA2BA8BFFA2323EAE37393726D
:1013200017EE903AFA2BA8BFFA2323EAE3730EF8DC
:101330000130A38807EE903AF8EEE77A013167EEC4
:10134000A67AFDEEE77A17EE903AB3F57A7FA8BF5A
:101350004FF47A7323EAE3738F429381BFF673AF3E
:10136000F0BDB7EE007AC7E70AD7233C14E90508B9
:1013700090F88E306BB3B0F85A308BB190F88F2064
:1013800002EB82036421C3EB0313B3FBF1F3A0F878
:101390005A30962312FB03F3B3FBF1F3A0F85C3051
:1013A00043884BB190F88F3003EB8303C3EB0313F7
:1013B0006422B3FBF2F34380B0F846304BB190F8AF
:1013C0008F30962213FB02F36422B3FBF2F3A0F8F2
:1013D0004630704790F821304BB3438B83B190F87F
:1013E0002230FA2213FB02F203EB8303B3F57A7F78
:1013F000A8BF4FF47A7364218383B2FBF1F2428376
:10140000838843B190F82230FA2213FB02F364225E
:10141000B3FBF2F38380C3884BB190F8223003EB27
:101420008303B3F57A7FA8BF4FF47A73C380704704
:1014300070B50A4C0A4E002594F8863013B1204648
:10144000FFF7BAFE2046FFF793FF01353046FFF75E
:10145000C1FF042D04F1A404EED170BD0CED0020F9
:1014600050600020034BD3F8B40508B106F0DEBE8F
:10147000704700BF08EC002008B50B46054902463E
:10148000D1F8B40528B10449FDF75EFABDE808407B
:10149000E8E708BD08EC002091F600080FB407B596
:1014A00004A951F8040B0191FFF7E6FF03B05DF8C2
:1014B00004EB04B0704738B50B4B03EBC0050C468A
:1014C00095F82022094803EB8203D3F8B010FFF708
:1014D000E5FF95F826322BB1611C0548BDE8384080
:1014E000C9B2DBE738BD00BF78E80508625D0608D1
:1014F000F5480608024B0146D3F8B405FEF7CAB812
:1015000008EC002008B504460848FFF7F3FFFFF792
:10151000A9FF074BD3F8880010F0B0FE0CF0D2F909
:10152000012C01D146F0C8F8FBF774FFF646060817
:1015300008EC00200048DDE7CD5106080CB4C306D6
:1015400007B500D561B9049805A90191FFF794FF8B
:10155000FFF7F0FF012003B05DF804EB02B0704725
:101560000020F8E708B5FFF7C5FFBDE80840E1E750
:1015700010B504460348FFF7BDFF2046BDE8104004
:10158000F0E700BF0247060808B5034610462AB137
:10159000DB0600D511B1FFF7EBFF002008BD2DE9F8
:1015A000F04F2DED028B0A468BB000218246FFF7EB
:1015B000EBFF6F4D814605F1800B00266D4B1C78CB
:1015C000AB7AB34200F395801035AB45F5D140F2CC
:1015D0001620FCF75DFED0E902530CB12C461D46E7
:1015E0000DF1100B1522002158464BF064FB00272B
:1015F0002E78002E44D06978039130460CF006FD19
:1016000095F9023002935A1C534208EE100A5341D6
:10161000002C00F0A9800399002214F802C0B44500
:1016200004EB020040F09C8090F90280029A42454F
:1016300040F0948042788A4208BF012301220BF8CF
:10164000072003F001034A4683F00101504603934B
:10165000FFF79AFF039B81464CB1474A18EE101AD8
:10166000CDE900A230464246FEF7B4F9039B434A57
:1016700018EE101ACDE900A23046029AFEF7AAF938
:101680000137152F05F10305B2D16CB33A4FDFF8DE
:10169000EC8004F13F061BF8013B02930BBB207862
:1016A000F8B194F9022001321BD061780CF0AEFC45
:1016B0004A46054601215046FFF766FF94F902208D
:1016C000029B294681462078CDE900A7FEF782F9E2
:1016D0002078029BCDE900A84FF0FF322946FEF7A3
:1016E00079F90334B442D6D10BB0BDEC028BBDE81E
:1016F000F08FE888FCF7CCFDD0E902230CB114464A
:101700001A46297A6B7A06FB013312F9038014B367
:10171000E756B8450CBF012300234A4614BF0121F8
:10172000002150460293FFF72FFF029B814644B1F0
:10173000114A3146CDE900A228463A46FEF7FEF8A6
:10174000029B0E4A3146CDE900A228464246FEF7EA
:10175000F5F8013632E74FF0FF37DAE700236DE79F
:1017600003323F2A7FF459AF4FF0FF386BE700BFD9
:101770007004002008EC0020591901083D150108EB
:1017800008B50948FFF7F4FEFFF76CFE074B00248D
:1017900083F8B845C3F8B84683F8BC4621F096FFF5
:1017A0002046FFF7AFFE00BF0747060808EC002001
:1017B0002DE9F04F8BB0074640F216200391FCF75D
:1017C00067FD039A044600213846FFF7DDFE404AD4
:1017D000D4E90253147806460CB12C461D46152256
:1017E000002104A84BF067FA05F13F03039395F835
:1017F0000090B9F1000F31D095F801A0002C65D010
:10180000224600231178494558D128336B4492F879
:101810000180012203F8182CD045324614BF012163
:10182000002138460CBF4FF0010B4FF0000BFFF7C3
:10183000ABFE064654B1B8F1000F07D0254B00931C
:101840005A463B4641464846FEF722F9224B009352
:101850005A463B4651464846FEF71AF9039B033564
:101860009D42C4D13CB3DFF86C90DFF86CA0651CDE
:101870000DF11008403418F8013BCBB915F8013CC4
:10188000B3B116B13046FFF773FE297815F8010C95
:10189000CDF800903B460022FEF7FAF8002215F83A
:1018A000010CCDF800A03B461146FEF7F1F80026EA
:1018B0000335A542DFD10BB0BDE8F08F0133152B06
:1018C00002F103029ED14FF00008A5E7A046A3E76E
:1018D00008EC0020591901083D150108154B1B683B
:1018E00070B52BB31448154EFFF73CFEFFF7BAFD59
:1018F000FCF7E0FA0025FCF713FB044640B1132087
:1019000010F038FDFFF716FEBDE870400C4829E6E0
:101910003046FFF7C3FD782D06D80135FFF7A2FD4D
:1019200064200BF0EDFFE6E7FFF704FE2546F5E740
:1019300070BD00BF0C2B00202E4706084CB50608D2
:1019400048470608034B0146D3F8B40508B106F032
:1019500059BC704708EC00200CB407B510F020000B
:101960000BD079B92320FFF7EDFF049805A9019169
:10197000FFF782FDFFF7DEFD012003B05DF804EB09
:1019800002B070470020F8E72DE9F04F914689B08A
:101990000C461A4600218046FFF7F6FDDFF8ECB052
:1019A00006464D460027B9F1000F6CD029460622A5
:1019B00020464BF056F90028324614BF0121002181
:1019C00040460CBF4FF0010A4FF0000AFFF7DCFD64
:1019D0000646287815F052FF079010B3687915F085
:1019E0004DFF079BEA785B790793AB7895F801E0A8
:1019F0004FF461714FF0190C1CFB03131CFB021216
:101A0000297900B14079CDF804E0CDE90232079B95
:101A10000093CDE904103B465A4651464046FFF735
:101A20009BFF207815F02AFF079010B3607915F01E
:101A300025FF079BE2785B790793A37894F801E090
:101A40004FF461714FF0190C1CFB03131CFB0212C5
:101A5000217900B14079CDF804E0CDE90232079B4D
:101A60000093CDE904103B465A4651464046FFF7E5
:101A700065FD0137142F04F1060405F1060592D126
:101A800009B0BDE8F08FCA46CBE700BF4E47060855
:101A90002DE9F04F174689B01A460C4600218146C1
:101AA000FFF772FD3B4EDFF8F4B007F16C038046A0
:101AB0003D46079394F90410374A002392F9080031
:101AC000884263D00133092B02F10C02F6D1079B47
:101AD0000C359D4204F10C04ECD109B0BDE8F08F47
:101AE00029460C2220464BF0BCF80028424614BF81
:101AF0000121002148460CBF4FF0010A4FF0000AB7
:101B0000FFF742FDEA7995F9043006EB8202804640
:101B1000D2F8002304922A7A06EB82025146D2F8C8
:101B200000230392AA7906EB82024846D2F80023EA
:101B300002926A7906EB8202D2F8002301922A68A7
:101B400000925A46FFF708FFE27994F9043006EB59
:101B500082025146D2F800230492227A06EB8202D6
:101B60004846D2F800230392A27906EB8202D2F80B
:101B700000230292627906EB8202D2F800230192DE
:101B8000226800925A46FFF7D9FCA0E7002FA7D1A0
:101B9000BA46D9E778E80508F457002067470608F1
:101BA0002DE9F04F8BB00C46089200211A460746EB
:101BB000FFF7EAFCDFF8B4B0089D099000264FF06B
:101BC00019094FF46178089B002B4BD029460A2253
:101BD00020464BF046F80028099A14BF0121002145
:101BE00038460CBF4FF0010A4FF0000AFFF7CCFC5B
:101BF0002A890692EA8805922A790492EA78039261
:101C0000AA78099019FB028202926A7819FB028273
:101C100001922A78009233465A4651463846FFF7D9
:101C20009BFE22890692E288059222790492E2784C
:101C30000392A27819FB02820292627819FB028257
:101C4000019214F80A2B009233465A465146384600
:101C50000136FFF773FC1E2E05F10A05B3D10BB058
:101C6000BDE8F08FDDF820A0DBE700BF8447060861
:101C70002DE9F04F2DED088BDFF82CA195B08046B3
:101C800091461F460C4616464FF0000B94ED008A15
:101C9000B5EE408AF1EE10FA7FD0D4ED019A94EDC2
:101CA000029AD4ED038AB9F1000F49D0D6ED00BAFB
:101CB00096ED01BAD6ED02AA96ED03AAB4EE6B8AB0
:101CC000F1EE10FA6ED1F4EE4B9AF1EE10FA69D102
:101CD000B4EE6A9AF1EE10FA64D1F4EE4A8AF1EEAB
:101CE00010FA0CBF012100213A460D46404681F012
:101CF0000101FFF749FCB0EE6B0A074611A8FDF79A
:101D000059FCB0EE4B0A07900EA8FDF753FCB0EE5D
:101D10006A0A06900BA8FDF74DFCB0EE4A0A059042
:101D200008A8FDF747FC0599069A079B03900291C6
:101D30000192009352465B4629464046FFF70CFE4F
:101D4000B0EE480A11A8FDF735FCB0EE690A054669
:101D50000EA8FDF72FFCB0EE490A06900BA8FDF780
:101D600029FCB0EE680A059008A8FDF723FC069B45
:101D7000059A0390CDE9005302925B46524600213A
:101D800040460BF1010BFFF7D9FBBBF1080F04F143
:101D9000100406F110067FF479AF15B0BDEC088B86
:101DA000BDE8F08F00219FE7A74706082DE9F74F10
:101DB00092460C461A4600218146FFF7E5FBDFF804
:101DC00070B0804656460025BAF1000F2ED031463D
:101DD000042220464AF045FF0028424614BF012154
:101DE000002148460CBF01270027FFF7CDFB738871
:101DF00001933AF82530009380462B465A463946DF
:101E00004846FFF7A9FD6388019334F8043B00932B
:101E10005A462B46394648460135FFF78FFB042DBD
:101E200006F10406D0D103B0BDE8F08F5746EAE7CB
:101E3000BB4706082DE9F04F89468FB017460021B1
:101E40001A460646FFF7A0FBDFF878A005460024F7
:101E50000DF1240B59F824300293594602A842F0A0
:101E6000ADFA67B357F82430029A0393934218BF30
:101E700001212A4608BF002130460CBF4FF001085F
:101E80004FF00008FFF780FB04A9054603A842F0C5
:101E900095FA04A900912346524641463046FFF781
:101EA0005BFD2346CDF800B0524641463046013432
:101EB000FFF744FB402CCDD10FB0BDE8F08FB84602
:101EC000EFE700BFCC4706082DE9F04F924685B0FA
:101ED0000C461A4600218146FFF756FBDFF874B026
:101EE000804655460026BAF1000F31D0294604221B
:101EF00020464AF0B6FE0028424614BF01210021C8
:101F000048460CBF01270027FFF73EFBEB78029302
:101F1000AB7801932B880093804633465A46394666
:101F20004846FFF719FDE3780293A378019334F84C
:101F3000043B00935A463346394648460136FFF77C
:101F4000FDFA102E05F10405CDD105B0BDE8F08FE6
:101F50005746E8E7D64706082DE9F04F87B0144604
:101F600003911A4600210546FFF70EFBDFF838B152
:101F700006464FF00008062303FB08F707F5A07795
:101F80004FF00009039BDB5D0493002C00F0888078
:101F9000E35D049A05939A4218BF0121324608BFB7
:101FA000002128460CBF4FF0010A4FF0000AFFF74E
:101FB000EBFA059B0646CDE900935A464346514647
:101FC0002846FFF7C9FC049B5A46CDE900935146C9
:101FD0004346284609F10109FFF7B0FAB9F1060FA7
:101FE00007F10107CED108F10108B8F1060FC2D1FF
:101FF000DFF8B4B04FF4B277039BA7F5B27913F8CA
:1020000007A0002C4ED0E35D04939A45324614BFDE
:102010000121002128460CBF4FF001084FF00008B5
:10202000FFF7B2FA049B0646CDE900935A46062311
:1020300041462846FFF790FC0623CDE9009A1A4A4C
:1020400041462846FFF77AFA013740F26F139F4264
:10205000D2D1039B93F86F71B4B194F86F81474567
:10206000324614BF0121002128460CBF0124002460
:10207000FFF78AFA002300930B4ACDF80480072368
:1020800021462846FFF768FC00230093064A019783
:10209000072321462846FFF751FA07B0BDE8F08F25
:1020A000A24690E7A046C7E7E84706082DE9F04FAB
:1020B00089B00C46079200211A460746FFF764FADA
:1020C0000026079DDFF8A0B00690B2464FF0190930
:1020D0004FF46178079B43B32946062220464AF015
:1020E000C0FD0028069A14BF0121002138460CBF0C
:1020F0004FF0010A4FF0000AFFF746FA6A7906909E
:1021000019FB028205922A7919FB02820492EA786D
:102110000392AA7802926A7801922A780092334652
:102120005A4651463846FFF717FC627919FB02827E
:102130000592227919FB02820492E2780392A27836
:1021400002926278019214F8062B009233465A46A6
:10215000514638460136FFF7F1F90A2E05F106051A
:10216000B8D109B0BDE8F08FFC4706082DE9F04F63
:102170000F4689B0144600211A460646FFF704FAB6
:102180000546002C00F0DB8022783B789A4218BF8D
:102190000121024608BF002130460CBF4FF0010864
:1021A0004FF00008FFF7F0F923789B4A05464146B7
:1021B0003046FFF7D1FB3B78974A41463046FFF760
:1021C000BDF9002C00F0BD8062787B789A4218BF80
:1021D00001212A4608BF002130460CBF4FF00108FC
:1021E0004FF00008FFF7D0F963788C4A0546414666
:1021F0003046FFF7B1FB7B78884A41463046FFF70F
:102200009DF907F1CA030493822304F1CA0B0593D5
:102210004FF002094FF0000A3B78534500F39380DA
:10222000002C00F0F38097F8EA3094F8EA209A4204
:1022300018BF01212A4608BF002130460CBF4FF0CD
:1022400001084FF00008FFF79FF994F8EA30744A4C
:10225000054641463046FFF77FFB97F8EA30704A63
:1022600041463046FFF76AF907F1EC09002C00F00F
:10227000CF8004F1EC034A4604F1FC014FF0010861
:102280009A4633F802CB32F8020B844518BF4FF060
:1022900000088B42F5D188F001012A46C9B23046C8
:1022A000FFF772F9082105465046FDF7CBFA5D4A63
:1022B000034641463046FFF74FFB97F8EA10484681
:1022C000FDF7C0FA574A034641463046FFF736F954
:1022D000002C00F09F804FF0FC094FF0010807EB45
:1022E000090104EB0900FDF76FFC09F1040900285E
:1022F00018BF4FF00008B9F58E7FF0D188F00101CA
:102300002A46C9B23046FFF73FF9082104F1FC0024
:10231000FDF7DEFA444A034641463046FFF71CFB10
:1023200097F8EA1007F1FC00FDF7D2FA3E4A03469F
:102330004146304609B0BDE8F04FFFF7FFB8A04670
:1023400039E7A04657E7059B3B440693002C5BD03A
:10235000059B0698234419460793FDF735FC049B1B
:102360001A789BF800309A4206BFB0FA80F84FEA1C
:1023700058184FF000084B4609F11002F85AE15A7C
:102380000233884218BF4FF000089342F6D188F01C
:1023900001012A46C9B23046FFF7F6F8627804EB2D
:1023A000090105469BF81800FDF71DFA02909BF8FD
:1023B00000300193079B00931C4A0AF10103414638
:1023C0003046FFF7C9FA049B7A78187E079307EB2B
:1023D0000901FDF708FA079B049A02901B78019304
:1023E0000132069B04920AF1010A00930F4A5346F8
:1023F00041463046FFF7A2F8059B09330BF1010B6C
:1024000009F11009059307E7A046DCE7A04624E799
:10241000A04652E7A04683E7154806082748060865
:10242000554806086D480608844806083C480608D2
:102430002DE9F04F89B00F4691460021139A984636
:102440000646FFF7A1F887EA09096FEA0903DFF8F2
:10245000849006930446002528460FF029FD129B20
:10246000184230D0069BDFF870B0034014BF4FF025
:10247000010A4FF0000A049310EA070314BF4A460A
:102480005A462846059307920FF024FD079A0390B9
:102490000090434651463046FFF75EFA049BB3FA7C
:1024A00083F1224649093046FFF76EF8059A039BEF
:1024B000009304464346002A14BF5A464A465146F2
:1024C0003046FFF73BF80135182DC5D109B0BDE8FE
:1024D000F08F00BFB54706089B4806082DE9F04F6E
:1024E0000A4687B000210646FFF74EF83B4C0590A0
:1024F0003B4A2378608802EB8303D3F8B0A0FBF754
:10250000C7FE83680493374BC1681A78002A4BD002
:10251000DDF810800491002721796279049B07FB84
:10252000012213F80290B8F1000F3FD018F80250C2
:10253000059A4D4514BF0121002130460CBF4FF0D4
:10254000010B4FF0000BFFF71FF8013705907DB32B
:1025500005F00F022D0940350292CDE90075224A9F
:10256000534659463046FFF7F7F9B9F1000F2AD024
:1025700009F00F024FEA1919029209F14002CDE960
:1025800000725346184A59463046FEF7D7FFA279E3
:10259000012A38BF0122BA42BEDC144B0834A342E0
:1025A000A6D107B0BDE8F08F9046B4E74546BFE737
:1025B000B8F1000FD9D00E4A00975346594630461D
:1025C000FFF7CAF9D1E77306E1D4094A00975346E9
:1025D00059463046FEF7B2FFD9E700BF98EA050832
:1025E00078E8050808EC0020A248060878EB050802
:1025F000B84806080FB407B504A951F8040B0191B7
:10260000FEF73AFFFEF796FF03B05DF804EB04B067
:1026100070472DE9F041037903F0E002402A51D0E0
:1026200004D85AB1202A29D0BDE8F081602A4CD0C4
:10263000802AF9D182794179264812E003F0070314
:10264000052B16D8DFE803F0101510150309D0F894
:1026500005102148BDE8F041CCE7D0F805205142F3
:102660001E48BDE8F041C5E7B0F80720B0F80510F6
:10267000F6E7B0F90720B0F90510F1E74679184DF3
:10268000184805EBC605FEF735FF95F8447300249E
:102690000123A74203D8BDE8F041FEF74BBFD5F8B0
:1026A000406356F824204FEA84084AB113B90E4813
:1026B000FEF720FF56F808100C48FEF7EFFE002347
:1026C0000134E6E741790A48C4E7BDE8F04109482A
:1026D00090E700BF1B490608CC480608E2480608F8
:1026E00078E80508F9480608594C0608625D0608AE
:1026F0000A490608324906082DE9F04387B0FBF77E
:10270000C9FB02698389018802928268019242882A
:10271000009242681B4EDFF880801B4FDFF87C90F0
:1027200004461A48FFF766FF002515B94046FEF734
:1027300019FF3B689D4213DA33781548052B96BF85
:1027400009EB83030022D3F8E824B38800932946D9
:1027500073880135FFF74EFF062D06F10606E4D11A
:1027600044F016F981884388CB1A616803FB011194
:102770000591FBF719FC05990246064807B0BDE82C
:10278000F04337E74C4E0020BC4D00204A49060874
:10279000B4490608C3490608A849060878E80508A8
:1027A0000249034801F5FD610EC923E700F0FF1F50
:1027B000E049060810B5752104462DF005FA0146DA
:1027C0000948FFF717FF1A2120462DF0FDF90146B1
:1027D0000648FFF70FFF1B2120462DF0F5F9BDE855
:1027E00010400146024805E7F4490608074A060872
:1027F0001A4A060838B50B4DE87810F0FD0405D1EB
:102800000948FFF7F7FE2046FFF7D4FFEB78013BBE
:10281000012B06D80548FFF7EDFEBDE83840012042
:10282000C8E738BD506000202D4A0608384A06081F
:102830002DE9F04F634B644C1A686449644B65485A
:10284000B2FBF3F293B0FEF729FEB4F8BE26624E57
:10285000624FDFF8E081DFF8B0914FF47A73B2FB9A
:10286000F3F103FB11220A20B4F9C03692B2B2FB95
:10287000F0F25B48FFF7BEFE5A4A5B495B48FEF741
:102880000DFEFEF757FE5A4B5A4A997B5A4B5B484E
:1028900006EB8101D31AD1F80015B4F8B025FFF783
:1028A000A9FE5748FEF726FE94F8C2165548FEF7D3
:1028B000F5FD5548FEF71EFE94F8C3165348FEF783
:1028C000EDFDFEF737FE5248FEF714FE00210A46E2
:1028D000FB7F0B4113F0010F01F1010508D012B18C
:1028E0004846FEF707FE29464046FEF7D7FD01227F
:1028F000072D2946ECD1474D95F8CA1405F5C47348
:1029000005F13C02012918BF134693F88C30032BC4
:1029100002D04148FEF7C2FD404B95F8CA14A3F51A
:10292000A672012918BF134693F88C30012B02D1EF
:102930003B48FEF7B3FD394B95F8CA14A3F5A672D0
:10294000012918BF13461B695B7B012B02D935484F
:10295000FEF7A4FD344FDFF8E0A0DFF8E0B0FEF7AB
:10296000E9FDD4F8C4360393002507F1200957F890
:10297000041B002964D0012303FA05F8039B18EA1D
:10298000030F1CD018F01F0F19D01AF8050059F8C2
:10299000252052F8202035B12448CDE90412FEF755
:1029A000A9FDDDE904125846FEF778FDB8F1020FE3
:1029B00005D194F8E51611B11D48FEF76FFD0135FC
:1029C000D5E700BF0000002008EC00204B4A0608B5
:1029D00040420F00544A060878E80508506000207D
:1029E000674A0608F0FF022000080000884A06082F
:1029F000805700200080000800400008AC4A06080C
:102A0000DB4A0608ED4A0608F54A0608F74A0608B2
:102A1000FF4A0608F45A0020184B06087C5C002088
:102A2000204B0608254B060880ED0508594C060882
:102A3000334B06080F4B0608F00400202D4B060808
:102A4000FEF778FD7A4B7B481A687B4B1978137A2E
:102A5000527A06EB8101D1F83C15FFF7CBFD774B9D
:102A6000774819684FF47A73B1FBF3F1FEF716FD5E
:102A700007A8FDF7C1FA38B107A90AA847F052FB29
:102A800070480AA9FEF70AFDFEF754FDD4F8A827FE
:102A9000002A00F0888007EE902ADFED6B6AB8EE1E
:102AA000E77AC6EE877AFDEEE77A17EE903AB4F849
:102AB000600E58B107EE900ADFED636AF8EEE77A30
:102AC00086EEA77AFDEEC77A17EE900AD4F828575B
:102AD0005DB107EE905ADFED5C6AF8EEE77A86EEBC
:102AE000A77AFDEEC77A17EE905AB4F8621E6429F1
:102AF000A8BF6421CDE900055448FFF77BFD94F899
:102B0000643E94F8652EB4F8681E514806EB8303C2
:102B1000D3F85035FFF76EFD4E4B4F48198889B2F8
:102B2000FFF768FDFBF7B6F9016921B182684B48F0
:102B3000120DFFF75FFD4A48FEF7DCFC494B1B68AE
:102B40001B0660D594F8943E032B8CBF464847483B
:102B5000FEF7D0FC94F80C34022B26D14448FEF743
:102B6000C9FC94F8943E042B44D84248FEF7C2FCBA
:102B700094F8A43E002B44D006EBC303D3F86815A9
:102B80003D48FEF78BFCFEF7D5FC3C483C4FFEF77A
:102B9000B1FCD4F8AC450125002C38D1FEF7CAFCB5
:102BA00013B0BDE8F08F134681E702200FF01CFA46
:102BB000054608B93348D2E737F0A8F895F904106C
:102BC00006EB80000131D0F800232F48FEF766FCA9
:102BD00094F80F34012B04D12C48FEF78BFC2C48C1
:102BE000BDE7AB792B4806EB8303D3F80013FEF760
:102BF00055FCF4E794F80E340BB92748B6E727489C
:102C0000B4E72749BCE72748FEF774FCBBE794FA12
:102C1000A4F3B3FA83F305FA03F206EB8303384611
:102C2000D3F89C1524EA0204FEF738FCB4E700BF91
:102C300000640020374B0608FC630020A82A00200F
:102C4000494B0608634B060800247449764B060876
:102C5000BC4B0608AC4D0020E34B0608F24B0608BF
:102C60000D4C060894570020134C06081F4C06080C
:102C70002F4C060800B60608774C0608934C060849
:102C8000834C0608354C06083F4C0608534C060892
:102C9000584C0608804706085C4C06086C4C060831
:102CA000434A0608874C06082DE9F04FDFF8788183
:102CB00098F8033099B0002B00F098805148524E9C
:102CC000DFF868B1DFF86891DFF868A1FEF74AFC29
:102CD00000252F460BA9E8B215F014F89DF8343002
:102CE000002B53D0139C54B107EE904A9FED470A36
:102CF000F8EE677A80EE270A49F0DEF904460B9A6F
:102D000029465846FEF7CAFB109A002A70D002FBEB
:102D100004F04FF47A73B0FBF3F30993DDF848C085
:102D2000BCF1000F66D00CFB04F142F21073B1FB52
:102D3000F3F198F80330082D18BF7F18002B5BD0F3
:102D40001798079015980690169805900A231198E1
:102D50004FF47A7EB0FBFEFE0998CDF810E0B1FB8F
:102D6000F3FE03FB1E11CDE902E10999B1FBF3F17A
:102D700003FB1100CDE90010BCFBF3F321465046E4
:102D8000FFF738FC0023C6E90D33B36201351D2D72
:102D900006F140069ED198F8033023B31C4C1D4821
:102DA000D4F8AC2ED4F8A81ED2084FF47A73B1FB35
:102DB000F3F3D4F8B01EFFF71DFC0A221648B7FB48
:102DC000F2F102FB1172FFF715FC144B1B78432B39
:102DD00006D1D4F8B42ED4F8B81E1148FFF70AFC77
:102DE0000023C4F8B03E19B0BDE8F08F0D4866E787
:102DF000099293E761469CE721464846FFF7FAFBB4
:102E0000C0E700BFA94C060828F300208096184BA5
:102E100008EC0020504D0608704D06089F2B00203E
:102E2000944D0608074D060880570020114D0608EE
:102E300040500608204D060810B586B00E4B04938E
:102E40000E4B03930E4B02930E4B01930E4B0F4A06
:102E50000F49009304460F4B0F48FEF71FFBFEF788
:102E600069FB3CB10D4A0E490E4806B0BDE8104062
:102E7000FFF7C0BB06B010BDFE4D0608034E0608A6
:102E80000E4E0608174E0608234E0608BE4D0608CD
:102E9000C84D060887570020D34D0608294E06085E
:102EA000394E06083E4E06080120C5E713B52C48EA
:102EB000FEF720FB2B4B93F82130002B4DD02A4CF2
:102EC0002A48FEF74FFB94F8503F2BB194F8523F3D
:102ED00013B194F8513F7BB9254B264893ED280A4E
:102EE0008DED010AFEF706FBB4F8603E9DED010A88
:102EF00033BB2148FEF736FBB4F8541F1F48FEF7DA
:102F0000CDFA94F8503F13B31D48FEF72BFBB4F8ED
:102F1000581F1C48FEF7C2FA94F8523FCBB118482C
:102F2000FEF720FBB4F8561F1748FEF7B7FA94F8DF
:102F3000513F83B1124802B0BDE81040FEF712BB0A
:102F400049F0BAF881B21148FFF754FBD4E71048B2
:102F5000DBE70F48E4E70E48EDE70E48EBE700BF7C
:102F60006B4E06089857002008EC0020814E06089A
:102F7000C4FA0020884E0608A24E0608B14E060884
:102F8000D14E0608E14E0608FB4E0608AC4E060878
:102F9000DA4E060897CC06082DE9F04F6F4B1B78E8
:102FA00089B0002B00F0D4806D4D6E48A9686E4C3E
:102FB000DFF8F0A1FFF71EFB69686C48FFF71AFB0A
:102FC0006B4B6C48D4F8702FD3E90031C91AB1FBB0
:102FD000F2F2FFF70FFBFEF7ADFA6748FEF7C2FA11
:102FE0006648FEF7BFFA04F674734FF000080793C3
:102FF000634B1B785FFA88F4A34222D8614C624F7E
:10300000FEF798FA2646002556F8041B3846013587
:10301000FEF744FA162DF7D1FEF78CFA5A4E012529
:10302000234661681B683046C91A0135FEF736FA37
:10303000162D04F10404F3D109B0BDE8F04FFEF7FA
:1030400079BA079B142603EB840306FB045693ED21
:10305000000AB6F80E9049F02FF896F81EE01EF020
:10306000010F14BF52222D221EF0020F14BF542351
:103070002D231EF0040F07EE903A14BF56232D2384
:103080001EF0080F14BF4FF0430C4FF02D0C81B20F
:103090001EF0800F4FF03C0BB1FBFBF105914FF0A0
:1030A000640114BF4FF0530E4FF02D0E80B201FBA0
:1030B00009F1671CCDE902E10093049017EE903A04
:1030C000CDF804C039465046FEF7E8F9B37FDB0778
:1030D0003AD55C232D4A6343D118D05891ED010AAB
:1030E00070B1DFED2B7AB8EE400A20EE270A07EE2A
:1030F000900AF8EE677A80EE270A48F0DDFF00B20A
:10310000642290FBF2F102FB11022248FEF7C6F99D
:10311000142101FB075701FB0454F988628A0491CA
:10312000218B0391E18A0291A18B0191A18A0091E7
:1031300002F0030319214B431748218A9208FFF735
:1031400059FA08F1010853E71448FEF7D3F9DFE70D
:10315000134809B0BDE8F04FFEF704BA881D0020FF
:10316000902E00201B4F060808EC00202B4F06086D
:103170000C300020424F06086F4F0608CB4F060860
:10318000685800203C2F00207B500608B02B002000
:1031900000401C4644500608595006085050060886
:1031A0007F500608275006080EB403B503AA52F84C
:1031B000041B0192FCF780FA064BD3F8B4251AB928
:1031C00005495868FCF766FA02B05DF804EB03B0F5
:1031D000704700BF08EC0020CD5106082DE9F047EC
:1031E00098460B7903F0E004402C81460F461646C2
:1031F00031D1684DDFF8A081DFF8C091002422E0D2
:103200003B7903F00703013B042B04D8DFE803F00C
:1032100006080B0E2000315D28460AE03157FBE717
:1032200036F81410F8E736F91410F5E756F82410BC
:103230004046FEF733F97B79013BA34202DD484665
:10324000FEF758F901347B79A342D9DCBDE8F08759
:1032500056F82410E0E703F00703052B58D8DFE801
:1032600003F0030C141619313578602C5ED045D864
:10327000002C66D0202C7CD0E8E796F90050602C1A
:1032800054D03BD8002CF5D148E03588EDE7B6F9AD
:103290000050F4E7D6F800A0202C554669D02BD872
:1032A000002CD3D151463C48FEF7F8F8D7F805106A
:1032B0008A4518D8B8F1000FC8D03848BDE8F047A3
:1032C000FEF7ECB8202C356853D015D8002CBDD1B2
:1032D00029463048FEF7E2F8D7F80510A94202DB8C
:1032E0004B42AB42E6DDFEF725F93A682C492B4606
:1032F0004846BDE8F04757E7602C17D0802CA5D191
:103300003178284B2848002914BF31461946D5E7A3
:10331000202C2DD007D8002C98D12546B7F9054090
:10332000B7F9076011E0602CE8D100257B7945FAF8
:1033300003F3DB07BDE8F0474CBF1C481C48FEF711
:10334000ADB8B7F80540B7F8076012482946FEF750
:10335000A5F8AC42C7DCAE42C5DBB8F1000F3FF4C4
:1033600075AF324621461348BDE8F047FEF796B8E0
:1033700000257A79104B03EBC20393F8442395425E
:10338000B1DAD3F8403353F82500BDE8F047FEF733
:10339000B1B800BFF6480608DF4806089B5006088B
:1033A000A1500608D0B50608625D06084749060820
:1033B00097CC06082246060878E80508F54A06086C
:1033C0002DE9F04F85B0164601911A46824600213C
:1033D0003046FEF7D9F8324C06F0100305464FF0A0
:1033E00000090293FEF73EF82379019A03F01803CF
:1033F000934203D0002A48D1182B46D1284B4FF0D6
:103400000D0B0BFB0933B3F80900FAF741FF8046B7
:103410002046FCF761F8D8E902210746024401443E
:103420002046FBF7F1FF80F001012A460390C9B264
:103430003046FEF7A9F8DDE90223054602B123BBB9
:10344000174A0BFB09FB52F80BB0B2060FD573B944
:10345000144803935946FEF721F8D8F80820039B37
:103460003A4421465046FFF7B9FEFEF763F80E488E
:103470005946FEF713F8D8F80C2000233A442146A9
:103480005046FFF7ABFEFEF755F809F1010940F28F
:103490004B23994504F10D04A4D105B0BDE8F08F8C
:1034A000C4F90508BB500608BC50060813B504460D
:1034B000084601920091FCF72BF9DDE90013024662
:1034C000204602B0BDE8104088E60EB403B503AA5A
:1034D00052F8041B0192FCF7EFF8054B05495868B8
:1034E000FCF7D8F802B05DF804EB03B0704700BFFA
:1034F00008EC0020CD5106080049E6E7C650060852
:1035000038B50C46054615492046FCF75DFB30B939
:10351000FDF78EFF1248BDE83840FEF723B8114989
:103520002046FCF751FBA8B90F4A82F88A0182F8BD
:10353000920182F82E0282F8360282F8D20282F8D4
:10354000DA0282F8760382F87E03084A82F82100C4
:103550000748E0E72846BDE83840CDE7D5500608E3
:10356000DB500608F650060808EC002050600020EA
:10357000FE50060801490246A7E700BF1A51060897
:103580002DE9F04380468BB00846FBF7DBFF40B1E6
:1035900000234D491A4601200BB0BDE8F043FEF769
:1035A00077BACDE90700099008464D1CFCF748FCA6
:1035B00044B220460EF09CFC0646002842D08DF80E
:1035C000204001242846FCF7FBF8054638B10023CB
:1035D0000A221946FCF76CFB01340790E4B2DFF8CD
:1035E000F09000272846FCF7EBF8054618B3FCF7E7
:1035F00027FC3649002251F804CB6045D3B203D0F2
:103600000132102AF7D1002309EB8302D2F80023FC
:10361000904210D1022F1CD0032F1FD05A1E012F11
:10362000D2B211D00B2A03D88DF821300134E4B284
:103630000137042FD6D1052C16D840460BB0BDE873
:10364000F04397E70446BDE7042AF1D88DF822300D
:10365000ECE7052BECD88DF82430E7E79A1E0D2A0D
:10366000E6D88DF82330E1E707AB03CB9DF82320A4
:1036700030601868164B716003EB8202B060D2F8BC
:10368000002304929DF8242003EB82020021D2F84B
:10369000002303929DF8222003EB82020846D2F811
:1036A000002302929DF8212003EB8203094AD3F8FC
:1036B00000330193079B00939DF92030FDF73EFFF7
:1036C0000BB0BDE8F08300BFA0EF002078EB050849
:1036D00078E80508674706082DE9F04F024691B0E3
:1036E0000846FBF72FFF0B46044620B1104611B0E9
:1036F000BDE8F04F3EE74FF0FF32CDE908209C4A8D
:103700009C4FD2F88820DFF8B49292F83810DFF896
:1037100068A2CDE90C10CDE90E02CDE90A00964968
:1037200007AA184649F09AFAA046054626464DB91A
:10373000089A0C9EB2424FD19048FEF75BFF11B041
:10374000BDE8F08F062E12D8DFE806F0041E23280D
:10375000353C410049462846FCF77EFA78B14FF4E3
:1037600080600EF041FC90F904300893012407AA10
:103770005146002049F072FA01360546D7E728463F
:10378000FCF75EFB0890F2E72846FCF759FB09902E
:10379000EDE72846FCF777FA0A90E8E7284646F076
:1037A000D1FF394602462846FCF732FA002808BF06
:1037B0004FF00108DBE72846FCF742FB00230C90A2
:1037C0000F93D4E72846FCF73BFB0D90CFE7284644
:1037D000FCF759FA0E90CAE7694F51B23B4613F90C
:1037E000010B814208D00135092DF8D1002165482F
:1037F0000131FEF7FFFEA2E763480121FEF7FAFE62
:1038000072B2002317F9011B8A4200F009810133CB
:10381000092BF7D132460121E9E7A6F11402534200
:103820005341059308AD00235F1CEB68002B36D194
:1038300095F900B058460EF09FFBD5F804A020B1D2
:10384000D0F80090B9F1000F5DD1BAF1000F1BD193
:103850004FF461436B604FF0010AAB680BB903236F
:10386000AB600023D5F8049002932A7A1946CDE97B
:10387000009258461A460EF0A7FCE86038B9434853
:103880003946FEF7B7FE5AE74FF0000AE5E74A4629
:103890003946BAF1000F34D03D48FDF7FFFD022F45
:1038A00005F110054FF00103BED1059B0F9F0B9D45
:1038B0004BB13848FDF756FE3B681B6A1BB13649D1
:1038C0002A4638469847B8F1000F4ED03349344B5A
:1038D000142E18BF19463348FEF78CFE142E09D15A
:1038E000B8F1000F06D02B68DB691BB12E4900220E
:1038F00028469847002C63D100223946284640F0DC
:10390000AFFD2A48C9E7C5F80C90BAF1000F25D0E1
:10391000274839465246FDF7C1FD5146484603F057
:1039200065FBD5F808A0BAF1000F0FD099F8042074
:1039300092450BD01F4853463946FDF7AFFDD9F8E5
:1039400000305FFA8AF19B6948469847D9F82C30D5
:10395000002BA4D00023C9F82C30A0E7D9F8082008
:1039600015483946FDF79AFDDBE70D49B3E700BF7F
:1039700008EC002049510608054706084F51060883
:1039800018E00508935206086851060874510608A5
:103990009051060847520608ED6F0108315106089C
:1039A000CF51060870520608DBF70008B45106082C
:1039B000D051060822520608FD5106083E5106085D
:1039C00005F0ECFC052009F09BFFDFF87080DFF8C4
:1039D000709000264FF0030A99F80030B3428BD95B
:1039E00018F801BBBBF1000F15D058460AF038FBA0
:1039F000044680B1584605F025FC08B1A0F806A0A1
:103A000009210590F7F7B6FBA379059813F0010F8C
:103A100003D0F7F7D9F80136DEE7F7F7CFF8FAE782
:103A2000054832460221FEF7E5FD099B002B3FF4D5
:103A3000F4AE0023F5E600BF68510608E43C002020
:103A400068580020F0B5054687B00846FBF77AFDB8
:103A50000B46044640B100231C491A46012007B01A
:103A6000BDE8F040FEF778BA1949194F02AA184686
:103A700049F0F4F803AEB8B1032C04D12846FFF79F
:103A800079FD07B0F0BDFCF7DBF902AA46F8040B9C
:103A900039460020013449F0E1F8ECE70D483246A0
:103AA0002146FEF7A7FDECE7032CE7D1DDE903464D
:103AB000059B01931A463146E0B236F077FA019B36
:103AC0000028EBD12846FFF717FDDAE79CFB002022
:103AD00005470608E8470608F8B5064608460C46B6
:103AE000FCF7AEF920210546204649F0FBF80446D4
:103AF00018B93046BDE8F8403CE5114F114E3B780F
:103B000032789A4201D0FAF707FB0F4B20461D602E
:103B100046F018FE012201462046FAF7A5FA3B7846
:103B200032789A4201D0FAF7F7FA204646F00AFEB8
:103B30002A460146BDE8F8400448FEF75BBD00BFD9
:103B4000082B0020C44D0020042B0020A55206089D
:103B50002DE9F041064688B008460D46FCF770F99D
:103B600020210446284649F0BDF820B9304608B067
:103B7000BDE8F041FEE4FCF763F922460546014644
:103B80000F48FEF737FD85B1202D2A46694628BF2C
:103B900020222046FAF7DCFAE84606460027B7421C
:103BA00008DBAD1B3444002EEDD1FDF7C3FC08B09B
:103BB000BDE8F08118F8010BFDF7C4FE0137EEE710
:103BC000BB5206082DE9F043064687B008460C466E
:103BD00046F0B8FD082843D1671E03AD07342946D7
:103BE0003A46A84612F8010FFBF7E8FFA24201F897
:103BF000010BF7D10023DFF87C908DF8143017F813
:103C0000010FFBF7DBFFC1B205F8010B484601913C
:103C100049F068F820B10199284649F063F828B1C5
:103C20003046FFF769FC07B0BDE8F083A742E6D154
:103C30000F4940462BF070FC0D480E49082310F840
:103C4000012B11F8014B18326A44013B02F80C4C6D
:103C5000F5D109488DF8143003A9FEF7CBFCE2E753
:103C60000028E9D0304607B0BDE8F04382E400BF49
:103C700098570020707C0608D352060807B50093B9
:103C800013460A460249FFF720FC03B05DF804FB27
:103C9000DA5206082DE9F041064686B00846FBF7E1
:103CA00051FC0F46054640B100235D491A460120EC
:103CB00006B0BDE8F041FDF767BE0846FCF7C0F866
:103CC0001328044600F3A38006264643781C8DF88B
:103CD0001750FBF775FD534D074670B1FCF7B0F870
:103CE000C0B213F0E1FD40B1AB19027983F8AC2406
:103CF0009DF8173001338DF817303846FBF760FD1B
:103D0000074668B1FCF79CF80D2809D8062303FB89
:103D1000045383F8AD049DF8173001338DF8173044
:103D2000DFF8FC80B11C0DF1170241443846FCF766
:103D30008BF8FBF745FD074668B1FCF781F80128D1
:103D400009D8062303FB045383F8B0049DF8173009
:103D500001338DF817303846FBF732FD80B1FCF7A0
:103D60006FF8C0B213F0A0FD50B1062303FB04535B
:103D7000027983F8B1249DF8173001338DF817309C
:103D80009DF81720042A4FF006032FD103FB04539C
:103D90000022A3F8B0241EF059F8062303FB0455B3
:103DA0004FF4617695F8AC0413F068FD95F8AF24F4
:103DB00095F8AE741923804695F8B10413FB076794
:103DC00013FB026613F05AFD437998F8052003931C
:103DD00095F8B0340097CDE90163134895F8AD34F8
:103DE0002146FEF707FC06B0BDE8F081052A05D1A3
:103DF00003FB0453002283F8B124CCE7062A1FBF3B
:103E000008EB0602002348F806309380C3E7074911
:103E100013232A46304606B0BDE8F0412EE700BF26
:103E2000B4F0002008EC00204E470608F3520608C4
:103E30002DE9F04380468BB00846FBF783FB0F4625
:103E4000044640B100235E491A4601200BB0BDE88C
:103E5000F043FDF7A5BE0846FBF7F2FF1D28054617
:103E600000F3A5800A264643781C8DF82740FBF70F
:103E7000A7FC044630B1FBF7E3FF9DF82730013380
:103E80008DF827302046FBF79BFC4E4C074660B16F
:103E9000FBF7D6FF0D2808D80A2303FB0543187348
:103EA0009DF8273001338DF82730DFF81491711C0D
:103EB0000DF1270249443846FBF7C6FFFBF780FCAB
:103EC000074660B1FBF7BCFF222808D80A2303FB92
:103ED0000543D8739DF8273001338DF827303846D5
:103EE000FBF76EFC074660B1FBF7AAFF0D2808D868
:103EF0000A2303FB054318749DF8273001338DF81E
:103F000027309DF82730062B0CD009EB0602002342
:103F100049F80630404653601381FFF72BFB0BB086
:103F2000BDE8F0830A2606FB054600233846738267
:103F3000B382FBF745FC074638B1FBF781FF9DF8DC
:103F40002730708201338DF827303846FBF738FC74
:103F500050B1FBF775FF0A2303FB054398829DF8D8
:103F6000273001338DF82730174B4FF0FF325A605E
:103F70000A2202FB05424FF46170938A0693538A2A
:103F80000593137C0493D37B0393917B192313FB39
:103F900001010291517B13FB01030193137B0093F9
:103FA00000210A4A2B460846FDF7C8FAB7E7084938
:103FB0001D23224640460BB0BDE8F0435EE600BF3D
:103FC0000CFD002000FD002064040020844706084A
:103FD000F35206082DE9F34105460846FBF7B2FA0D
:103FE0000C46074640B1002333491A46012002B06F
:103FF000BDE8F041FDF7DABE30492046FBF7E4FDAD
:10400000034670B92C4A4FF47A704FF4FA610133C9
:10401000042B1080518002F10402F8D102B0BDE8F7
:10402000F0812046FBF70CFF0328064640D82046C7
:10403000FBF7C6FB074670B1FBF702FF4FF0010824
:1040400004463846FBF7BCFB48B9284602B0BDE839
:10405000F041FFF78FBA40F2EE248046F1E7FBF71C
:10406000EFFEB8F1000FF0D0A4F2EE2240F2DC53E4
:104070009A4203D8A0F2EE229A4209D9104940F69A
:10408000CA0340F2EE22284602B0BDE8F041F5E551
:104090000C4B0D4A03EB86030021A3F83841A3F82B
:1040A0003A01CDE9004033460846FDF747FAB5E747
:1040B000064903233A46E6E738FE00204951060840
:1040C000F952060800FD0020BB4706080753060802
:1040D000F0B5074689B00846FBF734FA0E460546A8
:1040E00040B1002319491A46012009B0BDE8F0404B
:1040F000FDF7A0BE0846FBF7A3FE3F2804461DD8E7
:104100003046FBF75DFB0146204635F08DFF78B168
:104110000E4803AE314600EB840040F04FF90C4AE4
:104120000096234629462846FDF708FA09B0F0BD57
:10413000384609B0BDE8F040FFF7DEB905493F2336
:104140002A46384609B0BDE8F04097E59CFB0020C0
:10415000CC470608F3520608F0B5074685B0084676
:10416000FBF7F0F90E46054640B100231C491A46FC
:10417000012005B0BDE8F040FDF7A6BE0846FBF7FC
:104180005FFE0F28044623DC3046FBF719FB01468F
:10419000204635F0C7FEA8B1124B04F1400203EBF4
:1041A0008203294693F8972F029293F8962F019253
:1041B000B3F8943F00930C4A23462846FDF7BEF916
:1041C00005B0F0BD384605B0BDE8F040FFF794B942
:1041D00006490F232A46384605B0BDE8F0404DE5B4
:1041E0009CFC002008EC0020D6470608F352060885
:1041F0002DE9F04F074689B00846FBF7A3F98B4637
:10420000054640B100234C491A46012009B0BDE8DB
:10421000F04FFDF74BBF494B084693F800A093F8C9
:10422000019093F8EA80FBF70BFE092804467BDC3B
:10423000062646430BF101008DF81F50FBF7C0FA2C
:104240003D4D834648B1FBF7FBFD0D289FBF9DF810
:104250001F30A85501338DF81F305846FBF7B0FAD0
:10426000834660B1FBF7ECFD824508D3062303FBD0
:10427000045358709DF81F3001338DF81F30584695
:10428000FBF79EFA824660B1FBF7DAFD484508D895
:10429000062303FB045398709DF81F3001338DF8FB
:1042A0001F305046FBF78CFA814660B1FBF7C8FD22
:1042B000804508D3062303FB0453D8709DF81F30B4
:1042C00001338DF81F30311D0DF11F02294448467E
:1042D000FBF7BAFD9DF81F30062B09D0AA19002361
:1042E000AB5138469380FFF745F909B0BDE8F08F30
:1042F0006343EA184FF461765079192111FB00608D
:104300000590107911FB00610491D17803919178A7
:10431000029152780192EB5C00930021084A2346F7
:104320000846FDF70BF9E0E7064909232A46384617
:1043300009B0BDE8F04FA1E498600020CC650020F2
:10434000FC470608F35206082DE9F7438046084665
:10435000FBF7F8F80B46054628B14046FFF70AF987
:1043600003B0BDE8F0832D49DFF8B09001AA1846EC
:1043700048F074FC2F4604462E467CB9022DECD141
:10438000A7F57A73B3F57A7F20D925494FF4FA63FC
:104390004FF47A724046FFF771FCE1E74DB1012D11
:1043A0000FD001AA4946002048F058FC01350446C8
:1043B000E3E7214640463FF0B1FF431C0646F0D1FB
:1043C000CEE72046FBF73CFD0746EAE7154B1B68A6
:1043D000B8B25B689847FF2EBCEEC00A0CD1124BF6
:1043E000F8EE407A1A78114BA24213DC10EE101A44
:1043F0000F48FEF7FFF8B3E70E4B0F48F8EE407A90
:1044000003EB860310EE102AC3ED527A3146FEF715
:10441000F1F8A5E7E3EC017A0134E5E70547060882
:10442000A4590608A86400206858002048FE00200F
:104430001C53060800FD00200F5306082DE9F34128
:1044400006460846FBF77EF80D46074670B1002485
:1044500001A9204640F050F8013401463046FFF7EC
:10446000EDFF122CF4D102B0BDE8F0810846FBF755
:10447000E7FCC4B2112C72D8681CFBF7A1F93C4DC3
:104480008046E8B93B4B03EB440393F868118A1E5E
:1044900051425141374B03EB440393F86821AA5C26
:1044A000002955D093F86931192040F2EE2100FB24
:1044B00003133148214602B0BDE8F041FEF79AB837
:1044C0000178284648F00EFC70B1032C94BF0022FE
:1044D00001222A4902EB4202431B0A4452FA83F3A7
:1044E00093F80476032F05D1304602B0BDE8F041C1
:1044F000FFF702B84046FBF763F908B3022FF3D188
:10450000FBF79EFC40F6CA0280B29042194BA8BF4E
:10451000104640F2EE22904203EB4403B8BF10462F
:10452000A0F2EE201922B0FBF2F083F86901BB1E65
:10453000594259410F4B03EB440383F86871A9E7D3
:10454000022FF4D1304602B0BDE8F041FFF712B8B7
:104550000B48214602B0BDE8F041FEF74BB80949CF
:1045600011233A46304602B0BDE8F041FFF786BB62
:104570006C7E060800FD00202B53060878E805082D
:104580003B530608075306082DE9F74FDFF89C91C7
:10459000DFF89C8105460F463846FAF7D3FF0646FA
:1045A00040B100235A491A46012003B0BDE8F04F3C
:1045B000FDF75EBB052249463846FBF729FB60B98B
:1045C000534B00221A601A611A621A631A641A6540
:1045D0001A661A6703B0BDE8F08F4E4904223846C8
:1045E000FBF716FB04463846002C44D1FBF7E8F8ED
:1045F00083460028EED046F0A5F8474BC2B253F8E8
:1046000004ABBAF1000F07D144493A46284603B03B
:10461000BDE8F04FFEF759BF51465846CDE900239B
:10462000FBF7F6FA0134DDE9002306460028E6D15F
:10463000374A0346174600210133082B42F8101B66
:10464000FAD108EBC403D3F804C0BCF1000F03D0C7
:1046500018F834E0764505DB3148324F5146FDF716
:10466000C9FF99E70CEB06130FCB07EB061484E8A0
:104670000F000136EEE7FBF7E3FB072804463DD8C1
:104680003846FBF79DF8064658B3FAF7F5FD204B80
:1046900003EB041383ED000A01273046FBF790F883
:1046A000064638B1FAF7E8FD194B03EB041383ED26
:1046B000010A01373046FBF783F8064638B1FAF7AE
:1046C000DBFD134B03EB041383ED020A0137304685
:1046D000FBF776F838B9284603B0BDE8F04FFEF78F
:1046E00049BF0746D9E7FAF7C7FD0948032F00EB92
:1046F000041484ED030A3FF454AFECE70A4907239E
:104700003246284603B0BDE8F04FFFF7B7BA00BF06
:10471000C45900204853060884EE05084D53060886
:104720005E530608CF510608F352060849510608A1
:1047300024E0050810B504460848FCF713FFFAF713
:10474000DBFC20B1BDE810400548FCF70BBF20465C
:104750000449BDE81040FEF7B8BE00BF6853060824
:10476000725306087A5306082DE9F04F8FB00446BD
:1047700002AA0846B14948F071FA064640B9034614
:104780000246AF494120FDF7F1FC0FB0BDE8F08FC4
:10479000AC49FBF719FA0746F8B9A84902AA48F04C
:1047A0005DFAFBF74DFB0828054606D9A649082304
:1047B0003A462046FFF762FAE7E7A14C23788342A6
:1047C00001DC2570E1E706463146204632F0F4FB75
:1047D00023780136B342F7DCF3E79C493046FBF718
:1047E000F3F90546D0B9954902AA48F037FAFBF724
:1047F00027FB0828064603D9954908232A46D8E707
:104800008F4C6378834201DC6670BEE728463146F0
:1048100001353FF0ABFD082DF8D1F5E78D49304665
:10482000FBF7D2F90746F0B9844902AA48F016FA14
:104830000028AAD0FBF704FB0828054603D98649BF
:1048400008233A46B5E77E4C94F8EA30834207DD08
:104850000146204632F0FAFB2946204632F004FC9D
:1048600084F8EA5091E77D493046FBF7ADF90546FB
:1048700018BB734BDFF8C49193F8EA7006AE01469B
:104880001022304648F017FAB046BD4202AA80F224
:104890000E814946002048F0E1F910B970493A46C6
:1048A0000EE1FBF7CDFA013528F8020BEDE796E8AB
:1048B0000F006C4C84E80F0067E76B493046FBF74C
:1048C00083F9054600283BD15D4B0DF1180893F89C
:1048D000EA90464607464F45584902AA4FF0000065
:1048E00080F2F28048F0BAF9014610B95F494A46B1
:1048F000E6E00322304648F02FFAB2464FF0000BB4
:10490000304645F01FFF584502D801370436E2E72C
:104910009AF80000FBF752F90BF1010B0AF8010BB2
:10492000EEE753494A46CBE041462046032232F0A7
:104930002BFB0135043408F10408AF42F4D124E71D
:104940004C493046FBF740F90546002840F0AC8062
:104950003B4F3A4997F8008002AA48F07FF90028B7
:104960003FF413AFFBF76CFA461E01D4B04503DCED
:104970004149434601221CE7304902AA002048F081
:104980006DF9014600283FF400AF4FF000080822FF
:1049900003A8CDE903888DF8148048F0DDF90DF106
:1049A0000C0903A845F0CEFE40451CD8234902AAB5
:1049B000002048F053F900283FF4E7AE90F800A03B
:1049C00097F80190DFF8C4B04FF000084D451B493F
:1049D00002AA4FF000007EDA48F040F9024658B9CA
:1049E00026494A466CE099F80000FBF7E7F808F121
:1049F000010809F8010BD4E7B5B91378303B092B4E
:104A000012D91F490192FBF7DFF8019A40B1104615
:104A10005946FBF7D9F8019A002839D019494FE0D7
:104A20004FF001084FF0FF3510460192FBF708FAEE
:104A30000028019A2EDA144942E000BF0547060813
:104A4000CC65002081530608875306089253060858
:104A50009B530608A9530608B5530608C753060812
:104A6000B6540608B8660020F1530608D654060866
:104A7000FD5306081B54060820540608F654060881
:104A80000146060833540608685406082C540608E4
:104A9000A846C7E70EAB03EB4503013523F8200C0E
:104AA00094E71B494A460BE01A49324608E01A4986
:104AB000002048F0D3F800283FF4F9AE17493A46F1
:104AC0002046FEF702FD60E648F0C8F800287FF4B3
:104AD00028AF134C31E748F0C1F80028E1D106EBCC
:104AE000C6008230082203A9384432F04DFA5046FD
:104AF000FBF764F8BC196A0084F8CA0007EB0610DB
:104B000006A9023048F074F884F8E2803DE600BF60
:104B10007D540608A054060805470608D353060826
:104B2000C86600202DE9F041144B1B6888B004468C
:104B3000F3B11A6804A9D56A18466A46A84706461A
:104B400088B1DFF8448004AC6D46002735F8022BAD
:104B500034F8021B40460137FDF74CFDBE42F5DC40
:104B600008B0BDE8F08106492046FEF7AEFCF7E745
:104B7000044908B0BDE8F041FEF7A7BC8060002002
:104B8000355506084D5506081B55060813B504464D
:104B90000846019145F0D6FD024678B10F2804D1B0
:104BA00001990A4848F0C4F840B1084B084A09493D
:104BB000204602B0BDE81040FEF787BC0349064816
:104BC00002B0BDE81040FDF715BD00BF294E060834
:104BD000545506085F5506088955060813B504465E
:104BE0000846019145F0AEFD0199024670B10428D6
:104BF00003D10A4848F09CF840B1084B084A0949DB
:104C0000204602B0BDE81040FEF75FBC03490648ED
:104C100002B0BDE81040FDF7EDBC00BF394E0608FC
:104C2000975506085F550608A75506082DE9F04375
:104C300006469BB008460C4645F084FD0027054615
:104C40001C22394602A8019748F035F82DB3402DB3
:104C500008D03A4940232A4630461BB0BDE8F0430D
:104C6000FEF733BC0DF1040804F14009022221468D
:104C7000684648F071F80023102209A968468DF8AB
:104C80000270FBF715F8099B0DF10202934221D146
:104C90000234A14508F8010BE8D100213D220AA801
:104CA000099109AC48F007F8002D3AD0244B1D7843
:104CB000C5B12449202201A847F0D3FF90B1204676
:104CC0002049FAF7DFFD204A204923463046FEF707
:104CD000FCFB04E01A781E493046FEF7F6FB1BB0D9
:104CE000BDE8F0831B4B1B78DBB9D5B9154A01AD84
:104CF0002B4603CBA342106051601D4602F108020F
:104D0000F6D1154B0F490122204683F88C21FAF782
:104D1000B9FD1248FCF72CFC11482146FDF76AFC4E
:104D2000DDE70D4B93F88C311BB9054B1B78002B3D
:104D3000F2D004492046FAF7A5FDEDE7BA5506087A
:104D4000B23A0020B43A0020F85506085F5506082C
:104D5000DC55060808EC002000FD0020025606087D
:104D6000115606082DE9F74F834608460D4645F0D3
:104D7000E9FC3A4F0446D7F80090B8B93848394DA5
:104D8000394FFCF7B7FB012655F8041B49B106FA69
:104D900004F313EA090F02D03846FCF77FFB013415
:104DA000F2E703B0BDE8F04FFCF7C4BB02462F4961
:104DB0002846FAF72DFF78B92D482A4C2D4DFCF7DF
:104DC00099FB54F8041B0029EBD00B78002BF8D08A
:104DD0002846FCF763FBF4E72B782D2B214B03BF10
:104DE000013504F1FF344FF0010A4FF0000A0026AC
:104DF00053F8048BB8F1000F07D11F492A465846D3
:104E000003B0BDE8F04FFEF760BB2246414628469E
:104E10000193FAF7FDFE019BF0B90123B3409A0517
:104E200005D5164803B0BDE8F04FFCF79BBBBAF1BF
:104E3000000F0CD029EA030311483B60FCF75AFB32
:104E40000C48414603B0BDE8F04FFDF7D3BB49EA3B
:104E500003030C483B60F1E70136C9E7A464002076
:104E60001E560608F0EE0508285606080C4D0608E2
:104E70002C560608834C06084D530608375606087C
:104E8000435606084C5606082DE9F74F814608465A
:104E90000E461746984645F055FC0446E8B940488A
:104EA000404DFCF7FBFA20460DF002F83B68184233
:104EB00006D020460DF00EF801462846FCF7EEFA23
:104EC0000134182CEFD13B6813B93748FCF712FBBB
:104ED00003B0BDE8F04FFCF72DBB02463349304626
:104EE000FAF796FE0546A8B93148FCF703FB2C46B5
:104EF000304D20460CF0DCFF10EA080F06D02046AB
:104F00000CF0E8FF01462846FCF7C8FA0134192CDA
:104F1000EFD1DDE733782D2B48F0807303BF0136E6
:104F200004F1FF34012500254FF0000A019350469B
:104F30000CF0D0FF2246834601463046FAF768FE61
:104F400000BB50460CF0B4FF019B03421AD08DB158
:104F5000BAF1180F1CBF3B6840EA03081648C7F8AF
:104F60000080FCF7C7FA1348594603B0BDE8F04F7C
:104F7000FDF740BBBAF1180F1CBF3D6885433D608B
:104F80000E48EEE70AF1010ABAF1190FCFD10C4928
:104F90003246484603B0BDE8F04FFEF796BA00BF70
:104FA00054560608824C06085E5606080C4D060844
:104FB0002C560608834C0608435606084C5606082D
:104FC0004D530608014A40F202235DE7F05F0020DE
:104FD000014A6FF07F4357E7E85F002010B50446B1
:104FE0002AF00EFB28B920460449BDE81040FEF720
:104FF0006CBABDE810400248FDF7FCBA65560608D9
:105000007456060810B5044608460B46FAF79AFA95
:1050100028B9094903221846FAF7FAFD28B90748C2
:10502000FCF7A6FA0120FCF76DFA20460449BDE81A
:105030001040FEF74ABA00BF7F560608835606089E
:10504000A55606082DE9F04F074691B08248834DDA
:105050000E46FDF7CFFA8249C5F890D1002385F8B6
:1050600094310622012309783046402485F8954181
:1050700008F0F0FB0A2008F043FC95F894310C2B63
:10508000DAB240F2E4809DF80C50FE2D36D0FF2DB0
:105090000BBF15240F2401260026944240F0D78030
:1050A000611EC9B2684639F029F804F140030DEBDE
:1050B000030414F8413C834240F0C48006F1FF38F9
:1050C0009DF80D3067485FFA88F8B8F1010F8DBF81
:1050D00003F01F079DF80E709DF80F4061378CBFDD
:1050E0005C091D46FCF706FA022E64D0013C042C34
:1050F0005FD8DFE804F005585A5E5C000226CCE772
:105100005948DFF8C091DFF8C0B1FCF72BFA5748D7
:10511000FCF7F0F96C464FF0000A14F8011B484602
:105120000AF1010AFCF7BAF9BAF10C0F49D1FCF700
:1051300001FA022E4FD06422B5FBF2F102FB1152AC
:105140004B483B46D2B2C9B2FDF754FAB8F1010F51
:1051500071D8484A484B9DF810104848484D0029DE
:1051600014BF11461946FDF745FA9DF81110454B3D
:105170004548002914BF19462946FDF73BFA022E7F
:1051800059D19DF812404148FCF7B4F94CB3FF2CBB
:1051900037D00A22B4FBF2F102FB11423C48D2B2F2
:1051A000FDF728FA20E03B48ABE73B48A9E73B483E
:1051B000A7E73B48A5E700238DF83F300DF11F001E
:1051C0009FE7384B03FB0AF2B2F1553FA5D858468A
:1051D000FCF790F9A1E734483A462946FDF70AFA68
:1051E000B7E72846FCF7BEF99DF813402F48FCF7B7
:1051F00081F944B1FF2C21D02D482146FDF7FAF961
:1052000004E02C48EEE71E48FCF7ACF91C4E294F91
:10521000DFF870800DF11305002415F8013F7BB114
:10522000FF2B0CBF3A464246214623480134FDF786
:10523000E1F9042CF1D111B0BDE8F08F1D48E3E78E
:105240003246F1E71D493846FEF73FF9F3E71C48BF
:10525000FCF788F9EFE700BFD456060800FD0020F0
:1052600068580020E5560608F05606081657060846
:1052700028570608B4560608BD5606085F570608A4
:10528000C4560608775E0608765706087D57060856
:1052900091570608F7560608FF56060807570608EE
:1052A000434A0608ABAAAAAA445706089957060813
:1052B000F6480608C8560608A9570608B45706084F
:1052C000C457060817460608D0B506082DE9F74F5B
:1052D00005460846FAF736F90B46044618B9324A2D
:1052E00092F896712FB9284603B0BDE8F04FFEF74B
:1052F00003B92E49DFF8C080DFF8C090DFF8C0A006
:1053000001AA184647F0AAFC264610B904F054F842
:1053100007E04EB9014628463FF000F8421C04461B
:105320001AD103B0BDE8F08FFAF78AFD2F28834623
:1053300034D80FB104F032F8BBF1060F13D01C497A
:10534000012309785FFA8BF2E0B208F083FA59463C
:105350004846FDF74FF90027144901AA00200136FD
:1053600047F07CFCD1E7DAF800301B0112D5FF2CA6
:105370000ED0E1B22846FFF765FEE8E72846FFF7C2
:1053800061FE01370A4B1A78F9B28A42F6D8DEE795
:105390000027F7E70748FCF7E5F8D8E72F22414652
:1053A0002846FEF792F8D7E700FD002005470608DB
:1053B0006858002065560608DE570608CD570608CF
:1053C000945700202DE9F84FDFF8A880DFF8889087
:1053D000DFF8A4A007460C46204645F0B3F9064680
:1053E00058B91D4B1D481A781D4B03EB8203D3F8A7
:1053F0000816BDE8F84FFDF7FDB8024641462046C5
:10540000FAF706FC60B1DFF864B000255BF8041B16
:10541000B1B9224638461349BDE8F84FFEF755B8F2
:105420001148124C124DFCF765F854F8041B19B1E1
:105430002846FCF733F8F8E7BDE8F84FFCF77AB8F0
:1054400032462046FAF7E4FB01350028DED189F820
:1054500000505446C0E700BF61580020FE570608C0
:1054600078E805084D5306082C56060884EE050812
:10547000834C06080C4D0608CF510608F8B50746C0
:105480000846FAF75FF8D0B1204BD3F894600136A4
:1054900030460CF01FFD34460546F0B90134192C96
:1054A000A8BF002420460CF015FD0546A8B9B4425B
:1054B000F4D138461649BDE8F840FEF706B808466C
:1054C000FAF7BEFC04460CF005FD054628B9214656
:1054D0001048BDE8F840FDF78DB80C4BC3F8944078
:1054E0000CF014FF0C4821462A46FDF783F8182CCF
:1054F0009DBF0A480C2101FB04000020BDE8F840D4
:1055000098BF90F8F4060CF035BF00BF640400208B
:10551000085806081C5806083258060878E8050896
:1055200038B5124D04460846FAF70CF860B1104B36
:10553000104893F900104B1C0ABF0F4BC9B21978E1
:10554000BDE83840FDF756B80846FAF779FC03285D
:1055500004D8C0B2FBF722FC2946E4E720460749FD
:10556000BDE838400322FDF7B0BF00BFCF510608A9
:10557000640400204B580608805700205B5806083A
:10558000F0B5032985B005460C46164614D80B4FD6
:105590003970FBF7CFFF0A492846FFF7C1FF0949D9
:1055A000224601A8F9F7E2FA01AB32460821284663
:1055B000FDF706FFFF233B7005B0F0BD640400203B
:1055C000CF5106084B58060838B5124D0446084618
:1055D000F9F7B8FF60B1104B104893F901104B1C5C
:1055E0000ABF0F4BC9B25978BDE83840FDF702B881
:1055F0000846FAF725FC032804D8C0B213F0DCFCF7
:105600002946E4E720460749BDE838400322FDF774
:105610005CBF00BFCF51060864040020475806084D
:105620008057002056580608F0B5032985B0054676
:105630000C46164614D80B4F7970FBF77BFF0A49CE
:105640002846FFF7C1FF094922466846F9F78EFA56
:105650006B46324610212846FDF7B2FEFF237B70D1
:1056600005B0F0BD64040020CF5106084758060875
:1056700038B50D460446174905222846FAF7C8FAF8
:1056800050B9154B1A7A12B9012119725A72BDE834
:1056900038401248FBF766BF114903222846FAF743
:1056A000B7FA80B90C4D2B7A4BB16B7A3BB10D49EF
:1056B0002046FDF70AFF00232B726B7238BD0A48A3
:1056C000FBF750FFF7E720460849BDE83840FDF7F3
:1056D000FCBE00BFD55D060808EC00207658060821
:1056E000205F06088C580608C3580608A556060809
:1056F000F8B5174C237A054663B1637A53B115495F
:10570000FDF7E3FE28461449FDF7DFFE0020207276
:105710006072F8BD114B93F88C51BDB1104B1878E5
:105720000028F6D10F4B104A03F1200716461868DF
:105730005968144603C40833BB422246F7D10123FB
:1057400086F83B3008F0F2FD2846E2E70120E0E76A
:1057500008EC00208C580608D758060800FD0020E9
:10576000B23A0020B43A0020D867002008B5FFF70D
:10577000BFFF50B1054B01229A73FBF7CFFC0448E1
:10578000FBF7F6FE0020FBF7BDFE08BD80570020AA
:10579000F55806082DE9F74F064601AA08462E4996
:1057A000DFF8C480DFF8C490DFF8ACA047F056FA09
:1057B0004FF0000B04465D4601270CBBBBF1000F08
:1057C00026D1264C002D42D025482946FCF712FF51
:1057D00023780BB9F9F7BEFEF8F792FD0023637248
:1057E000FBF726FE15B12846F9F755FE9FB1304666
:1057F000FFF77EFF78B1FBF791FC0020FBF782FEFC
:10580000BBF1000F0AD02046FAF71AFB85B2C5B9E2
:105810003046FDF771FE03B0BDE8F08F41462046EB
:10582000FAF71AFA80B949462046FAF715FA00281D
:10583000EED05F4601AA5146002047F00FFA044619
:10584000BBE74FF0000BF5E74FF0010BF2E705481F
:10585000FBF78EFEC0E700BF0547060808EC0020F6
:105860000559060828590608FC5806080C5E060863
:105870002DE9F74F444BDFF82CA11A785B788AF8B2
:105880000130424B8AF800201B78054688460BB948
:10589000F9F760FEF8F734FD00263D4CB1460D23C4
:1058A0003B4A7343414652F803B05846FAF7D4F9DD
:1058B000002841D0B9F1000F01D0FBF73BFE35487D
:1058C0005946FBF7EBFD002221462846FDF7EEFD89
:1058D000FBF730FE237903F01803082B46D0102B7A
:1058E00049D02046FCF795FE294A0D2303FB0623E9
:1058F000B3F80900F8F7CCFC0746D8B12046F9F711
:10590000EBFDD7E902210090024401442046F9F75B
:105910007BFD78B9019059461F48FBF7BFFD019AFE
:10592000B9681346009A28460A442146FDF756FCFA
:10593000FBF700FE09F10109013640F24B239E42BC
:1059400004F10D04ABD10020F9F7A5FDFF238AF87F
:1059500000308AF80130B9F1000F11D10F494246E9
:10596000284603B0BDE8F04FFDF7AFBD0C4928460F
:10597000FFF7D6FDB5E70A492846FFF725FEB0E751
:1059800003B0BDE8F08F00BF8057002008EC002076
:10599000C4F90508C05006083E5906084D530608CC
:1059A000CF510608640400202DE9F74F074608464A
:1059B0000E4644F0C7FE044620B1012826D13278B5
:1059C0002A2A23D1B348B44EDFF8E892FBF7CAFD88
:1059D0000025B2464FF00D0B40F24B280BFB05F3B0
:1059E00048465AF80310FBF759FD221E18BF012242
:1059F000314638460135FDF759FDFBF79BFD45451E
:105A000006F10D06EAD103B0BDE8F08F3D21304626
:105A100047F068F9002800F0378101460A4611F87E
:105A2000014D202CFAD0921B0130814610F8011B49
:105A30002029FAD0DFF860B25FFA82FA4FF000084E
:105A40000D2303FB08F10BEB010452465BF8011038
:105A500000913046FAF7DCF80546002857D1009946
:105A6000084644F06FFE824551D1267906F0E001E8
:105A7000402900F0CC800ED8002956D0202900F013
:105A80009E8038468549FDF720FD204603B0BDE8DD
:105A9000F04FFCF7BEBD602900F092808029F0D164
:105AA000484644F04FFEE379A679DB0705460CD55E
:105AB0002046F9F72DFE0378014633B12A464846C1
:105AC00047F036F9002840F0D980002D00F0D6804C
:105AD000AE42C0F0D3800D2303FB08B3204693F8F9
:105AE00005A0F9F715FE3246002147F0E4F8AA4573
:105AF0002CD86B492A46484647F01AF930B320465D
:105B0000F9F706FE2A46494647F072F81EE008F10A
:105B1000010840F24B23984592D1624932463846FB
:105B200003B0BDE8F04FFDF7D0BC06F00703042B2F
:105B30001CD10B460A224846FAF7BAF8D4F80530C9
:105B4000834201469DD32046F9F7F6FD0D2303FB62
:105B500008F855485BF80810FBF7A0FC0022214626
:105B6000384603B0BDE8F04FFDF7A0BC052B0FD1C0
:105B700001230A224846FAF79BF8D4F805308342FD
:105B80000146FFF67EAF5B4283423FF77AAFDAE72A
:105B90004846FAF755F9B4F80550B4F8071016F06E
:105BA000050FAAB218BF2AB28BB218BF0BB290422F
:105BB000FFF667AF98423FF764AF0146C3E76579E8
:105BC0003A4A02EBC505002695F844230092B246F6
:105BD0003346009AB24202D9BAF1000F03D0002B2B
:105BE0003FF44FAFB2E7D5F8401351F8260060B14B
:105BF00049460193F9F7E8FF019B30B93146204649
:105C00004FF0010AF9F798FD53460136E1E7637951
:105C1000009306F00706013E009BAB4296DD484626
:105C2000814610F8013B202BFAD02046F9F770FD91
:105C30008246042E04D8DFE806F0031010161F0079
:105C40004846FAF7FDF80AF8050048462C2147F0C7
:105C500049F8013500F10109DEE74846FAF7F0F8A6
:105C60002AF81500F1E700230A2200214846FAF736
:105C70001FF84AF82500E8E70123F5E70C4932460A
:105C80003846FDF722FCFCE63146384603B0BDE855
:105C9000F04FEDE54E590608C4F905089C59060871
:105CA000D0B506084D5306089159060878E805084E
:105CB00061590608C05006082DE9F04F80468BB0A8
:105CC00008460D4644F03EFD024698B3A6492846D4
:105CD000F9F79EFF044668BBFBF72CFCA348A44DD4
:105CE000A44FA54EDFF8D882FBF73CFC14203EF011
:105CF00051FB0721B4FBF1F1C1EBC102A21A013241
:105D000001313846FBF7CAFB2B7E6A7E06EB830324
:105D1000D3F8B01052B19948FCF76CFC01340E2C4A
:105D200005F12405E5D10BB0BDE8F08F4046FCF746
:105D300061FCF3E72846924905AA46F08FFF054625
:105D400020B901464120FBF72AFCECE78D49F9F721
:105D50003BFF20B98C494046FDF7B7FBE3E78B4E8C
:105D60000827002431682846F9F72EFF002808BFCD
:105D70003446013F06F11006F4D154B9844928464F
:105D8000F9F722FF28B183492A464046FDF79DFBDB
:105D9000C9E700207A498DF8130005AA46F05EFF96
:105DA0000546002C3AD080B1FAF74AF8461E09D4CD
:105DB000A37A9E4206DAE2684AB1012303FA00F0B0
:105DC000104204D174492A46DFE7744DFAE7E088AF
:105DD000F8F75EFA7249D0E902320978002908BF63
:105DE0001A46217A637A06FB0133002712F903A0D1
:105DF000039702EB030B624905AA002046F02EFF31
:105E00008146A0BB6749012344B39BF9002020468B
:105E1000CDE900313146F9F791FD84E768B10DF124
:105E20001301F9F7E6FF28B19DF81360304603F03F
:105E300009FA20B95C492A46A7E7584DFAE73046E7
:105E4000F5F7B4F88246304608F0CCF803903046B7
:105E500008F006F9A34607462646CCE7CDE900310F
:105E60009DF8130052463946F9F7B4FD5BE7454902
:105E7000F9F7AAFE054670BBACB14C4FF6B22079DB
:105E80006AB23146F5F75CF800283FF44CAF02885F
:105E9000037800932946C2F303233846120BFCF71C
:105EA000A9FB0135EBE7414C386879790E2D6AB2D0
:105EB0003FF439AFF5F796F800283FF434AF028885
:105EC000037800932946C2F303232046120BFCF704
:105ED00091FB0135E8E736494846F9F775FE002899
:105EE0003ED04846F9F7ACFF054642B26CB1207986
:105EF000F1B2F5F725F8D8B9CDF8009022682D4910
:105F0000731C4046FDF7E1FA0DE7EBB20D2B386844
:105F1000797909D99DF813302749CDF800901A09ED
:105F2000403203F00F03ECE7F5F75CF80028F1D0FE
:105F300006AF39462846F9F7B9FC08A95046F9F7E3
:105F4000B5FC55454AD06DB2002C3BD08BF80050C3
:105F500000972168194808AB721CFCF74BFBE2E67E
:105F60004FF0FF35E4E700BFAA590608AF5906080D
:105F70001C010020C559060878E805083A5B0608A8
:105F8000054706080C4D0608D7590608700400207E
:105F9000EB590608EF590608FE590608CF510608C6
:105FA00008EC00203D1501080E5A0608205A060884
:105FB00060560608425A0608655A06088D5A0608B1
:105FC000834C06089DF81320039B0D489D70110912
:105FD000009708AB02F00F024031BEE734B12168F0
:105FE000084808AB721CFCF705FB9CE69DF81320E3
:105FF0000548110908AB02F00F024031F3E700BF7A
:10600000B05A0608D85A0608F35A06082DE9F04F88
:1060100080468BB008460D4644F094FB024630B9EA
:10602000014601200BB0BDE8F04FFBF7C1BB029069
:10603000AD492846F9F7ECFD029A30B9AB49404624
:106040000BB0BDE8F04FFDF740BAA9492846F9F773
:10605000DFFD0446002857D1FBF76CFAA548A64F90
:10606000DFF8D4B2DFF8D482FBF77CFA17203EF0D9
:1060700091F917F9016B002E38D031465846DFF8F8
:106080009492DFF884A2FBF709FA01250023A9B254
:106090003046039308F01CF8029008F0A7F8027845
:1060A000039BCAB11BB90390FBF744FA0398029B08
:1060B00041789A79037802F0020208EB8303C1B1B8
:1060C0000091D3F8B0308D48002A14BF4A4652469A
:1060D0002946FCF78FFA01230135052DD7D113B9D5
:1060E0008748FBF73FFA01340D2CC2D10BB0BDE855
:1060F000F08FD3F8B0308348002A14BF4A46524686
:106100002946FCF777FAE6E700247F498DF813402B
:1061100005AA284646F0A2FD18B94046FDF7ECF95D
:10612000E4E70DF11301F9F764FE05460028F4D009
:106130009DF81360304603F085F820B97349404656
:10614000FDF7C3F9D2E7DFF8F89123464FF0FF34AB
:1061500003EB430212F8092096420BD0611C02D1D6
:10616000002A08BF1C460133152BF1D1631C15D141
:106170006749E4E71C46644905AA002046F06EFD25
:106180000646002800F09C805749F9F71DFD18BB12
:10619000604E614FDFF8AC81044613E00025EAE76A
:1061A000E97928680291F4F76FFF0246A8796B79C4
:1061B000029910F0020F14BF304638460090404656
:1061C000FCF718FA01349DF81300214607F01EFF72
:1061D00005460028E4D189E7504902223046F9F704
:1061E00017FD0746002849D1B01CF9F729FE9DF894
:1061F00013B00346BA46013739465846029307F0B2
:1062000005FF029B38B94FEA1B12454900960BF077
:106210000F0340323FE0C2799A42EBD1002D40D1CA
:106220004FF0FF36BAF1FF3F9DF8135008BF00252D
:1062300004EB440409EB04030AF101025A7009F863
:106240000450FF2208AC9A709DF813002246514674
:10625000F9F706FC06AA31469DF81300F9F700FC91
:106260009DF81320B2454FEA121120D12D4806ABFC
:1062700002F00F024031FCF7BDF937E72A493046FA
:10628000F9F7A2FC50B39DF81330284900961A097B
:10629000403203F00F034046FDF717F926E74FF0B1
:1062A000FF3A04EB44034B445E78013EBAE72048D2
:1062B000009406AB02F00F024031FCF79BF915E7A2
:1062C00004EB44041B4B0093A144024699F80110CF
:1062D0009DF813000123F9F7DBFB07E7002DDED162
:1062E0004FF0FF36B246A3E70C4D0608D759060813
:1062F000AA5906080F5B0608DC4506082F5B06084E
:10630000505B0608415B060805470608565B060811
:106310006D5B060848490608CF510608965B0608DB
:10632000035C0608BF5B060860560608995B060812
:10633000DD5B06083D150108285B060878E80508BE
:106340005C3C0020815B06082DE9F04F2DED028BAF
:1063500085B0064603AA0846924946F07FFC0746E8
:1063600040B901464120FCF7B9F805B0BDEC028BFD
:10637000BDE8F08F8C49DFF86482F9F725FC04460C
:1063800000283CD189488A4D8A4FDFF85492FBF7A8
:10639000E9F814203DF0FEFF2968AB79AA8801F1E5
:1063A0003F4108EB830301F57E01B2FA82F2890ACC
:1063B0004131D3F8B030C2F11F023846FBF76EF816
:1063C000E97911B14846FBF769F80134FBF7B2F8F7
:1063D000502C05F10805DFD1724903AA002046F0D0
:1063E0003DFC7549F9F7F0FB0028BED130466E49F7
:1063F000FFF70CFE6C493046FFF75EFCB5E7002561
:1064000008F5087919F8353008EB8303D3F8B01094
:106410000191084644F096F9019902463846F9F789
:10642000F7FB40B101351C2DECD164493A463046AA
:10643000FDF74BF899E75B4903AA46F00FFC08EB20
:10644000C5080746F9F7FCFC98F8263204464FEADF
:10645000C50A2BBB002825DC3B78002B00F09E8072
:10646000D144B9F80200F7F713FFE3B2019399F8AA
:10647000058099F80430019A846802FB038804EBD4
:1064800008013846F9F7B5FC002800F0878014F8B9
:1064900008A0BAF1000F1CD14948FBF763F864E784
:1064A000002805DD012B1A4638BF0122A24208DA76
:1064B000012B444938BF012301223046FDF7DEFBA2
:1064C00053E7384903AA002046F0C8FB013C0746C1
:1064D000C2E7504602F0B6FE814600285ED04FEA81
:1064E0001A13403308EE103A0AF00F03DFF8F48075
:1064F00008EE903A00270026B8F80200F7F7C8FE29
:1065000098F8042098F8053006FB02338268D15CC5
:10651000514523D1BD4204D101998E421ED00021A4
:10652000D15418EE902A18EE101A27485FFA86FB0D
:10653000FCB2FAF7B3FF59462046FAF7BCFFBD425A
:1065400009D12248FAF7AAFF20465946FAF7B3FFC5
:106550001F48FAF7A3FF1F48FBF704F898F8063026
:10656000012B06F1010638BF01239E42C4DB01372F
:106570001C2F08F10808BED1D9F80010B9F8042082
:10658000154801F13F4101F57E01B2FA82F2890A14
:10659000C2F11F024131FCF72DF8E6E63046FCF768
:1065A000ABFFE2E605470608AA5906082F5C060875
:1065B000183800206D5C0608785C06087C5C0608CC
:1065C000985C0608F3520608AA5C060845470608C8
:1065D000CE5C06084CB50608D85C060878E80508C5
:1065E000F548060898EA050838B51A4B5B79012B7F
:1065F00005462AD1184B1B683BB30846F8F7A2FFA3
:1066000070B90846F9F71CFC00F54373B3F5C36F86
:10661000044608D928461149BDE83840FCF755BF63
:106620000F4BB3F998410F48FAF7A2FF0E48FAF75B
:1066300061FFFAF717FF0D4BD3F888000BF01EFE31
:1066400007F040F92046F7F7F9FBBDE83840084865
:10665000FAF78EBF983A00200C2B0020F45C060855
:1066600000FD00200C5D0608F646060808EC002038
:106670002C5D06082DE9F84F1F4DDFF88490DFF8F8
:1066800084A006460C4637274FF000082046F8F74E
:1066900059FFD5F800B048B921465846F9F7DCFA59
:1066A00020B968682146F9F7D7FA80B15846FAF759
:1066B00021FF696811B15046FAF7F0FEA96811B1DF
:1066C0004846FAF7EBFEFAF735FF4FF00108013FB5
:1066D00005F11005DAD12046F8F734FF48B9B8F1D2
:1066E000000F06D1224630460449BDE8F84FFCF7BA
:1066F000ECBEBDE8F88F00BF98F00508655D0608A0
:106700005F5D0608595D060837B5044608460191E5
:1067100044F018F80199054602462046F9F778FA40
:1067200070B9625D1046F9F739FA00B932B901352E
:106730002C44204601340378202BFAD003B030BD1E
:106740000020FBE72DE9F04F0C4695B03449054693
:1067500020461746FFF7D8FF064600284FD131499B
:106760002046FFF7D1FF064600284AD12E49204691
:10677000FFF7CAFF0646002845D12C492046FFF7FF
:10678000C3FF0646002840D120462949FFF7BCFF39
:106790000028064612BF0824264601240FB144F003
:1067A000100424493046FFF7AFFF80B344F02004C3
:1067B000214B1B780BB9F8F7CDFEF7F7A1FD14F0CC
:1067C000090F00F01C831D48FAF7D2FE0020FCF7E9
:1067D00033FB14F4807307933CD11948FAF7C8FED1
:1067E0001848FAF7BFFE04F01803182B05D1164815
:1067F000FAF7BEFE1548FAF7B5FE01232BE0012497
:10680000CCE70224CAE70424C8E78124C6E710497C
:106810003046FFF779FF0028CAD044F48074C7E7F8
:106820008C5D0608935D06089B5D0608A15D060861
:10683000785C06081F59060808EC0020AF5D0608C2
:10684000B75D0608CF5D0608DB5D0608035E060837
:10685000AA5D060800230693FAF76CFE04F0100305
:10686000BB49BC480593FBF7C5FEBB49BB48FBF7DA
:10687000C1FE04F48473082B07D1B9492846FBF7FD
:106880008FFFB7492846FEF7D1F914F0800309932A
:106890000ED1B44B93F89C21002AB34A03F5CE7372
:1068A00006BF012113460021B04A2046FAF746FEF2
:1068B000AF492046FBF712FEAE492046FAF778FFB3
:1068C000AD492046FAF76BFEAC4BD3F800B0AC4BA9
:1068D0001B680493059B002B40F0D381A948FAF76D
:1068E00047FE059EA84B08939946049BDFF840A3FA
:1068F0006BEA03034FF000080A9359F8047B002F5A
:1069000040F0C181049BDFF82C9363EA0B0A089BDB
:1069100053F8042B03920893002A40F0DE819B4B2E
:106920009B4A9C492046FBF7B3F8099B002B40F09B
:106930007882DFF80493DFF804A399F800209AF82E
:106940000030954E9A4214BF01210021934A2046FF
:106950000CBF4FF001084FF00008FAF715FE9AF847
:1069600000308F4A06EB83030746D3F808364146CA
:106970002046FAF7F1FF99F80030894A06EB8306C2
:106980004146D6F80836874E2046FAF7D7FDD6EDB1
:10699000007A854AF5EE407AF1EE10FA0CBF01213B
:1069A00000212046FAF7CAFD3B4632467F49804F18
:1069B000804E2046FBF75CF97F4B01936FF07F42DE
:1069C00000923A6831682046FBF732FD7B4B019319
:1069D00040F202220092BA68B1682046FBF728FD17
:1069E000059B002B40F0A8817548FAF7C1FD059A78
:1069F00074487549DFF848C20826012710F8013BA2
:106A000011F8018B03F1500EEE440EF8208C1CF8A7
:106A100001EB0EF15009E94409F8108C2FB1A3EBFA
:106A20000E0EDEF1000747EB0E07013EE6D187F0C0
:106A3000010120468DF83860FAF7A6FD634A8DF80B
:106A4000486010AB39462046FAF786FF5F4A0CAB28
:106A500039462046FAF772FD5D4B5E4A5E49204694
:106A6000FBF7E8F95D4B5E4A5E492046FBF72CFADE
:106A70005D4B584A58492046FBF76EFA5B4B5C4A1F
:106A80005C492046FAF780FF5B4A5C4B02F20C41FE
:106A90002046FBF785F85A4A5A4B02F20C41204631
:106AA000FBF784F9584B594A59492046FBF75EFBDE
:106AB000584B594A59492046FBF7F8FA059B002BD9
:106AC00040F03C815648FAF753FD564F4FF0000B0B
:106AD000A7F57B7841460222384646F0C2F80028E6
:106AE00014BF01210021039A97F800A020460CBF93
:106AF0004FF001094FF00009FAF746FDBAF1020F15
:106B0000039040F01E8198F801204FF0190A40F2DE
:106B1000EE231AFB0232019298F80020424B9A5C55
:106B200000925B46414A49462046FAF715FF7A78BB
:106B30003D4B40F2EE211AFB021201923A789A5C28
:106B400000925B46394A49462046FAF7F7FC79E05D
:106B5000294E060889550608394E0608A755060825
:106B6000CF51060800FD0020D0B50608135E0608C8
:106B7000205E06082A5E0608214B0608C46900202C
:106B8000A4640020795D0608F0EE0508475E06085B
:106B9000A0EF0020C0FE002078E805084E5E060841
:106BA000545E0608C45900205D5E0608186800207F
:106BB000E85F00204C6A00206C5E0608735E0608E1
:106BC000815D0608006B0020707C0608D352060821
:106BD000505606089CFB002030FF00207F5E060810
:106BE0009CFC0020300001207A5E0608855E0608C5
:106BF000B4F00020A00001200CFD0020895E0608F2
:106C000038FE0020925E06089A5E0608CC650020D9
:106C1000B0640020A35E060898600020DC680020B5
:106C2000855D0608540201206C7E06082B53060879
:106C3000305E06083C5E0608CC6A002061580020E1
:106C4000985700200BF1010BBBF1120F07F102075F
:106C500008F102087FF43EAF754B2246002128461A
:106C6000FCF7AEFB230700F18280724E224631789A
:106C70002846FEF785FC717822462846FEF7D4FCAC
:106C8000B3E06D4E2EE63B7823B30A9A012303FA54
:106C900008F31A400CBF012100210392204632461E
:106CA0000B93FAF771FC049B63EA0B020B9B1A42ED
:106CB00014BF012100213B46524606462046FAF702
:106CC0004BFE039900393B46524618BF012120462E
:106CD000FAF734FC08F101080FE6039B1B784BB36D
:106CE000049B4FF0010808FA07F813EA080F0BD0CD
:106CF0006BEA030313EA080F4A46039B14BF012102
:106D000000212046FAF728FE1BEA080F12D01AEAE3
:106D1000080832460CBF012100212046FAF734FC56
:106D2000B8F100010646039B4A4618BF01212046E0
:106D3000FAF704FC0137EAE5404A59E6404B039371
:106D4000C3E698F800203F4B9A5C00925B464946A8
:106D50003D4A2046FAF700FE3A783A4B9A5C009298
:106D60005B46394A49462046FAF7E8FB6AE70027BE
:106D7000F9B2224628460137FEF702FC042FF7D16C
:106D8000DFF8B080314F98F800303B70079B33B983
:106D90002F48FAF7EDFB2F492846FEF7C1FBFF23EA
:106DA0003B70F1B2224628460136FEF73DFC042E28
:106DB000F7D198F801307B70079BA3B92648FAF702
:106DC000D7FB24492846FEF7FFFB2448FAF7D0FBFF
:106DD0002348FAF78FFBFF237B70002015B0BDE836
:106DE000F04FF8F758BBFF237B70069B002BF4D0C5
:106DF0001C48FAF7BDFB1C48FAF7B4FBEDE7A10706
:106E000006D50C4B224619782846FEF7B9FBE4E775
:106E10006207E2D5074B224659782846FEF704FC64
:106E2000DBE7034B224618212846FCF7C9FADCE7CA
:106E30008C5D0608446B0020795D0608815D0608BC
:106E4000855D06086C7E06083B5306086404002036
:106E5000A75E0608CF510608CA5E0608F15E06085E
:106E60000E5E0608045F06081A5F0608002269E441
:106E7000012267E4224BB0F5FA6F1A680346A8BFF7
:106E80004FF4FA63B3F57A7FB8BF4FF47A73D20444
:106E900016D540F2DC52904215D007EE903A40F2FF
:106EA000DB529042F8EE677A1FD8DFED166A9FED4D
:106EB000167A9FED160A77EEE67AA7EE870A7047F4
:106EC000B0F57A7F02D89FED120A704707EE903A2C
:106ED000DFED106A9FED107A9FED100AF8EE677AE9
:106EE00077EEE67AA7EE870A7047DFED0D6A9FED31
:106EF0000D7A9FED0D0A77EEE67AA7EE870A7047C6
:106F00009457002000007A44D62000C000E082445C
:106F10000000000000407A4466100040000040423B
:106F200000A0BB44D62000400000834410B5844636
:106F30004FEA810E102312F4004F14BF0E240724D1
:106F40005200013BCCF8004092B2F444F3D100EB84
:106F500081128C01035142F82130122010BD00BF74
:106F600010B584464FEA810E0424130B03EB430350
:106F700018331201013CCCF8003092B2F444F4D141
:106F800000EB01130A01845043F82140062010BD94
:106F9000704700BF704700BF034B00EB400003EB9E
:106FA000C000407C704700BFC81D0020002318228D
:106FB000027043708370C370704700BF704700BF9A
:106FC000704700BF0020704701207047704700BF26
:106FD000704700BF704700BF704700BF9FED010AB8
:106FE000704700BF000000000020704703681B6965
:106FF000184730B5084B002293F900405D7801191D
:107000000132CD729D780555082ADC788C7503F124
:107010000403F1D130BD00BF94170608C36B33B130
:107020005B68C26D9BB29A4205D3D01A7047D0E913
:1070300007239A42F9D2C0681044C01A704700BFB3
:10704000D0E909120369914238BFC9188A1A016C44
:1070500039B14968013B12FA81F2934204D9981A76
:107060007047013B981A704700207047036C13B1BA
:1070700090F86C007047D0E90903181AB0FA80F054
:1070800040097047C26B10B4034662B1C26DC1685B
:107090005C69881A013A205C5DF8044B08BF0A4617
:1070A000C0B2DA657047006A5C69411C205CDC682C
:1070B000A14238BF0A46C0B25DF8044B1A6270475D
:1070C000036F70B504460D460BB19847B8B1636ABB
:1070D000A269D554636A2169226C01338B4228BFAF
:1070E0000023636232B3EFF31183502282F31288DC
:1070F000266C3268D20703D5DBB283F3118870BDEA
:10710000726892B272B9D4E909518D421ED0A06959
:107110000844F06014D9691A89B27160A56200222E
:1071200084F86C20326842F00102DBB2326083F3F3
:10713000118870BDA26ED36843F08003D36070BD28
:107140002069411A89B27160A262E8E7012284F8DD
:107150006C20D1E7036F03B118477047F8B590F87A
:107160008530012B1CD0002A164619DD0269436ABE
:1071700005460F46D41AB442A869A8BF344639461A
:107180001844224645F034FD6B6A2A692344361BB5
:10719000B3FBF2F0002E02FB10336B622744E9DCF4
:1071A000F8BD00BF90F88530012B2BD0036C53B392
:1071B00070B4EFF31183502282F31288066C3268A8
:1071C000D20704D5DBB283F3118870BC70477268B4
:1071D00092B272B9D0E909518D4220D084690C4431
:1071E000F46016D9691A89B271608562002280F84C
:1071F0006C20326842F00102DBB2326083F3118806
:1072000070BC70477047826ED36843F08003D360D0
:1072100070470469611A89B271608262E6E70122EF
:1072200080F86C20CEE700BF70B5094C236873B1BD
:107230000546002606E099681A681E73216090478B
:10724000236823B15A68AA1A002A1846F3DA70BDD7
:10725000A406012070B5204C2378012B00D070BD0E
:107260001E4B1B68002BFAD01D4D2B6828465B680F
:1072700098470028F3D01B4B1B4E1A68338892881E
:107280009A4219D31949096800224968EA622A68B2
:1072900003FB01F12846D3689847154A33885268A2
:1072A00001333380002ADAD0116893884A69134287
:1072B00018BF1B048B6170BD0D4B5B6800222270F0
:1072C000002BCCD00B499A8809781B68890748BFE6
:1072D00012049A6170BD00BFC84D00200C2B002025
:1072E000102B0020C04D0020C64D0020B84D0020BE
:1072F000B02A0020BC2A002008B5254B1B68DB04FF
:107300000AD5B5EE400AF1EE10FA12D19FED210A2E
:1073100044F0D2FE80B208BDDFED1F7AB4EEE70A7A
:10732000F1EE10FA1CDA9FED1D0A44F0C5FE80B2A2
:1073300008BDDFED197AB4EEE70AF1EE10FAE5D4F4
:107340009FED177AB4EEC70AF1EE10FA14D870EE7A
:10735000677A9FED147A9FED140AA7EE870AE4E797
:1073600070EE677A9FED117A9FED110AA7EE870AFA
:1073700044F0A2FE80B208BDDFED0E7A9FED0E7ADA
:1073800070EE677A9FED0D0AA7EE870ACDE700BF82
:10739000945700200080BB440000404200007A4423
:1073A00000E0824466BEFFBE0060BB4438DFFF3EA3
:1073B00000407A440000834466BEFF3E00A0BB4408
:1073C000F8B5C64B1D6815F004072DED048B40F091
:1073D0000081DFEDC38AC34C15F0200505D094F879
:1073E000805015F0020540F0908094F8B8309FED81
:1073F000BE8A13F0010340F0AC8094F8B920002A53
:107400007ED1D4ED2F7A9FEDB97ADFEDB96A67EEC0
:10741000877A94ED317AE8EEA67A38EEC77AC4ED31
:107420002F7A84ED307A65B194F8CC20D4F884308A
:10743000C4F8C83001218A4284F8BA1018BFC4F8D1
:10744000C030AC4B1E780E2E00F00781DFEDA47A21
:10745000002794ED377A94ED386A77EEC76AD4ED59
:10746000367AA6EE267A77EE676A84ED377AE6EE0C
:10747000267AC4ED367AC4ED357A0FB1C4ED307A90
:10748000D4ED396A94ED3B7A9FED9B5A94ED3C6ABA
:10749000C4ED397A77EEE66AF0EE475AD6EE855AB1
:1074A000F0EE477AE6EE257A94ED3A0AC4ED3B7A9F
:1074B00037EEC07AA6EE070A84ED3A0A44F0FCFDE6
:1074C00002B282EAE273A3EBE2739BB2092B7ED98C
:1074D000002AACBF0A380A3005B20E2EA4F8F450C8
:1074E00060D0242E09D1DFED857A94ED300A20EEAC
:1074F000270A44F0E1FD824B5880BDEC048BF8BDB7
:1075000084F8BA3084F8B9307BE7D4ED247AB4F843
:107510009430F8EEE77AC4ED217A002B00F08A80EF
:1075200007EE903ADFED746A9FED767AF8EEE77A2F
:1075300086EEA78AB4EEC78AF1EE10FA88BFB0EEE5
:10754000478A94F8B83013F001034FF001053FF477
:1075500054AF94F8B930002B56D094ED319A78EEB0
:10756000C99A002D3AD094F8BA30002B54D0D4EDFB
:10757000217A94ED320A5F4B1E7877EEC07A0E2E98
:10758000C4ED357A5FD094F8CC30002B75D0022B47
:1075900002D00FB1012B31D0D4ED357AF0EE698AEB
:1075A000012756E7DFED547A554C9FED540A28EE3B
:1075B000278A28EE800ABDEEC88A18EE103A23808A
:1075C00044F07AFDBDEC048B6080E580F8BD0025B9
:1075D00083E7444C0127D4ED1D8AFDE6454B1E7818
:1075E0000E2E2AD094F8BA509FED3D8A002DCAD1B4
:1075F000002FD1D094F8CC30002BCBD1F0EE697AAB
:107600000127F0EE698A24E794ED2F9A012384ED97
:10761000319A84F8B930A2E7002F56D0D4ED217A00
:1076200037EEE80A012330EE090A84F8BA3084ED17
:10763000320AA0E79FED2C8A83E7D4ED357A94F8DF
:10764000BA509FED278A9FED2D0A27EE800A44F05D
:1076500033FD2B4B0E269880C8E7DFED2B7A94ED97
:10766000217A274B27EE277A0027BDEEC77ADFED78
:107670001C7A17EE102A9A80EBE6002F8CD094ED3E
:10768000356A94F8CD30DFED216A07EE903A76EE58
:10769000688AB8EEE77A78EE897AF0EE698AF0EED9
:1076A000E77A67EE877AF4EEE67AF1EE10FAC4BF75
:1076B00068EE266A86EEA78AF7EE007A77EEC87A39
:1076C00067EEA97AE6EE087AC3E60A4B1E780E2E1C
:1076D0007FF462AFD4ED357A3D46B4E7CCF20020BA
:1076E00000000000A40601209A99993ECDCC4C3FA1
:1076F000CDCC4C3E9F2B00200000C842CDCCCC3DD1
:10770000A02B00206666663F0AD7233C00401C463B
:10771000F6F7F4B810B5044644F0CEFC81B220462A
:10772000BDE81040F6F7EAB8F8B54569002D67D016
:107730002C68236A1B7B002B40F09080D4E904174F
:1077400063684E68002F3ED030687A686FF300009F
:10775000306010686FF300001060087C0E68022231
:1077600002FA00F141F00C017160397C8A403968FD
:1077700042F00C024A605A686FF341025A605A683C
:107780006FF300025A60236A1B697BB1236A686C3D
:107790001B699847012800F09D80022801D005E070
:1077A0002362236ADA691433002AF9D1236ADA6979
:1077B0003ABB586918B399692162C3E90522BDE84B
:1077C000F840F2F777BF9A681006FCD49A68D2079F
:1077D00013D430686FF300003060087C096802221F
:1077E000824042F00C024A605A686FF341025A60CC
:1077F000236A1B69002BC9D1D8E7DA68E6E7206263
:10780000F8BD226A94F82410127B1433D2B223629A
:10781000002932D1002A51D12846F2F763FE2968A7
:107820000A6AD369002BEBD0D06953698C69002BAD
:107830004BD0012666732D68636083B268696381EB
:107840000028DDD092693C48C969002A0ABF024677
:107850000120002048734A604B81F8BDAB68002BC3
:107860003FF46CAFD4E904171A689B8893614E68A3
:107870006368002F7FF468AFA5E72E68376AB069A8
:10788000B9683B68002B48D04FF0010C80F80DC060
:1078900043608BB229684381496951B1F0697968C5
:1078A0004381254B00290ABF19460123002341606B
:1078B0004373002384F82430002AADD0AB68002B3A
:1078C000AAD01A689B889362A6E71E461B4BFF2727
:1078D0001F70AFE7236A2968143B23620A6AD369E1
:1078E000002B3FF463AFD66953698F69E3B18446D7
:1078F00087F80DC07B60B3B22E687B817669002E5D
:107900003FF454AFC96992694B810B4B002A04BF05
:1079100000201A4648734A6048E79C46074B4FF0E0
:10792000FF0E83F800E0B1E79C46044B4FF0FF0EDA
:1079300083F800E0DCE700BF243C00201A010020AF
:107940008160F5F7E3B900BF0171F5F7DFB900BF5A
:107950002DE9F84FB44C94F8B830DB072DED028BCD
:10796000804679D5B14B94F8F6501F88B04E012D62
:107970005FD0022D38D0002D44D094ED428AF37BA5
:1079800033B1B38923B1AB4B1B78002B40F0E880B7
:1079900094F8F720AA4238BF2A46317A632907D8DB
:1079A000022D00F0FD8094F80031002B40F00E8194
:1079B000A14BDFEDA26A1A70D4E94630C4F81C313D
:1079C0001B1A07FB03F307EE903AF8EEE77AB0EEE6
:1079D000487AA7EEA67AB17B84ED427A002970D16D
:1079E000BDEC028BBDE8F88FB4F8FA30BB42C4D2CC
:1079F000934B94ED428A1B68C4F80C31012584F83E
:107A0000F650BCE7B4F8FC30BB421ED38C4BD4F824
:107A10000C111A68F37D03EB830303EB8303521A03
:107A2000B2EB830FA9DB012594ED428A84F8F6506E
:107A3000A5E7B4F8FE30BB4280F09E80B4F8F83081
:107A4000BB423CBF002584F8F6507D4B94ED428A42
:107A50001B68C4F80C3192E794F8F650DFF8CC912B
:107A6000EB1E012B39D9B9F80800C0F30B0043F025
:107A700095FB092840F3C1806D4EB9F80070F3887A
:107A80009F4203D33288BA42BFF471AFB7EB430FC2
:107A90003FF76DAF0323DFED6B7A664A84F8F6306B
:107AA00084F8F7300023B0EE678AC4ED427A137091
:107AB000A4F8F830A4F8FA30A4F8FC30A4F8FE30AA
:107AC00092E0012A00F09280022A89D1BDEC028B5B
:107AD0000720BDE8F84F0AF04DBC554EB9F80070CC
:107AE000F3889F4202D33288BA4202D2B7EB430FE7
:107AF00076DDB9F80800C0F30B0043F04FFB09280E
:107B000040F38F80337D002584F8F65084F8F750D9
:107B1000002B00F09D80474A137099B2B288738899
:107B200012FB01F213FB01F3717C92B28A429BB209
:107B3000A4F8F82086BF521A92B200228B42A4F811
:107B4000FA3086BF5B1A9BB20023A4F8FE30642390
:107B500084F801310023A4F8FC20C4F8043106E7BE
:107B600011F0D6F900284CD102239D422A4684F810
:107B7000F73038BF1A4610E7314BD4F80C111A68A9
:107B8000337E03EB830303EB8303521AB2EB830FC1
:107B9000FFF6F3AE022594ED428A84F8F650EEE645
:107BA00094F8000190B90123C4F8048184F80031ED
:107BB000254BC1F1640100FB01F183FB0103C917EF
:107BC000A1EBA351643184F80111F1E6D4F804016A
:107BD0001E4BA8EB00009842EADB84F80111E7E6AF
:107BE000032D7BD194ED428A0325C8E6BDEC028BC0
:107BF0000820BDE8F84F0AF0BDBBB9F800700C4E84
:107C0000B5E6337C834207D301239D422A4684F89C
:107C1000F73038BF1A46C0E6002384F8F7302A460A
:107C2000BBE6032DDED0A8E6A406012070FA0020F2
:107C300064F000206DFA00206CFA0020ACC52737F4
:107C4000A82A0020000000006BCA5F6B8096980095
:107C5000274A284D126892F96C103288B7FBF2F26D
:107C60000132082A28BF08225FFA82FC914285F877
:107C700000C02BD051B3204991F800E00EF1010172
:107C800001F00301714521D0DFF870B04FF0FF30F3
:107C90004FF0A40A0AE0B0F1FF3F02D1002B08BF69
:107CA0000846013101F00301714512D00AFB01B30E
:107CB00093F96C309A42EED10846C0B2F9F76EF8EB
:107CC0002B78B9F8007094F8F65026E71D46634605
:107CD00023E7431CF1D1634600251EE7B9F80800ED
:107CE000C0F30B0043F05AFA09283FF7C6AE44E64A
:107CF000E45F00206DFA0020805700200CED00208A
:107D00002DE9F843CE4CA36820469847002800F0A0
:107D10008F80B4F90E30A17D06EE903AB4F91030A0
:107D200007EE903AB4F9123007EE103AF8EEE66A30
:107D3000F8EEE77AB8EEC77A0123092984F85430BF
:107D4000C4ED126AC4ED137A84ED147A72D004F192
:107D5000480027F0C5FCBB4DAA8DAB6A002A40F055
:107D6000F980B94A1268520700F1C180B3F90020C6
:107D700094ED125A94ED136A94ED147A05EE902A5C
:107D8000B3F90220B3F9043006EE902A07EE903AD8
:107D9000F8EEE55AF8EEE66AF8EEE77A75EE655A1F
:107DA00076EE666A77EE677A2B88C4ED125AC4EDD8
:107DB000136AC4ED147ADBB395ED025A95ED056AAA
:107DC00095ED087AD5ED033A95ED064AD5ED094AC9
:107DD00075EEC55A76EEC66A77EEC77AA5EEA35A57
:107DE000A6EE846AA4EEA77AD5ED015AD5ED046A11
:107DF000D5ED077A85ED025A35EE652A76EE662ACC
:107E000037EE673AE3EE825AE2EE846AE4EE837A72
:107E1000C5ED015AC4ED125A85ED056AC5ED046A37
:107E2000C4ED136A85ED087AC5ED077AC4ED147ABE
:107E3000BDE8F883D4ED0B5A94ED0C6A94ED0D5A1D
:107E4000D4ED094A94ED084A804B67EEA55A27EE17
:107E5000866A67EE857A94ED0A5A1B78A6EEA46AC4
:107E6000E6EE845AE6EE857AD4ED0E6AD4ED0F4A3A
:107E700094ED105AE6EE875AF0EE466AE4EE876A11
:107E8000E5EE077AC4ED125AC4ED136AC4ED147A14
:107E9000002B7FF460AF6E4B93ED055A93ED036AB0
:107EA00093ED047AD3ED014A93ED004A26EE866AFB
:107EB00026EE877A66EE856A93ED025AA5EEA47ADD
:107EC000E5EE856AA5EE846AD3ED064A93ED075A7E
:107ED000D3ED085AA7EEA46AA7EE857AE7EEA56A65
:107EE00084ED126A84ED137AC4ED146A33E7594EB7
:107EF000B6F82C21322A63D0002A40F0CF8096F8C1
:107F00004A21002A3FF432AF06F59E7007C8524F4F
:107F10004FF0000C87FB028E86F84AC1D217A68963
:107F2000C2EB2E12921B9A8087FB0062C017C0EB37
:107F3000221087FB0127C917C1EB27111880598030
:107F4000464B0122A3F80EC0C3F80A20F9F718F92E
:107F5000AB6A0BE7B2F5C87F00F084803D4994ED31
:107F6000127AD1ED486AD4ED137A94ED146AF8EEE2
:107F7000E66A002676EE876A91ED497AA664B8EE45
:107F8000C77AFDEEE66A37EE277AD1ED4A7AC1ED7F
:107F9000486AF8EEE77ABDEEC77A77EE867A002077
:107FA000FDEEE77A012A188081ED497AE66458806F
:107FB000C1ED4A7A2665988075D0013AAA85D0E647
:107FC0001A68C6F83021B3F90420A6F83421234AF0
:107FD000DFED237AD268C6F8382194ED127A0020BA
:107FE000002177EE877AA0641980B6F82C21FDEE87
:107FF000E77A322AC6ED4F7A00F0828096ED507A09
:10800000D4ED137AD4ED146AE064B8EEC77A012A8D
:1080100037EE277AD6ED517A5980F8EEE77ABDEE41
:10802000C77A77EEA67A2065FDEEE77A998086ED2D
:10803000507AC6ED517A74D0013AA6F82C215EE749
:10804000D0F2002020600020945700204904002036
:10805000C85A0020A40601201F85EB5198F000208B
:1080600000000000D4ED126A94ED137AD4ED147A76
:10807000364EFDEEE66ABDEEC77AFDEEE77A0020E9
:108080000021A064C6ED486A198086ED497AE06453
:108090005980C6ED4A7A206599808EE7D6ED4F7AF1
:1080A000F8EEE77A99E717EE906ADFF8A8E0B4F8FF
:1080B0000C80C8368EFB061916EE90CAF11717EE23
:1080C000107AC1EBE9110CF1C80CA1EB0801998001
:1080D000C8378EFB0C614FEAEC7CCCEBE11C8EFBCD
:1080E000071EFF17C7EBEE17A3F800C05F80184B01
:1080F000C3F80A20D881F9F743F8AA8DAB6A5CE788
:1081000094ED137AD4ED147AE064BDEEC77AFDEEF7
:10811000E77A598086ED507A2065C6ED517A9980CC
:108120008AE70B2086F8492186F848110AF022F9DF
:10813000AB6AD6F830211A60B6F934219A80044A25
:10814000D6F83811D160B6F82C2175E7A4060120C5
:1081500098F000201F85EB51244B82B09A79019052
:1081600092B393F82630DFED226A224A07EE903A66
:10817000F8EEE77A204B127886EEA77A83ED667ADE
:1081800002B3B3F85611DFED1D6ADDED017A07EE9B
:10819000101AB8EE477AF8EE677A27EE267AF7EEED
:1081A000006A27EE277A03F5AC7377EE266A002182
:1081B000C7EE267A03EBC2021960083343ED017A59
:1081C0009A42F9D102B070470D4A12681201F9D5EE
:1081D00093F82630DFED066A07EE903AF8EEE77A7C
:1081E000054B86EEA77A83ED667AEBE7DC3C002050
:1081F0005555554068580020A406012027D4D23692
:108200009457002010B5437B82680446581C607365
:10821000D154627B237B934206D82AB12368D4E9E8
:10822000010198470023637310BD00BF427B42B138
:1082300010B503680446D0E9010198470023637331
:1082400010BD704730B5056895F800E0BEF1010F2C
:1082500095B004468C4608D0BEF1020F02D11946F3
:108260002B6A7BB1002015B030BD95F90400411C8C
:10827000F8D00328F6DC217900926246F5F71AFC63
:1082800015B030BDCDE90A210DF10F020492012293
:10829000CDE90532CDE908336CF07F018DF81C3053
:1082A0008DF830208DF844200D9310931293002206
:1082B0000023CDE90E238DF80F10EFF3118C10235E
:1082C00083F3128803681B6A0BB3069B04A802465B
:1082D0001BB1D3691432002BFBD12B6A6BB19968A7
:1082E00039B99A4209D0196829B15B68996800299F
:1082F000F7D01433F3E7C3E900405FFA8CFC8CF34A
:1083000011882268136A002BFCD10120ABE704AB73
:108310002B625FFA8CFC8CF31188F2F7CBF9F0E753
:1083200030B593B00DF1070508920022CDE9025255
:10833000CDE906228DF807108DF81420012109934C
:108340000B920E9210920023002204918DF82810B7
:108350008DF83C10CDE90C2301680446EFF3118C35
:10836000102383F3128803681B6A0BB3049B02A8D3
:1083700002461BB1D3691432002BFBD10B6A6BB1DF
:10838000996839B9934209D0196829B15B6899682D
:108390000029F7D01433F3E7C3E900405FFA8CFCFF
:1083A0008CF311882268136A002BFCD113B030BD06
:1083B00002AB0B625FFA8CFC8CF31188F2F77AF94E
:1083C000F0E700BF30B40568EFF3118C102383F39E
:1083D000128803681B6AEBB18B6804460A461BB11E
:1083E000D3691432002BFBD12B6A6BB1986838B972
:1083F000934209D0186828B15B6898680028F7D0C4
:108400001433F3E7C3E900415FFA8CFC8CF3118865
:1084100030BC704729625FFA8CFC8CF3118830BC49
:10842000F2F748B9F0B5056895F800C0BCF1010F46
:1084300093B0044608D0BCF1020F02D12E6A002E80
:1084400043D0002013B0F0BD95F90450681CF8D05B
:10845000032DF6DC684E542005FB00F006EB000E01
:10846000DEF81870002FECD02479CEF8242000F12B
:108470001C0232449BB2CEF820200022AEF82AC063
:10848000AEF81C108EF83420AEF82C308EF8362062
:1084900040F671038EF83620BA6911044FD4542384
:1084A00003FB056393F83630DBB2002B5DD0542319
:1084B00003FB0563012283F8362093F83610C9B216
:1084C000002969D1012013B0F0BDCDE908230DF1D9
:1084D000070302930123CDE9036361F07F018DF867
:1084E00028308DF83C3000220023CDE90666CDE926
:1084F0000C238DF807108DF814600B960E961096CD
:10850000EFF31186102383F3128803681B6A002B94
:108510006AD0049B02A802461BB1D3691432002B17
:10852000FBD12B6ACBB1996839B9934215D0196840
:1085300089B15B6899680029F7D01433F3E7013BF0
:10854000AAD1542303FB0563122283F8362093F843
:108550003630DBB2A9E7C3E90040F6B286F31188F2
:108560002268136A002BFCD1ACE76100542404FBA1
:108570000564183084F83530032323634FF4005228
:108580003044F5F731FAA269136843F0F60313603B
:1085900094F83610C9B293E7542303FB0563002215
:1085A000986983F8362040F671038269920610D5E7
:1085B000542303FB056595F8363020230129C36158
:1085C0003FF43FAF0D4A138801339BB20020138064
:1085D00038E7013BE9D1542303FB0565122385F8F5
:1085E000363095F83630E8E702AB2B62F6B286F308
:1085F0001188F2F75FF8B3E7D43A0020AC4D0020C1
:1086000030B58BB04FF0010C00910021CDE9012372
:10861000CDE90411CDE9061105688DF80CC00446BA
:108620008DF820C00991EFF3118C102383F3128889
:1086300003681B6A0BB3029B684602461BB1D369F1
:108640001432002BFBD12B6A6BB1996839B9934274
:1086500009D0196829B15B6899680029F7D01433EB
:10866000F3E7C3E900405FFA8CFC8CF311882268C1
:10867000136A002BFCD10BB030BDC5F820D05FFAD7
:108680008CFC8CF31188F2F715F8F0E730B593B055
:1086900000238DF807108DF806200DF10601012248
:1086A000CDE90332CDE90631CDE908320DF10705F8
:1086B0008DF814308DF828208DF83C200B930E9304
:1086C000109300220023CDE90C2301680295044693
:1086D000EFF3118C102383F3128803681B6A0BB32A
:1086E000049B02A802461BB1D3691432002BFBD1B4
:1086F0000B6A6BB1996839B9934209D0196829B1ED
:108700005B6899680029F7D01433F3E7C3E90040A8
:108710005FFA8CFC8CF311882268136A002BFCD161
:1087200013B030BD02AB0B625FFA8CFC8CF3118886
:10873000F1F7C0FFF0E700BF2DE9F04F05682F7893
:10874000012F85B008D0022F02D12B6A002B3CD01C
:10875000002005B0BDE8F08F95F9045090F804A012
:108760008DF80F20681CF3D0032DF1DCB34C54239B
:1087700003FB054398690028EBD00E460DF10F016D
:108780000022596202211A6383F83470998583F8B4
:10879000362083F8362042F211738269120418D40D
:1087A000542303FB054393F83630DFB2EFB1542373
:1087B00003FB0543012283F8362093F83630DBB201
:1087C000002B40F0EE800120C3E7FFF75FFF0120A0
:1087D000BFE7013BE1D1542303FB0543122283F899
:1087E000362093F83630DFB2E0E74FF0540808FB4C
:1087F00005F808F118004FEA4A0AA04420445146FF
:108800004FF400520190F5F7EFF8D8F818100198DE
:1088100088F8367042F211738A69970711D554238C
:1088200003FB054393F836805FFA88F7BFB1542302
:1088300003FB0543022283F8362093F83630DBB27F
:10884000BEE7013BE8D1542303FB0543122283F822
:10885000362093F836805FFA88F7002FE7D18E62D2
:10886000542606FB054696F83630002B40F0D5809E
:10887000338D013B9BB2338596F834304FF02A0993
:1088800009FB05F94B44143304EB43035A88013ABE
:1088900092B25A8096F834304B44143304EB4303BD
:1088A0005B889BB2002B4BD0B8464FF0120B06F101
:1088B0003607B16987F8008042F211738A6992071E
:1088C0005CD53B78DBB2002B40F0AE8096F834C02C
:1088D00005EB4502C2EBC2026244083254F822C0E2
:1088E0000CF1010E44F822E09CF800208A62328DDF
:1088F000013A92B2328596F834204A44143204EB9D
:108900004202B2F802C00CF1FF3C1FFA8CFCA2F844
:1089100002C0328D92B24AB996F834204A441432D9
:1089200004EB4202528892B2002A5FD196F83430AA
:108930004B44143304EB43035B889BB2002BB8D148
:10894000542303FB05430022996983F8362042F241
:1089500011738A69900618D5542303FB054393F8D5
:108960003630DBB2002B6DD0542303FB05430622C7
:1089700083F8362093F83630DBB221E7013B9DD1F6
:1089800087F800B03B78DBB29DE7013BE1D154238F
:1089900003FB0543122283F8362093F83630DBB20E
:1089A000E0E7542303FB05430022996983F836204E
:1089B00040F671038A6992060DD5542303FB0544E2
:1089C00094F836301E4A2023CB61138801339BB2C2
:1089D00000201380BDE6013BECD1542303FB05448A
:1089E000122384F8363094F83630EBE73B7042F2CD
:1089F00011738A69120609D53A78D2B2002A3ED19B
:108A000051460190F4F7F0FF01988FE7013BF0D158
:108A100087F800B03A78D2B2F0E7032386F8363010
:108A200096F83630DBB2CBE6542303FB0543042231
:108A300083F8362093F83630DBB2C1E6D43A002012
:108A4000AC4D00202022CA614A6863F309024A60E3
:108A50004A6863F30C324A604A6863F317424A601B
:108A60004A6863F318624A604A6863F38A225423AF
:108A700003FB05434A6093F83630DBB2A0E654238B
:108A800003FB0543052283F8362093F83630DBB22A
:108A900096E600BF30B595B000230122CDE905323E
:108AA000CDE908338DF81C300D93109312930DF11E
:108AB0000F030DF107050B928DF830208DF844203F
:108AC0000A93002200238DF80710CDE90E230168D8
:108AD00004950446EFF3118C102383F31288036886
:108AE0001B6A1BB3069B04A802461BB1D369143250
:108AF000002BFBD10B6A6BB1996839B9934209D04D
:108B0000196829B15B6899680029F7D01433F3E735
:108B1000C3E900405FFA8CFC8CF311882268136A69
:108B2000002BFCD19DF80F0015B030BD04AB0B62DB
:108B30005FFA8CFC8CF31188F1F7BCFDEEE700BF07
:108B4000154A164B90421B6828BF1046B0EB930F96
:108B500014D2B0EBD30F13D2B0EB131F12D2B0EB81
:108B6000531F11D2B0EB931F10D2B0EBD31F0FD213
:108B7000B0EB132F0ED24FF4807070470220704775
:108B8000042070470820704710207047202070474D
:108B900040207047802070470051250200000020CF
:108BA000013903292CD81B4B4FF0280C0CFB01FC7E
:108BB00010B403F5CE746344644493F89C210460BC
:108BC0004FF0010C022A80F838C003F5CE7419D09A
:108BD000C9B2114A09015258C3F8A02172B1022248
:108BE00083F89C2100F110014FF480722430A2819F
:108BF000C3E96D1060465DF8044B70470020FAE74A
:108C00000020704793F8A9216244604683F8A921A7
:108C1000F1E700BFA40601209C3C00202DE9F04FA5
:108C2000DFF88482DFF884B29C4C85B04FF0010AF3
:108C30004FF0000998F80030022B0DD009F101091E
:108C4000B9F1040F0AF1010A08F128080BF1050B2C
:108C5000F0D105B0BDE8F08F9BF903506A1C00F01D
:108C6000E480EDB228465FFA89F30D2D62D88C4A74
:108C7000002104E00131202902F103025AD01778C3
:108C8000002FF7D156789E42F4D1854A854E01EBEC
:108C90004101114405EB4502897806F8221006EBE4
:108CA00082026E009160526861688A4200F0CF8053
:108CB000A16A8A4200F06281E16C8A4200F062811E
:108CC000216F8A4200F06781D4F894108A4200F044
:108CD0006C81D4F8B8108A4200F07581D4F8DC10A9
:108CE0008A4200F06C81D4F800118A4200F072814F
:108CF000D4F824118A4200F07681D4F848118A42CF
:108D000000F06C81D4F86C118A4200F07E81D4F8B6
:108D100090118A4200F07481D4F8B4118A4200F0B4
:108D20008181D4F8D8118A4200F0818114F80C2C8A
:108D3000002A7DD00135EDB2854296D900230193FA
:108D40009BF904506B1C79D0EDB22E465FFA89F284
:108D50000D2D62D8524B002104E00131202903F18E
:108D600003035AD018780128F7D15F789742F4D1DD
:108D70004B4B4C4F01EB4101194405EB45038978FE
:108D800007F8231007EB83034FEA450E99605B68F1
:108D900061688B4200F08C80A16A8B4200F0F68003
:108DA000E16C8B4200F0F480216F8B4200F0F78081
:108DB000D4F894108B4200F0F580D4F8B8108B42B0
:108DC00000F0FA80D4F8DC108B4200F0F280D4F886
:108DD00000118B4200F0FB80D4F824118B4200F08C
:108DE0000B81D4F848118B4200F00281D4F86C1149
:108DF0008B4200F01381D4F890118B4200F00A816D
:108E0000D4F8B4118B4200F01B81D4F8D8118B42F6
:108E100000F0128114F80C3C9BB10135EDB2AE426A
:108E200096D20023C8E9043308E70D2000251AE78D
:108E3000142204F80BAC04F80C2C7BE70D2600255B
:108E400084E7132304F80BAC04F80C3CE5E73A463E
:108E5000BC460CEBCC0104EB81070CF1010197F847
:108E600018C0019107F11801BCF1000F7FF462AF47
:108E7000142322440B70019887F819A0C8F8102019
:108E8000F2F714F807493A6A731901EB83039968FA
:108E9000136861F30603136052E700BF1C01002052
:108EA000CCDA05081403002040080120545A0020A1
:108EB0000021084600EBC00304EB830301301F7E52
:108EC00003F1180C002FA8D113222144764683F811
:108ED00019A08CF80020C8F8141003930290F1F741
:108EE000E5FF33462B441D46039B1A6A564B03EBA2
:108EF00085039968136861F306031360DDE90130A7
:108F0000002B8ED0D8F8142053681D6867F3000535
:108F10001D60137CD8F810501268D5F804C00221E7
:108F200001FA03F343F00C035360DCF800E067F34D
:108F3000000ECCF800E095F810C02D6801FA0CF195
:108F400041F00C016960D8F818501026C5E9026795
:108F50002F82D8F804106F600C312960D8F81C50AB
:108F60003B46C5E90017C5E9027738492F823A46E2
:108F7000F1F7BAFF012388F80C305FE624224FF0A6
:108F8000010C66E748224FF0020C62E7242191E7CA
:108F9000482102208EE76C224FF0030C59E76C2128
:108FA000032087E79021042084E790224FF0040CEF
:108FB0004FE7D82106207DE7B42105207AE7D822A3
:108FC0004FF0060C45E7B4224FF0050C41E7FC21B9
:108FD00007206FE7FC224FF0070C3AE74FF4A2722C
:108FE0004FF0090C35E74FF490724FF0080C30E762
:108FF0004FF4A27109205DE74FF49071082059E702
:109000004FF4C6724FF00B0C23E74FF4B4724FF0DD
:109010000A0C1EE74FF4C6710B204BE74FF4B471F6
:109020000A2047E74FF4D8724FF00C0C11E74FF4C9
:10903000EA724FF00D0C0CE74FF4EA710D2039E79E
:109040004FF4D8710C2035E714030020297701086C
:1090500010B5036804469B689847FF230122A37359
:10906000627310BD036810B504461B6898472368F7
:1090700001219B6820469847E37B0133E37310BDD1
:10908000F0B583B00446089F0193384616460D4656
:1090900041F058FB2268E6722844A0729769019B50
:1090A000324629462046BC4603B0BDE8F040604742
:1090B00003689B6A184700BF03685B6D03B11847DC
:1090C000704700BF0368DB6C03B11847704700BFEF
:1090D000002310B5C37342748A6C016004460373A5
:1090E0000AB119469047236801219B68204698479A
:1090F000FF222368A273DB6C012262731BB120463E
:10910000BDE81040184710BD4A484B494B4BDFF8AB
:1091100030C12DE9F04F4FF0010A4FF002094FF036
:10912000040808271026202540244FF0800E30F830
:10913000022F12F0010F03D01960A3F804A0083326
:1091400012F0020F03D01960A3F80490083312F054
:10915000040F03D01960A3F80480083312F0080F3D
:1091600002D019609F80083312F0100F02D01960EE
:109170009E80083312F0200F02D019609D800833C2
:1091800012F0400F02D019609C80083312F0800F5B
:1091900003D01960A3F804E0083312F4807F05D0EF
:1091A0004FF4807B1960A3F804B0083312F4007FF9
:1091B00005D04FF4007B1960A3F804B0083312F413
:1091C000806F05D04FF4806B1960A3F804B00833AA
:1091D00012F4006F05D04FF4006B1960A3F804B0CF
:1091E000083312F4805F05D04FF4805B1960A3F858
:1091F00004B0083312F4005F05D04FF4005B19602F
:10920000A3F804B0083312F4804F05D04FF4804B1C
:109210001960A3F804B00833D20B04D04FF4004215
:1092200019609A80083301F5806161457FF47FAF52
:10923000BDE8F08FFADC0508000002401838002075
:109240000020024010B50409013C072C16D80D4A35
:1092500032F8141000F00F0341FA03F212F0010289
:109260000ED0012098400138084041F097FF064B8E
:10927000064A1B5D184402EBC00010BD002010BD63
:10928000104610BDFCDC05080CDD05081838002070
:10929000F8B50C4F97F834308BB10B4C0025A6680D
:1092A00030790135FFF7CEFF18B1217DF279F1F762
:1092B000E7FF97F83430AB4204F14C04EFDC0120B7
:1092C000F8BD00BFE8440020C41A002038B50546A8
:1092D00000780C46FFF7B6FF611CC9B2044610B116
:1092E00041238371C17120466978F1F743FFAB7860
:1092F00020461BB1BDE83840F1F760BCBDE83840FE
:10930000F1F762BC0D4B2DE9F0411F680C4E05468C
:109310000024A74201DCBDE8F08104EB440303EB29
:109320000608F05CFFF78EFF854204D121464046D7
:10933000BDE8F041CAE70134EBE700BF9C5A0020CA
:109340006C5A0020054B53F8203033B11A689B88C3
:1093500051690B4218BF1B0493617047B02A00206B
:109360000C4B0D4A93F800C052F820200123834093
:1093700003EA0C0341B1003B18BF01231AB19188E5
:1093800033B1136899617047B3FA83F35B09F5E76A
:109390000904F6E7BC2A0020B02A002010B5054CCD
:1093A00023681B6998472368002283F836209A6354
:1093B00010BD00BFA864002010B5084C236893F8C6
:1093C000352012B1DB68984700B910BD044A236804
:1093D00012689A63012183F8361010BDA86400203A
:1093E000A82A002038B50C4614F8011B41B10546E7
:1093F0002B6828461B68984714F8011B0029F7D1F1
:1094000038BD00BF03681B68184700BF03682DE91B
:10941000F0415F6A1FB13B46BDE8F0411847044682
:109420000D46164600E023689B6820469847B042E8
:10943000F9D3002E08DD2E44236815F8011B1B68A4
:1094400020469847B542F7D1BDE8F08103685B68D4
:10945000184700BF03689B68184700BF0368DB68B4
:10946000184700BF03685B69184700BF03689B6A21
:1094700003B11847704700BF0368DB6A03B11847A0
:10948000704700BF03682DE9F04116469A6A04460A
:109490000D460AB1904723685F6A5FB1324629469C
:1094A0002046B8472368DB6AC3B12046BDE8F041D7
:1094B000184723689B6820469847B042F9D3002E8E
:1094C000F0DD2E44236815F8011B1B6820469847E1
:1094D000B542F7D12368DB6A002BE6D1BDE8F08105
:1094E00070B504460E461546236820469B6898478B
:1094F000A842F9D32A4631462046BDE87040C1E76C
:109500002DE9F843456FC04F95F800C017F91CE0EE
:109510005FFA8EF30D2B044640F29B80006C00280E
:1095200049D0BA4E7368834200F00881B36A98420A
:1095300000F06081F36C984200F06281336F9842D2
:1095400000F06E81D6F89430984200F06B81D6F826
:10955000B830984200F06A81D6F8DC30984200F0CA
:109560006981D6F80031984200F06881D6F824313C
:10957000984200F06981D6F84831984200F068813D
:10958000D6F86C31984200F06581D6F89031984257
:1095900000F06481D6F8B431984200F06581D6F8C5
:1095A000D831984208BF0D2700F0C98016F80C3C4E
:1095B000002B00F00E81E36B002B48D0934E7268B5
:1095C000934200F08E80B26A934200F01581F26CF3
:1095D000934200F01381326F934200F01381D6F86A
:1095E0009420934200F02081D6F8B820934200F0F6
:1095F0001F81D6F8DC20934200F01E81D6F80021AE
:10960000934200F01D81D6F824219A4200F01A817D
:10961000D6F84821934200F01981D6F86C21934284
:1096200000F01A81D6F89021934200F01981D6F803
:10963000B421934200F01681D6F8D821934208BF96
:109640000D234FD016F80C3C002B00F0CA80BDE86B
:10965000F8836F4B00211E461A4604E00131202991
:1096600002F103023BD010780428F7D1507860450E
:10967000F4D101EB410131440EEB4E00654A89788B
:1096800002F8201002EB800250689160216520648E
:1096900007EB4C0797F9012001323FF440AF00225D
:1096A00005E00132202A03F103033FF438AF1978B3
:1096B0000529F6D159786145F3D102EB42023244D3
:1096C000544B92780EEB4E0E03F82E2003EB8E0EC9
:1096D000DEF80430CEF80820E363E2641FE7206C74
:1096E000D6E7002303EBC30306EB83082A789F0029
:1096F00098F818300132D2B2002BA8D1F059464B5D
:1097000088F8192098420CBF362038200C2388F89E
:1097100018303FF055F9F259D2F8003143F0010307
:10972000C2F80031D8F82030E16C1A6861F3060203
:109730001A606B6804336366BDE8F883002707EBA3
:10974000C70706EB87080CF1010C98F818305FFA90
:109750008CFCBF00002B7FF42EAFDFF8BC90F059DB
:1097600088F819C00B2348450CBF3620382088F8EC
:1097700018303FF025F9F359D3F8002142F00102E7
:10978000C3F800214B450CBF36203820D8F82030D4
:10979000226D196862F30601196095F82F903FF069
:1097A0000FF9F2591D49D2F8003143F00103C2F814
:1097B000003198F91100C8F80C10C9F301124FEAF2
:1097C0009911C8F8144039F021FA6B680433236604
:1097D000F1E60B230CF1010C06F80C3C06F80BCC5F
:1097E000E9E62B780C22013306F80C2C06F80B3C2A
:1097F000BDE8F8830127A2E7012373E7022371E79D
:1098000002279CE703236DE7046700201C0100206A
:10981000CCDA05081403002000640240C1B100083E
:1098200003278CE704278AE704235BE7052786E7FD
:10983000052357E7062782E7062353E707277EE736
:1098400007234FE708234DE7082778E7092349E76F
:10985000092774E70A2772E70A2343E70B276EE715
:109860000B233FE70C233DE70C2768E7324B70B52D
:109870001D68EB6BAC6E002B3ED02368580605D5F7
:109880006FF04003236095F8856086B12B6C03B3BD
:1098900023681A0744BF236863682368DB0605D57D
:1098A0006B6B0BB19847AC6E2368636870BD95F81D
:1098B0007A00FFF7C7FCE36866F3C303E3600123A4
:1098C00085F885300028E1D02821F1F725FCAC6E21
:1098D000DCE723681906DBD5D5E90923934216D0C6
:1098E000AA692969D25C0133D2B26260B3FBF1F29A
:1098F00001FB1233AB62CBE723689E06BDD5EB6A52
:1099000053B16068296B80B29847AC6EB5E7E368E5
:1099100023F08003E360BBE76368EA696969DBB24F
:109920008B54EB69EA68AC6E0133B3FBF2F102FBD6
:109930001133EB61A1E700BF24450020324B70B525
:109940005D68EB6BAC6E002B3ED02368580605D5E6
:109950006FF04003236095F8856086B12B6C03B3EC
:1099600023681A0744BF236863682368DB0605D5AC
:109970006B6B0BB19847AC6E2368636870BD95F84C
:109980007A00FFF75FFCE36866F3C303E36001233B
:1099900085F885300028E1D02821F1F7BDFBAC6EB9
:1099A000DCE723681906DBD5D5E90923934216D0F5
:1099B000AA692969D25C0133D2B26260B3FBF1F2C9
:1099C00001FB1233AB62CBE723689E06BDD5EB6A81
:1099D00053B16068296B80B29847AC6EB5E7E36815
:1099E00023F08003E360BBE76368EA696969DBB27F
